:020000040000FA
:1000000000020400000000003C9800003C98000042
:100010003C9800003C9800003C9800003C98000090
:100020003C9800003C9800003C9800003C98000080
:100030003C9800003C9800003C9800003C98000070
:100040003C9800003C9800003C9800003C98000060
:100050003C980000BA6C0000E06C00003C98000086
:100060003C9800003C9800003C9800003C98000040
:100070003C9800003C9800003C9800003C98000030
:100080003C9800003C9800003C9800003C98000020
:100090003C9800003C9800003C9800003C98000010
:1000A0003C9800003C9800003C9800003C98000000
:1000B0003C9800003C9800003C9800003C980000F0
:1000C0003C9800003C9800003C9800003C980000E0
:1000D0003C9800003C9800003C9800003C980000D0
:1000E0003C9800003C9800003C9800003C980000C0
:1000F0003C9800003C9800003C9800003C980000B0
:100100003C9800003C9800003C9800003C9800009F
:100110003C9800003C9800003C9800003C9800008F
:100120003C9800003C9800003C9800003C9800007F
:100130003C9800003C9800003C9800003C9800006F
:100140003C9800003C9800003C9800003C9800005F
:100150003C9800003C9800003C9800003C9800004F
:100160003C9800003C9800003C9800003C9800003F
:100170003C9800003C9800003C9800003C9800002F
:100180003C9800003C9800003C9800003C9800001F
:100190003C9800003C9800003C9800003C9800000F
:1001A0003C9800003C9800003C9800003C980000FF
:1001B0003C9800003C9800003C9800003C980000EF
:1001C0003C9800003C9800003C9800003C980000DF
:1001D0003C9800003C9800003C9800003C980000CF
:1001E0003C9800003C9800003C9800003C980000BF
:1001F0003C9800003C9800003C9800003C980000AF
:10020000FFFFFF00FFFFFF003C9800003C9800004C
:100210003C9800003C9800003C9800003C9800008E
:100220003C9800003C9800003C9800003C9800007E
:100230003C9800003C9800003C9800003C9800006E
:100240003C9800003C9800003C9800003C9800005E
:100250003C980000BA6C0000E06C00003C98000084
:100260003C9800003C9800003C9800003C9800003E
:100270003C9800003C9800003C9800003C9800002E
:100280003C9800003C9800003C9800003C9800001E
:100290003C9800003C9800003C9800003C9800000E
:1002A0003C9800003C9800003C9800003C980000FE
:1002B0003C9800003C9800003C9800003C980000EE
:1002C0003C9800003C9800003C9800003C980000DE
:1002D0003C9800003C9800003C9800003C980000CE
:1002E0003C9800003C9800003C9800003C980000BE
:1002F0003C9800003C9800003C9800003C980000AE
:100300003C9800003C9800003C9800003C9800009D
:100310003C9800003C9800003C9800003C9800008D
:100320003C9800003C9800003C9800003C9800007D
:100330003C9800003C9800003C9800003C9800006D
:100340003C9800003C9800003C9800003C9800005D
:100350003C9800003C9800003C9800003C9800004D
:100360003C9800003C9800003C9800003C9800003D
:100370003C9800003C9800003C9800003C9800002D
:100380003C9800003C9800003C9800003C9800001D
:100390003C9800003C9800003C9800003C9800000D
:1003A0003C9800003C9800003C9800003C980000FD
:1003B0003C9800003C9800003C9800003C980000ED
:1003C0003C9800003C9800003C9800003C980000DD
:1003D0003C9800003C9800003C9800003C980000CD
:1003E0003C9800003C9800003C9800003C980000BD
:1003F0003C9800003C9800003C9800003C980000AD
:100400004FD62100007F220000018800000000007C
:100410000C000700C0E028000100200011000700C8
:10042000000020000000E000020032000000020096
:1004300000000000A8960200000000000040DA0062
:100440000000FE004440A900A01620000000E000CB
:100450000300320000002000A00188004440A800F2
:100460000000060091018800800078000000EB0089
:1004700015003700E280400032A0B4009101BA00BC
:10048000E280400032A0B4009102BA00E280400055
:1004900032A0B4000002EB00472BDE00F507B200EB
:1004A000602CE10004003A000059EB008301E900F0
:1004B000FDFF3E00040037006128E100010032002A
:1004C0000082EB00040007001101BA000200E00006
:1004D000E8FF3A00000006003159BA008301E90044
:1004E0000C0032002159BA008301E90008003200F3
:1004F0000400E00003003A00E280400032A0B400B3
:10050000F5FF370011D9BA008301E900FAFF3A007C
:100510008100E800E180400032A0B4000000060045
:1005200000000000000000000000000000000000CB
:1005300000000000000000000000000000000000BB
:1005400000000000000000000000000000000000AB
:10055000000000000000000000000000000000009B
:1007D000889FBE008A9FBE00010578000100E000EE
:1007E0000400350008003C000000E000200032005A
:1007F0000500370060001000E080180002003B0098
:1008000001F02C001A0037000004BE006011B8008F
:100810006B0920000982CF00020039000882CF0056
:100820000441B000694252000E00320008003B0053
:1008300082817100610164008904D1000884D300C1
:100840008B05E8000442E800F9FF3A000500370094
:100850000804440089844C008B05E9000442E90047
:10086000FBFF3A000B0107000AF0A70001F0A0000F
:100870004F05BE004F04BE0000000600F4FF2F002D
:100880002A0137001400200028013700889FBE008D
:100890008A9FBE008C1F78003F010700460133008D
:1008A00003866C006450E1002E0032006420E100F9
:1008B000330032006150E1002F0032006120E1007E
:1008C0003100320085855500EB07B000090020009B
:1008D00008042000050037000804440089844C0007
:1008E0000A0031000603430087834B0000015300D8
:1008F00081815B00F8FF33000203BE000800A00006
:100900000804440089844C00F6FF3900C639DD0034
:100910008301730001003200130020008904D1001C
:100920000884D3000998A300050032000800A7003E
:100930000300A0008904D1000884D3008B05E800DF
:100940008904D1000884D3000001EB000281D200A9
:10095000D000070001F0A1000CF0A70001F0A000FA
:100960001E0137006420E100200132000801BE00B2
:100970000200BE00F7FF37006120E1001B013200DA
:100980006000B800F3FF37000000200001F82700E6
:10099000F0FF370003F0A200889FBE008A9FBE00D0
:1009A0008C1F7800FC000700030133006450E10055
:1009B0004F0032006420E1005200320003826C00DC
:1009C00007003B000905D0000306D000820F540049
:1009D0000C065D0002003900020032008901780037
:1009E000030678008582550004003D000003FD00E9
:1009F0008103FD008502EA008B854200840F7200AE
:100A000002003B0060001000E08018006011B80098
:100A10000005EB007A28E1000A00390006007800A2
:100A2000C75DDD00F707B200878075002D00370035
:100A3000828171000A017800610560008180D10027
:100A40000080D3008502E900F9FF3B000604400066
:100A50008784480002003B0060041400E0841C000E
:100A60000988A300070032008A8171008281710029
:100A7000610164008904D1000884D3008B05E8007B
:100A8000170037000978A30013003A000B00E000BC
:100A9000130034008B05E9000804440089844C00ED
:100AA0000A4474000978A3000D003A000B00E0002E
:100AB000070034008B05E9000804440089844C00D9
:100AC00001003A000B0020000978A300F7FF320074
:100AD0000001EB0002003700828171000A017800FA
:100AE0006C0007000CF0A70001F0A000BB0037006D
:100AF0006420E10002003A00838F6C00BB003300E9
:100B00000801BE000200BE00B4003700889FBE008E
:100B10008A9FBE008C1F78009F000700A60033004C
:100B200003866C006450E100240032006420E10080
:100B3000270032006150E100220032006120E10014
:100B4000210032008B854200EB07B1000134B80070
:100B5000003AB8000804420089844A00013AB8000B
:100B60000030B8008880400009014A0004003300CA
:100B70000000400081804800020149008B05E90027
:100B8000C909DD008301700001003200130020005C
:100B9000C814DE004814DD004709DE001200B20070
:100BA000C808DE00088470003A00070001F0A100C8
:100BB0000CF0A70001F0A000880037006120E100E0
:100BC0008A0032000801BE000200BE00F7FF3700B5
:100BD0006150E100FCFF3A00840037000001BE00D4
:100BE000850007000470A70003F0A10003F8A3002C
:100BF00013003A006509B100100032000900350009
:100C00006928E1000200350001002800000005000D
:100C100000004000818048008502E900FCFF3A00A6
:100C200000000600F88F4200050035008100D10069
:100C30000080D3008502E800FCFF3A0000000600B7
:100C40008000EB00000005006022B80006022000D2
:100C50000000D0008180D2000482D2008582D200C0
:100C60000000A0000202520083825A0003003100FB
:100C70000202420083824A000000A1000603E9004C
:100C8000F3FF3A0000000600EFFF07000400BE007B
:100C90000000060081002000618055000B003D002F
:100CA0000B00200061FE2F000100E1001D00340058
:100CB00082817100610164008904D1000884D3003D
:100CC0000000E800FAFF3A007100200061006400B3
:100CD000030070000200600009003200610444005B
:100CE000E0844C000988A500050032008B05E8006F
:100CF0006808E10002003A008904D1000884D300AA
:100D0000F20F20000258E10005003D00C75DDD0044
:100D1000F907B2008980750008007800000006001D
:100D20000BF827008B00780000000500889FBE00AC
:100D30008A9FBE00841F7800170007004F007800CC
:100D400011003300F0FF2F00838F6C0006003B0082
:100D5000040565000A00A7000800370009F0A60096
:100D60001000200008003700820F5400838F5C00C1
:100D7000030039001000200001003E0000002000A8
:100D800009F0A7000000EA004F05BE004F04BE00B6
:100D90000000E000000006000004BE00160007008E
:100DA0000003BE000405BE000200BE0012000700E2
:100DB000844F7500000006000200BE006450E10090
:100DC000050036006420E100020036000968A30037
:100DD00001003A000800BE000160A0004F06780044
:100DE0004F05BE004F04BE0000000600F0FF2F00BC
:100DF000F1FF2700F9FF3700C70ADE00F107B20054
:100E0000F50FB20008003200E1CF420002003200CC
:100E10000170A00024000500810F70000100320065
:100E20000408050044000500810F700002003A002C
:100E3000140005008502E9000000400081C0480060
:100E4000FCFF3B000170A000240005003E000000F4
:100E500008200000080000001B5B000044000000A8
:100E60001B5B000000440000001B00005B4300000F
:100E7000001B00005B3200004B0D0000004300002F
:100E8000000000001B5B000032440000005700001F
:100E9000617200006E6900006E6700003A20000079
:100EA0006E6F0000207600006F6C0000746100001F
:100EB00067650000206F00006E2000005670000083
:100EC000756C00006C7500007020000070690000F7
:100ED0006E000000203D000020000000565200007F
:100EE00045470000207400006F6F0000206C000078
:100EF0006F7700002C200000697300002074000050
:100F00006865000072650000206100002073000029
:100F1000686F0000727400003F0000002E20000087
:100F20003C0000002E200000000D00000A280000F8
:100F300000780000002900003E000000427500001B
:100F400073200000506900007261000074650000A9
:100F5000207600003300000046690000726D00003A
:100F6000776100007265000020760000362E0000D8
:100F700030200000723100003632000035200000C1
:100F80000020000028320000344600004A360000ED
:100F900034470000413000003032000020000000E3
:100FA00041330000004200003400000042350000E0
:100FB0000042000038000000554E00004B000000C9
:100FC0002900000049090000004F0000090000004E
:100FD00048090000004C000009000000456E0000B8
:100FE000746500007220000072610000772000002C
:100FF000766100006C75000065200000666F0000DF
:1010000072200000425200004700000030620000E1
:1010100000300000303000002C00000030300000B4
:10102000003000003132000033340000353600005B
:1010300037380000394100004243000044450000B9
:101040004630000078000000436F0000756C00001F
:10105000646E000027740000206B000065650000CE
:101060007020000075700000000000005350000068
:1010700049310000000000000029000000200000AD
:1010800057000000205200000049000032430000D9
:10109000310000003A200000000000002E00000097
:1010A00031570000303100000000000031410000E5
:1010B0004C53000000420000507600003300000056
:1010C00008080000080800000800000000000000F8
:1010D000204800007A0000000000000000410000ED
:1010E000525400003100000042420000494F00000D
:1010F00031000000524100005731000000000000A4
:101100004F430000443100000000000000000000D8
:1011100000000000290000000000000000000000A6
:101120002800FA000000EB00600F98000000EB00C0
:10113000006488000000EB00F0638800F06380002A
:10114000200798000000EB00100798000000EB005B
:10115000000F78000000EB00A04088000000EB00CA
:10116000500798000000EB00106488000000EB00BE
:10117000400798000000EB00000F980014003700B3
:101180000000EB00600798000B0037000E0890008D
:10119000EE0090004500DD008100400040C82000C6
:1011A000808040000040EB00804878006E00900096
:1011B0000000E800600798006E009000FF0F5000EC
:1011C000F2FF34000E0890000000E800000F9800C5
:1011D0000E089000E40F5000E9FF34000000EB001F
:1011E00020698800A1408000E00220000088B9004A
:1011F0006102200080804000C092200000804000FA
:101200003467020000000000D14080000020200070
:10121000008060000000E000040032007100200047
:10122000E0562000D6920200000000006072280004
:101230003467020000000000460437002069800087
:101240000000E00063003200206980000000E90037
:10125000206988000000EB00600798001E0037003E
:10126000F263800020698000EE0090004500DD0000
:101270008100400040C8200000804000904078007D
:10128000E0B720000000410001487800206980009C
:10129000EE0090004500DD008100400040C82000C5
:1012A0000080400010407800446C02000000000004
:1012B000F06380000000E800F06388006E0090009A
:1012C0000000E80060079800F1638000F00F200044
:1012D00000806000F063880020698000EE009000CC
:1012E0004500DD008100400040C820000080400033
:1012F000104078000004E000D9FF3A000000EB0045
:10130000206988003300370080AE2000104078004C
:10131000644060000004E0002E003200A140800024
:10132000E00220000088B900FA004000C0922000CE
:101330000080400010007800000001000000E00084
:1013400024003200A1408000E00220000088B900A3
:101350006102200080804000C09220000080400098
:101360003467020000000000607228003467020049
:101370000000000001648000F0638000808F500056
:101380001400320000648000600798000D003700F0
:10139000EE009000E0B72000008040001040780090
:1013A000446C020000000000EE009000F00F2000EE
:1013B00000806000600798006E0090000000E80068
:1013C00060079800EE009000F0638000808F50006E
:1013D000EFFF3A00666B0200000000000004E0002E
:1013E000C9FF32006E6C0200000000000004E00043
:1013F000030032007E6C020000000000D5033700BD
:10140000246C020000000000604F98006E489000BD
:101410000080FB006101B9000217980013179800C3
:10142000F0072000010020000E1190009E11900096
:10143000800F5100818F590052033E000E10900022
:101440009E1090000060010045033700FA0237004B
:10145000560137004B033700D8003700110337001F
:101460006B0137004703370077003700450337002B
:1014700027033700430337004203370024033700B4
:10148000160237003F033700720137003D03370073
:101490003C0337003B0337003A033700390337007A
:1014A000380337003703370036033700350337007A
:1014B00034033700020137003203370031033700AD
:1014C000300337002F0337002E0337002D0337007A
:1014D0002C0337002B0337002A033700290337007A
:1014E000280337002703370026033700250337007A
:1014F000240337002303370022033700210337007A
:10150000200337001F0337001E0337001D03370079
:101510001C0337001B0337001A0337001903370079
:101520001803370017033700160337001503370079
:101530001403370013033700120337001103370079
:10154000100337000F0337000E0337000D03370079
:101550000C0337000B0337000A0337000903370079
:101560000803370007033700060337000503370079
:101570000403370003033700020337000103370079
:1015800000033700FF023700FE023700FD0237007C
:10159000FC023700FB023700FA023700F90237007D
:1015A000F8023700F7023700F6023700F50237007D
:1015B000F4023700F3023700F2023700F10237007D
:1015C000F0023700EF023700EE023700ED0237007D
:1015D000EC023700EB023700EA023700E90237007D
:1015E000E8023700E7023700E6023700E50237007D
:1015F000E4023700E3023700E2023700E10237007D
:10160000E0023700DF023700DE023700DD0237007C
:10161000DC023700DB023700DA023700D90237007C
:10162000D8023700D7023700D6023700D50237007C
:10163000D4023700D3023700D2023700D10237007C
:10164000D00237005D003700016480002E0090005A
:10165000810F500055003200F16380002E00900091
:10166000810F500010003A00F06380008000E90014
:10167000F00F200000806000F0638800F1638000BC
:10168000E0B72000808040000040EB0080487800F8
:10169000F1638000210798008072280034670200FF
:1016A000000000002B0337000000EB00000F980043
:1016B0002E0090008000E900F00F20000080600004
:1016C00020079800C0722800346702000000000064
:1016D0002E01900062079800210037006E019000F3
:1016E0006E0090008000E800E0B72000008040001D
:1016F00090407800E0B720000000410001487800E9
:10170000EE009000E0B7200000804000104078001C
:101710000004E00007003200EE009000E0B7200077
:101720000080400010407800446C0200000000007F
:101730000300370000C2B300446C02000000000048
:101740000E0890000000E800000F98006E00900066
:101750008000E800F00F2000008060006007980023
:10176000EE009000F0638000808F5000DBFF3A00B5
:10177000F06380008000E900F00F2000008060002E
:10178000F063880000732800346702000000000046
:101790000E089000CC6902000000000030732800A1
:1017A0003467020000000000EA02370070C0B30096
:1017B000446C020000000000E6023700F163800084
:1017C0002E009000810F5000390032000000EB0025
:1017D000000F9800AE0190006307980021003700C9
:1017E0006E0190006E0090008000E800E0B72000DD
:1017F0000080400090407800E0B7200000004100E9
:1018000001487800EE009000E0B720000080400022
:10181000104078000004E00007003200EE00900065
:10182000E0B720000080400010407800446C0200C7
:10183000000000000300370000C2B300446C020047
:10184000000000000E0890000000E800000F980063
:101850006E0090008000E800F00F20000080600023
:1018600060079800EE009000F0638000808F5000C9
:10187000DBFF3A00F06380008000E900F00F2000F9
:1018800000806000F0638800007328003467020065
:10189000000000000E089000CC690200000000006B
:1018A000307328003467020000000000A9023700EE
:1018B00070C0B300446C020000000000A5023700B5
:1018C000246C020000000000604F9800EE48900079
:1018D000B0C5B30080CF50009E023A00246C0200D5
:1018E00000000000604F98006E4890000080FB00F0
:1018F000700F980010042000FE089000808F5000A8
:1019000054003200100420007E099000800F510026
:1019100009003C0010032000FE099000808F510058
:101920001200320040032000FE089000808F50001B
:101930001600320087023700300420007E09900034
:10194000800F51003200320030042000FE09900068
:10195000808F5100E100350040042000FE08900017
:10196000808F5000110032007A023700246C020090
:1019700000000000604F9800EE489000E0C7B30000
:1019800080CF5000AC01320072023700246C02009C
:1019900000000000604F9800EE489000E0C7B300E0
:1019A00080CF5000BF0132006A0237004E00900025
:1019B000E40F500005003400527B020000000000DC
:1019C0000000EB00400798006202370001648000CD
:1019D0002E009000810F5000090032002E00900070
:1019E0008000E900F00F20000080600020079800D0
:1019F000C072280034670200000000005502370062
:101A000070C0B300446C02000000000051023700B7
:101A1000F16380002E009000810F50000900320019
:101A20002E0090008000E800F00F20000080600091
:101A3000200798005073280034670200000000005F
:101A40004402370070C0B300446C02000000000084
:101A5000400237000000EB00000F780000648000B7
:101A60000000E90080007800F00F20000080600096
:101A7000600798008D003700EE009000E0B720006E
:101A800000804000104078000004E00082003A002E
:101A90006E0090008000E900F00F20008080600060
:101AA000E0B7200000804000104078000004E00013
:101AB000790032001E0FE8001E0090009E0F1000FB
:101AC000750036001E0090000000E8001007980026
:101AD00001648000F0638000808F500014003200A9
:101AE0000A003700F1638000E0B7200080804000EA
:101AF0000040EB0080487800F06380008000E9003F
:101B0000F00F200000806000F0638800F163800027
:101B100000648000808F5000F2FF3A00F163800083
:101B2000E0B72000808040000040EB008048780053
:101B30006E0090008000E900F00F2000008060003F
:101B4000000F9800110037008E089000E0B72000C9
:101B500000804000104078000004E00006003A00D9
:101B60000E0890008000E800F00F20000080600068
:101B700050079800090037000E0890008000E90027
:101B8000F00F200000806000000F98008E08900089
:101B9000F0638000808F5000EBFF3A0090732800C4
:101BA0003467020000000000A1408000E002200035
:101BB0000088B9006102200080804000C0922000AF
:101BC000008040003467020000000000D140800027
:101BD00000202000008060000000E00004003200CF
:101BE00071002000E0562000D692020000000000A4
:101BF0006072280034670200000000005E0190005F
:101C0000020F9800180037008E089000E0B72000FF
:101C10000080400010407800446C0200000000008A
:101C2000F26380008E089000E0B720000080400042
:101C300090407800E0B720000000410001487800A3
:101C4000F06380008000E800F00F2000008060005A
:101C5000F06388000E0890008000E800F00F20007C
:101C600000806000000F98008E0890006E009000C9
:101C7000808F5000E4FF3A00F1638000E0B720005D
:101C8000808040000040EB0080487800F3638000D3
:101C900023079800090037006E0090008000E900DB
:101CA000F00F20000080600060079800EE009000B8
:101CB000F0638000808F50006FFF3A00EE009000CC
:101CC000F0638000808F5000A2013A0070C0B30022
:101CD000446C0200000000009E0137000000EB0091
:101CE000000F7800006480000000E90080007800A8
:101CF000F00F200000806000600798008E00370021
:101D0000EE009000E0B72000008040001040780016
:101D10000004E00083003A006E0090008000E900BB
:101D2000F00F200080806000E0B7200000804000BD
:101D3000104078000004E0007A0032001E0FE80036
:101D40001E0090000000E9009E0F500075003A0050
:101D50001E0090000000E900100798000164800058
:101D6000F0638000808F5000140032000A003700BA
:101D7000F1638000E0B72000808040000040EB006D
:101D800080487800F06380008000E900F00F2000B8
:101D900000806000F0638800F163800000648000D0
:101DA000808F5000F2FF3A00F1638000E0B720001E
:101DB000808040000040EB00804878006E0090007A
:101DC0008000E900F00F200000806000000F980004
:101DD000110037008E089000E0B72000008040001E
:101DE000104078000004E00006003A000E08900061
:101DF0008000E800F00F200000806000500798008D
:101E0000090037000E0890008000E900F00F200064
:101E100000806000000F98008E089000F063800042
:101E2000808F5000EBFF3A00907328003467020067
:101E300000000000A1408000E00220000088B900FE
:101E40006102200080804000C0922000008040009D
:101E50003467020000000000D14080000020200014
:101E6000008060000000E0000400320071002000EB
:101E7000E0562000D69202000000000060722800A8
:101E800034670200000000005E009000000F980020
:101E9000180037008E089000E0B720000080400056
:101EA00010407800446C020000000000F2638000E3
:101EB0008E089000E0B7200000804000904078003D
:101EC000E0B720000000410001487800F063800086
:101ED0008000E800F00F200000806000F0638800C0
:101EE0000E0890008000E800F00F200000806000E5
:101EF000000F98008E0890006E009000808F5000B8
:101F0000E4FF3A00F1638000E0B7200080804000E9
:101F10000040EB0080487800F163800021079800C2
:101F2000090037006E0090008000E900F00F2000EB
:101F30000080600060079800EE009000F063800071
:101F4000808F50006EFF3A00EE009000F06380003A
:101F5000808F5000FF003A001E009000E10F5000FB
:101F600031003A009073280034670200000000003E
:101F7000A1408000E00220000088B900610220003A
:101F800080804000C0922000008040003467020042
:101F900000000000D1408000002020000080600090
:101FA0000000E0000400320071002000E056200034
:101FB000D692020000000000607228003467020020
:101FC000000000000A003700F1638000E0B7200045
:101FD000808040000040EB0080487800F063800083
:101FE0008000E900F00F200000806000F0638800AE
:101FF000F163800000648000808F5000F2FF3A009F
:10200000F1638000E0B72000808040000040EB00DA
:1020100080487800F2638000220798000000EB00FF
:1020200010079800CB00370070C0B300446C02006A
:1020300000000000C7003700016480002E009000FF
:10204000810F500013003200016480002E009000C8
:102050000100500080007800F00F20000080600038
:10206000000F980000732800346702000000000091
:102070000E089000CC6902000000000030732800B8
:10208000346702000000000003648000230798000A
:10209000B000370070C0B300446C020000000000C4
:1020A000AC003700F16380002E009000810F5000DB
:1020B00013003200F16380002E0090000080500079
:1020C00080007800F00F200000806000000F980072
:1020D0000073280034670200000000000E08900022
:1020E000CC69020000000000F07328003467020091
:1020F00000000000F0638000200798009500370082
:1021000070C0B300446C0200000000009100370072
:1021100010002000600F98000000EB0010079800EE
:10212000F1638000E0B72000808040000040EB00B9
:1021300080487800F06380008000E800F00F200005
:1021400000806000F0638800F16380002107980040
:102150001074280060670200000000007D00370056
:102160004E0090000000E800400798004E009000EC
:10217000F40F500077003A00166D020000000000D6
:1021800074003700F06380008000E800F00F20004A
:102190008080600000648000808F50006A00320000
:1021A0006E489000FF4F500067003600EE489000E8
:1021B000E0C7B30080CF500063003E00F1638000B1
:1021C0002E009000808F500015003A006E4890005D
:1021D000446C020000000000F16380006E49900032
:1021E000E0B720000080400002487800F0638000E3
:1021F0008000E800F00F200000806000F06388009D
:10220000F1638000E0B72000808040000040EB00D8
:1022100080487800F2638000220798004D00370064
:10222000F16380002E009000008050008000780054
:10223000F00F200000806000000F9800007328005D
:1022400034670200000000000E089000CC69020014
:1022500000000000F0732800346702000000000056
:10226000F0638000600798001D0037006E0090004A
:102270000001E800EE009000E0B720000080400080
:1022800090407800E0B7200000004100014878004D
:10229000EE009000E0B72000008040001040780081
:1022A0000004E00009003200EE009000E0B72000DA
:1022B0000080400010407800446C020000000000E4
:1022C0002074280034670200000000006E009000B7
:1022D0008000E900F00F2000008060006007980097
:1022E0006E0190002E0090008000E900F00F2000A9
:1022F00000806000800F5100DCFF3A006E489000C3
:10230000446C020000000000AE0090006E49900096
:10231000E0B7200000804000024878002E009000C6
:102320008000E800F00F2000008060002007980087
:10233000F06380008000E800F00F20000080600063
:10234000F06388000300370070C0B300446C0200E3
:10235000000000006E0890000000E000B7FB3200B3
:10236000F0638000400F980000648000300F9800F8
:102370000000EB00600F98000000EB00500F980089
:102380000000EB0010648800FC043700016480004A
:10239000E0B720000080400010407800604F9800B7
:1023A0006E4890000080FB006101B9002217980080
:1023B00033179800E0072000010020002E11900044
:1023C000BE119000800F5100818F5900BF043E0064
:1023D0002E109000BE10900000600100BD04370078
:1023E000BA043700B9043700B8043700B70437001F
:1023F000B6043700B5043700B4043700B30437001F
:10240000B2043700B3043700B0043700AF0437001C
:10241000B0043700AD043700AC043700AB0437001C
:10242000AA043700A9043700A8043700A70437001E
:10243000A6043700A5043700A4043700A30437001E
:10244000A2043700A1043700A00437009F0437001E
:102450009E0437009D0437009C0437009D0437001C
:102460007A043700BA0237002B01370030013700F9
:10247000D5013700C30137009404370093023700B9
:10248000920437009104370092043700910437001A
:10249000260437003F0437000A04370033033700AF
:1024A0003203370031033700300337002F03370082
:1024B0002E0337002D0337002C0337002B03370082
:1024C0002A0337008104370080043700DA0137001F
:1024D000C90037007D0437003F0037003E01370058
:1024E000300137007904370065003700A20137005A
:1024F000760437007504370074043700730437001E
:102500007204370071043700700437006700370029
:102510006E0437006D0437006C0437008F003700FD
:102520006A04370069043700B801370067043700D0
:1025300066043700650437003D0137006304370047
:102540006204370061043700E4023700EA03370011
:10255000F40237001E043700010437005B04370023
:1025600003013700270037003A00370074013700B5
:1025700056043700290037002B0037005504370078
:10258000180037005104370050043700540037005A
:102590001A0037004D0437001C0037005D0037007B
:1025A0004A0437006D0337004804370047043700FA
:1025B00046043700170037004F0137004304370047
:1025C0004204370041043700CD023700A500370030
:1025D000DD023700C30037007693020000000000E0
:1025E0003C043700B2070700A04080000000E00074
:1025F0003804320019080700360437006006070067
:102600003404370050090700320437002A09070054
:10261000300437009E0807002E0437009E74020025
:10262000000000002B043700A04080000000E00004
:1026300005003A00D1012000505A200060930200AA
:1026400000000000230437000673020000000000B1
:102650002004370080AE2000104078000000A10068
:102660000010A10081AE20008048780061012000A8
:10267000A0572000609302000000000015043700FE
:1026800080AE2000104078000000A0000010A100E3
:1026900081AE2000804878005101200000592000C0
:1026A00060930200000000000A04370080AE2000A2
:1026B000104078000030A00081AE200080487800F3
:1026C000C1012000E07E2000D69202000000000040
:1026D000107428006067020000000000FD0337004E
:1026E00080AE2000104078000030A10081AE2000B4
:1026F00080487800B1012000307D2000D692020091
:102700000000000010742800606702000000000054
:10271000F0033700A04080000000E00005003A0010
:10272000D1012000505A20006093020000000000F8
:10273000E8033700CB62A900C962A900510120005B
:10274000205C2000D69202000000000010742800D7
:102750006067020000000000DE033700A040800038
:102760000000E00005003A00D1012000505A20008E
:102770006093020000000000D603370080AE200006
:1027800010407800704060000004E00004003A004F
:1027900021022000F0E92000609302000000000008
:1027A000C962A800CB62A90041012000705D200031
:1027B000D69202000000000010742800606702003A
:1027C0000000000021E3A800B0C0B300FC900200AC
:1027D0000000000080007800F0042000808F50008E
:1027E00003003E00707428006067020000000000D3
:1027F00021E3A900B7033700006480008000E800EF
:10280000F00F20000080600000648800CC05070005
:10281000E4030700600798006E0090002E6A020033
:1028200000000000A07628003467020000000000CD
:102830006E009000CC69020000000000A076280025
:1028400034670200000000006E00900094670200F0
:102850000000000010742800606702000000000003
:102860009C033700006480008000E800F00F200027
:102870000080600000648800B1050700C9030700FC
:10288000600798006E0090000080FB008E920200AE
:1028900000000000600798006E0090002E6A0200A1
:1028A00000000000A076280034670200000000004D
:1028B0006E009000CC69020000000000A0762800A5
:1028C00034670200000000006E0090009467020070
:1028D0000000000010742800606702000000000083
:1028E0007C033700A04080000000E00005003A00B3
:1028F00011C0B30010C0B300628B020000000000E2
:1029000074033700A1012000B05E20006093020034
:10291000000000006F0337005100200050602000CD
:1029200060930200000000000000FE006903370011
:1029300006940200000000000000E0006503320081
:10294000A1002000A06020006093020000000000B1
:10295000400620002C92020000000000B29002000D
:102960000000000081BF2A00014001005903370028
:10297000310507000000E800000F98000200370052
:1029800022760200000000000E0890000000E9001E
:10299000000F98000E0890000000E000F8FF3A00D9
:1029A0004C033700240507000000E800000F9800E2
:1029B0000200370000760200000000000E089000C0
:1029C0000000E900000F98000E0890000000E000F1
:1029D000F8FF3A003F033700170507000000E80042
:1029E000000F98000B0037006101200040612000BB
:1029F000D6920200000000004476020000000000B1
:102A00001E670200000000001074280060670200CA
:102A1000000000000E0890000000E900000F980080
:102A20000E0890000000E000EFFF3A002903370095
:102A3000A04080000000E00005003A00D101200025
:102A4000505A20006093020000000000210337006C
:102A5000C002A900C202A80021E3A80020002000B3
:102A60002C92020000000000A0C0B300FC90020005
:102A70000000000080007800001B2000808F5000C4
:102A80000F00360090C0B300FC9002000000000070
:102A900080007800702B2000808F500008003600E6
:102AA00011012000A0622000D69202000000000068
:102AB0001074280060670200000000000C0037005E
:102AC000C002A900C202A900E076280060670200E7
:102AD0000000000021012000B0632000D692020017
:102AE0000000000010742800606702000000000071
:102AF00021E3A900F7023700A04080000000E000B9
:102B000005003A00D1012000505A200060930200D5
:102B100000000000EF023700C002A900C202A900B5
:102B200021012000B0632000D692020000000000C6
:102B3000107428006067020000000000E502370002
:102B4000F1002000C0362000D692020000000000F4
:102B5000169102000000000011002000B037200094
:102B6000D692020000000000107428006067020086
:102B700000000000D702370028910200000000008A
:102B8000D4023700AC040700000F98006100200059
:102B900090652000D6920200000000000E08900010
:102BA0006E6902000000000021002000F065200096
:102BB00060930200000000000E089000589202008E
:102BC00000000000C30237009B040700000F9800BC
:102BD0006100200090652000D692020000000000F5
:102BE0000E0890006E690200000000002100200025
:102BF00030EE200060930200000000000E089000FC
:102C00002C92020000000000B2023700A0408000B9
:102C10000000E00005003A00D1012000505A2000D9
:102C20006093020000000000AA02370078760200DC
:102C300000000000A7023700100020001064880088
:102C40001000200060079800100037000164800029
:102C50006E00900080804000F00F200080806000B7
:102C6000E0B720000080400090407800E0C3B3004F
:102C700080CF500002003A000000EB001064880092
:102C80006E0090000000E80060079800016480007A
:102C90006E00900080804000F00F20008080600077
:102CA000E0B7200000804000104078000004E00001
:102CB000E6FF3A00EE00900020022000808F5000D6
:102CC00002003400100020001064880010648000AE
:102CD0000000E0007F023A00006480008000E8000D
:102CE000F00F20000080600000648800AD02070043
:102CF0006007980001648000F00F20008080600071
:102D0000E0B720000080400090407800D0C3B300BE
:102D100080CF500040003A006E0090000000E000BC
:102D20003A0034006E009000E50F500037003C0080
:102D3000006480008000E800F00F20000080600048
:102D4000006488006E0090000000E90060079800B1
:102D50000000EB00000F98000B0037006E009000A1
:102D60008E0890004500DD008100400040C8200032
:102D7000808040000040EB00804878000E08900002
:102D80000000E800000F98000E089000FF0F5000B0
:102D9000F2FF34000000EB00000F98001300370032
:102DA000EE0190000E0A900001648000E0B7200060
:102DB00000804000104178004518DD00840040008C
:102DC00040C8200000804000024878000E089000B3
:102DD0000000E800000F9800006480008000E80018
:102DE000F00F200000806000006488000164800013
:102DF000E0B720000080400090407800E0C3B300BE
:102E000080CF5000E6FF3A00320237001000200069
:102E1000106488002F0237006E0090000000E00070
:102E20001B003A000000EB00000F98001400370070
:102E30000E0890000040E800CC690200000000008D
:102E4000E078280034670200000000000E089000BF
:102E50004500DD008000780040C820000080400070
:102E60003467020000000000607228006067020002
:102E7000000000000E0890000000E800000F98001D
:102E80000E089000E40F5000E9FF340011023700F3
:102E90006E0090000000E000090034006E00900019
:102EA000E50F500006003C00107428006067020027
:102EB00000000000EE009000216988000502370044
:102EC00010002000106488000202370000648000B7
:102ED0008000E800F00F200000806000006488009F
:102EE00030020700200F98001504070001648000DD
:102EF000F00F200080806000E0B7200000804000DC
:102F00009040780090C2B30080CF50000D003A008E
:102F1000A1408000E00220000088B900FC004000D1
:102F2000C092200000804000900078002E089000A1
:102F3000010001001074280060670200000000001A
:102F4000E40137001000200010648800E101370020
:102F50001000200010648800100020006007980016
:102F600010003700016480006E00900080804000F7
:102F7000F00F200080806000E0B72000008040005B
:102F80009040780020C2B30080CF500002003A0089
:102F90000000EB00106488006E0090000000E80064
:102FA00060079800016480006E00900080804000FF
:102FB000F00F200080806000E0B72000008040001B
:102FC000104078000004E000E6FF3A001064800042
:102FD0000000E000BF013A007100200010662000F0
:102FE000D69202000000000020C2B300446C020030
:102FF000000000002200370001648000F00F200074
:10300000008060000064880001648000E0B7200058
:103010000080400010407800446C02000000000076
:1030200001648000E0B7200000804000104078007C
:103030000000FB00200F980080AE200010407800B8
:10304000684060000004E000040032002E08900098
:103050008E92020000000000200F9800A140800026
:10306000E00220000088B900E8004000C092200083
:1030700000804000900078002E08900001000100C0
:10308000006480000000E8000064880001648000A3
:10309000F00F200080806000E0B72000008040003A
:1030A0009040780020C2B30080CF5000D2FF3A0099
:1030B00000648000F10F20000100600000648800BF
:1030C00020C2B300446C020000000000107428000D
:1030D00060670200000000007E013700A140800010
:1030E000E00220000088B90080007800C092200033
:1030F00000804000100078000000010075013700DA
:10310000A1408000E00220000088B9008080E80033
:10311000C0922000008040001000780000000100F4
:103120006C013700A1408000E00220000088B90057
:10313000E4004000C09220000080400010007800B1
:103140000000010063013700A1408000E002200080
:103150000088B900E6004000C092200000804000D6
:1031600010007800000001005A01370071002000B3
:1031700010662000D69202000000000089010700BE
:10318000200F9800006480000000E90000648800BF
:1031900001648000F00F200000806000006488005F
:1031A000250307000000E800000F98004503070012
:1031B000300798003E0090000000E0005D00320003
:1031C0003E0090008040780070AD200001487800FB
:1031D0003E009000E80F50000600340080AE200052
:1031E000104078000050A00081AE20008048780098
:1031F0005000370080AE2000104078000050A10041
:1032000081AE2000804878004A0037002E089000E8
:10321000869102000000000080AE2000104078007F
:103220000042B2000004E00004003A0070AD20004B
:1032300010407800E84F500009003A0080AE2000AE
:10324000104078000042B2000004E0000B003200A1
:1032500070AD200010407800F04F500007003200A1
:10326000B0C3B300446C02000000000070AD200049
:1032700010407800CC6902000000000080AE200001
:1032800010407800684060000004E0000400320054
:103290002E0890008E92020000000000200F98007F
:1032A000A1408000E00220000088B900E800400052
:1032B000C092200000804000900078002E0890000E
:1032C00001000100100F980000C2B300446C02001E
:1032D0000000000080AE2000104078000044B200E2
:1032E0000004E0001300320061002000806620002E
:1032F000D69202000000000080AE2000104078004E
:10330000684060000004E000040032001E089000E5
:103310008E92020000000000100F98001E0890001E
:10332000869102000000000000C2B300446C02005D
:10333000000000000E0890000000E900000F980057
:103340000E0890000000E000B0FF3A001074280062
:103350006067020000000000DE003700610020000E
:1033600080662000D692020000000000B202070032
:103370000000E800000F9800D20207003007980014
:103380003E0090000000E000440032003E0090004B
:103390008040780070AD2000014878003E00900029
:1033A000E80F50000600340080AE20001040780086
:1033B0000050A00081AE2000804878003700370020
:1033C00080AE2000104078000050A10081AE2000A7
:1033D0008048780031003700A1408000E0022000E2
:1033E0000088B900EA004000C09220000080400040
:1033F0001000780000000100100F980080AE20003F
:1034000010407800684060000004E00004003200D2
:103410001E0890008E92020000000000100F98001D
:103420001E089000869102000000000080AE20007F
:10343000104078000042B2000004E00004003A00AE
:1034400070AD200010407800E84F500009003A00AD
:1034500080AE2000104078000042B2000004E0007E
:103460000B00320070AD200010407800F04F50008B
:1034700007003200B0C3B300446C0200000000003B
:1034800070AD200010407800CC6902000000000000
:1034900000C2B300446C0200000000000E0890005F
:1034A0000000E900000F98000E0890000000E00006
:1034B000C9FF3A0010742800606702000000000095
:1034C0008400370081002000E06620006093020045
:1034D00000000000A1408000E00220000088B90048
:1034E000EC004000C09220000080400010007800F6
:1034F0000000010077003700810020006067200095
:103500006093020000000000A1408000E002200063
:103510000088B900EE004000C0922000008040000A
:1035200010007800000001006A003700E100200070
:10353000E06720006093020000000000A1408000CE
:10354000E00220000088B900F0004000C092200096
:103550000080400010007800000001005D0037008E
:10356000E1002000C068200060930200000000001D
:10357000A1408000E00220000088B900F200400075
:10358000C092200000804000100078000000010080
:1035900050003700C1002000D0642000D692020005
:1035A00000000000A1408000E00220000088B90077
:1035B000F4004000C092200000804000100078001D
:1035C000000001001E6702000000000041003700FB
:1035D00019020700000F9800D1002000A06A200007
:1035E000D6920200000000000E08900086910200B2
:1035F000000000000E0890000000E800000F980096
:1036000008003700A1408000E00220000088B900D7
:10361000F6004000C09220000080400010007800BA
:10362000000001000E0890000000E900000F980063
:103630000E0890000000E000F2FF3A00107428002D
:10364000606702000000000022003700FA01070056
:103650000000E800000F9800A1002000706B20001F
:10366000D6920200000000000D003700A14080004B
:10367000E00220000088B900F8004000C09220005D
:103680000080400010007800000001001E6702006A
:103690000000000000C2B300446C02000000000003
:1036A0000E0890000000E900000F98000E0890003E
:1036B0000000E000EDFF3A0001012000A0692000B9
:1036C000609302000000000002003700100020009C
:1036D00010648800006480008000E800F00F200083
:1036E0000080600000648800106480000000E0003A
:1036F0001C00320051012000106C2000D692020004
:1037000000000000BE08900000648000808F500020
:103710000700310000648000804078003E0890007F
:1037200000C05000CC690200000000000600370015
:1037300000648000804078003E08900000C0500087
:10374000CC690200000000000000EB00106488005B
:1037500010002000500F98001074280060670200CD
:103760000000000001648000F0638000808F500042
:1037700002003A0010002000500F98005E089000F0
:103780000000E00001FB32004E0890000064880059
:103790004E089000F06388000000EB00600F980076
:1037A00090F637000600FA000000EB0010079800C2
:1037B0000000EB00000F7800016480001E00900004
:1037C00080804000F00F200080806000E0B7200083
:1037D000008040009040780000C3B30080CF5000CC
:1037E00043003400016480001E009000808040008F
:1037F000F00F200080806000E0B7200000804000D3
:103800009040780090C3B30080CF500038003C0057
:10381000016480001E00900080804000F00F2000B6
:1038200080806000E0B720000080400010407800F9
:103830008000FB0000FD2F00008F40001E00900064
:103840000000E80010079800120037001E00780002
:103850006A00B900000F7800016480001E0090002B
:1038600080804000F00F200080806000E0B72000E2
:1038700000804000104078000000FB009E004000E7
:1038800000FD2F00008F40001E0090000000E800A7
:1038900010079800016480001E00900080804000A6
:1038A000F00F200080806000E0B720000080400022
:1038B00090407800F0C2B30080CF50005101340036
:1038C000016480001E00900080804000F00F200006
:1038D00080806000E0B720000080400090407800C9
:1038E00090C3B30080CF5000D8FF340045013700AB
:1038F000016480001E00900080804000F00F2000D6
:1039000080806000E0B72000008040009040780098
:1039100000C3B30080CF500035013A001E00900074
:103920000000E80010079800016480001E0090006D
:1039300080804000F00F200080806000E0B7200011
:10394000008040009040780020C6B30080CF500037
:103950000B003200016480001E0090008080400057
:10396000F00F200080806000E0B720000080400061
:103970009040780020C4B30080CF50002D003A0062
:103980001E0090000000E8001007980012003700A9
:103990001E00780000004000000F780001648000E5
:1039A0001E00900080804000F00F200080806000AA
:1039B000E0B7200000804000104078000000FB00CD
:1039C0009E00400000FD2F00008F40001E00900070
:1039D0000000E80010079800016480001E009000BD
:1039E00080804000F00F200080806000E0B7200061
:1039F000008040009040780010C3B30080CF50009A
:103A0000E3FF3200016480001E00900080804000CF
:103A1000F00F200080806000E0B7200000804000B0
:103A20009040780000C3B30080CF5000D8FF320030
:103A3000F4003700016480001E0090008080400088
:103A4000F00F200080806000E0B720000080400080
:103A50009040780080C7B30080CF50000B00320048
:103A6000016480001E00900080804000F00F200064
:103A700080806000E0B72000008040009040780027
:103A800080C5B30080CF50008E003A001E00900029
:103A90000000E80010079800470037001E0078007B
:103AA0004400DD00000F7800016480001E009000DB
:103AB00080804000F00F200080806000E0B7200090
:103AC0000080400090407800F0C2B30080CF5000EA
:103AD00018003400016480001E00900080804000C7
:103AE000F00F200080806000E0B7200000804000E0
:103AF0009040780090C3B30080CF50000D003C0090
:103B0000016480001E00900080804000F00F2000C3
:103B100080806000E0B72000008040001040780006
:103B20000000FB009E00400000FD2F00008F4000C1
:103B30001E003700016480001E009000808040005D
:103B4000F00F200000816000016480001E009000E2
:103B500080804000F00F200080806000E0B72000EF
:103B6000008040009040780000C2B30080C0700028
:103B7000E0B72000000041000148780001648000A7
:103B80001E00900080804000F00F200080806000C8
:103B9000E0B7200000804000104078000000FB00EB
:103BA0009E00400090FA2F00008F40001E00900001
:103BB0000000E80010079800016480001E009000DB
:103BC00080804000F00F200080806000E0B720007F
:103BD0000080400090407800F0C2B30080CF5000D9
:103BE0000B003400016480001E00900080804000C3
:103BF000F00F200080806000E0B7200000804000CF
:103C00009040780090C3B30080CF5000A3FF3400F1
:103C1000016480001E00900080804000F00F2000B2
:103C200080806000E0B72000008040009040780075
:103C300000C4B30080CF50000B003400016480004A
:103C40001E00900080804000F00F20008080600007
:103C5000E0B72000008040009040780060C4B300CE
:103C600080CF50008DFF3400016480001E00900062
:103C700080804000F00F200080806000E0B72000CE
:103C8000008040009040780000C6B30080CF500014
:103C90005C003400016480001E00900080804000C1
:103CA000F00F200080806000E0B72000008040001E
:103CB0009040780060C6B30080CF500077FF34009A
:103CC00050003700016480001E009000808040009A
:103CD000F00F200080806000E0B7200000804000EE
:103CE00090407800F0C2B30080CF5000450034000F
:103CF000016480001E00900080804000F00F2000D2
:103D000080806000E0B72000008040009040780094
:103D100090C3B30080CF50003A003C0001648000A3
:103D20001E00900080804000F00F20008080600026
:103D3000E0B7200000804000104078008000FB00C9
:103D400000FD2F00008F4000120037001E00780099
:103D50006A00B900000F7800016480001E00900026
:103D600080804000F00F200080806000E0B72000DD
:103D700000804000104078000000FB009E004000E2
:103D800000FD2F00008F40001E0090000000E800A2
:103D900010079800016480001E00900080804000A1
:103DA000F00F200080806000E0B72000008040001D
:103DB00090407800F0C2B30080CF50001100340072
:103DC000016480001E00900080804000F00F200001
:103DD00080806000E0B720000080400090407800C4
:103DE00090C3B30080CF5000D8FF340005003700E7
:103DF00010002000106488000000EB0020079800ED
:103E00000A003700016480001E009000008040001E
:103E10000064880001648000F00F200000806000D2
:103E2000006488001E007800200798002E00900093
:103E30000080FA00000006000400FA000064800020
:103E40008000E800F00F200080806000E0B72000D4
:103E50000080400090407800A0C3B30080CF5000A5
:103E600013003A00006480000080E80000648800CD
:103E700001648000F00F2000008060000064880072
:103E800048FE0700000F7800006480000000E90091
:103E90000064880001648000F00F20000080600052
:103EA000006488001E0078001007980002003700A8
:103EB00010002000100798001E0090000080FA00FB
:103EC000000006000400FA00006480008000E800A2
:103ED000F00F200080806000E0B7200000804000EC
:103EE00090407800B0C3B30080CF50000F003A007C
:103EF000006480008080E800F00F200000806000F7
:103F00000064880027FE0700000F7800006480002E
:103F10008000E900F00F200000806000006488004D
:103F20001E00780010079800020037000000EB0028
:103F3000100798001E0090000080FA0000000600A4
:103F40000000FA0005003700006480008000E800EF
:103F5000F00F200000806000006488000164800091
:103F6000E0B72000008040009040780000C2B3001D
:103F700080CF5000F4FF32000080FA0000000600FD
:103F80000400FA000000EB00000F780000648000DD
:103F90008000E800F00F20000080600000648800CE
:103FA000E7FF0700FFFD0700000F78001E00E0009C
:103FB0004D003A000000EB00100798001300370096
:103FC0001E0090000040E800CC69020000000000E4
:103FD0002079280034670200000000009E00900055
:103FE000E00220000088B9006102200080804000CB
:103FF000C0922000008040006067020000000000C6
:104000001E0090000000E800100798001E009000BD
:10401000E70F5000EAFF340071012000606D2000BE
:1040200060930200000000000000EB0010648800B4
:10403000130020008200200011002000100020004A
:1040400055000700000FE900E0FF2F009E0F100051
:10405000030032000080EB009E0F100005003A00C4
:10406000E1002000D06E20006093020000000000FC
:1040700042003700A1408000E00220000088B90023
:104080000102200080804000C0922000008040009B
:104090001000780000000100B29002000000000053
:1040A0001E007800A0408800A1408000E0022000AF
:1040B0000088B900FE004000C0922000008040004F
:1040C00010007800000001001E00E0000100320036
:1040D000C222A80051002000505720006093020027
:1040E00000000000250037001E0FE90070002000CE
:1040F0009E0F10001D003C00A1408000E002200047
:104100000088B9000102200080804000C092200099
:10411000008040001000780000000100B290020012
:10412000000000001E007800A0408800A140800030
:10413000E00220000088B900FE004000C09220008C
:104140000080400010007800000001001E00E00028
:1041500001003200C222A800510020005057200068
:1041600060930200000000000400370051012000AD
:10417000C07220006093020000000000F063800025
:104180008000E900F00F20000080600000648800DB
:104190000080FA00000006001E00FA00100F9800D0
:1041A000210F9800320F9800430F98000000EB0099
:1041B000400798000000EB00200798000000EB008B
:1041C000100798000000EB00000F780050792800DD
:1041D00034670200000000001E0890000000E000AC
:1041E00004003D00907928003467020000000000C0
:1041F000030037001E089000CC6902000000000098
:10420000B079280034670200000000006700370022
:10421000246C020000000000204F98002E489000FF
:104220000000FB00600F98006E089000ED0F50003A
:1042300029003200EE089000ED8F500007003C008E
:104240006E099000E80F51000D0032006E089000DA
:10425000EA0F50002000320035003700D002200065
:10426000EE089000808F50001E0032008007200072
:104270006E099000800F5100270032002C0037009B
:104280004E0090000000E000070032004E00900059
:104290000000E9004007980080722800346702009F
:1042A00000000000410037001E00E0000600320060
:1042B0000000EB00000F78008072280034670200D5
:1042C000000000003900370070C0B300446C0200E9
:1042D0000000000035003700100020002007980083
:1042E000320037004E0090000000E00006003A0067
:1042F000D0C2B300446C0200000000001000200097
:10430000000F78002900370070C0B300446C020031
:1043100000000000250037004E0890000000E0007B
:10432000030032000080EB00500F98005D00370062
:10433000AE489000F0C2B30080CF500018003400A7
:10434000AE48900090C3B30080CF500014003C00F2
:104350004E009000E30F50000600340070C0B30020
:10436000446C02000000000040002000400798005C
:104370000E0037002E489000446C02000000000040
:10438000CE0090006B0047002E49900082707800AC
:104390004E0090000000E80040079800030037003E
:1043A00070C0B300446C0200000000002E009000BA
:1043B0000000E00096FF32001074280060670200E1
:1043C000000000004E0090000000E00003003A00F2
:1043D0001E089000500F9800320037000000EB00DC
:1043E000100798004E0090000000E9004007980078
:1043F000CE00900031079800110037001E00900099
:104400006A00B90010079800BE0090004E009000AE
:10441000808050006B004700614078008000FB0006
:104420001E0090008080400000FD2F0000804000B2
:10443000100798004E0090000000E9004007980027
:104440004E0090000000E000ECFF3D009E00900058
:104450002E089000808F50000D0035009E009000C7
:104460003E089000808F500009003C001E00E000D4
:10447000040032001E0090000000EA00500F980077
:10448000080037001E019000520F98000500370009
:10449000B101200080EC20006093020000000000C9
:1044A00042FF37005E0890000080FA00000006001E
:1044B0000400FA00E07928003467020000000000E0
:1044C000A081200010407800446C02000000000031
:1044D000107428006067020000000000C07A280005
:1044E0003467020000000000D1002000A0802000FE
:1044F000D692020000000000A1BF2A000000EB00DD
:10450000146B020000000000000F78001E0078000D
:104510004800DE00CC69020000000000E0C2B300E9
:10452000446C0200000000001E007800CC6902000C
:104530000000000010742800606702000000000006
:104540006100200030762000D692020000000000BA
:10455000B0408000866A0200000000007100200068
:1045600010EC2000D692020000000000C040800045
:10457000866A020000000000107C280034670200F8
:1045800000000000C04080001007980020042300B5
:104590009E009000808F50001600320020042300FF
:1045A0009E009000808F500005003E0030002300E8
:1045B0009E009000808F50000A00320019003700E2
:1045C000300423009E009000808F50000D003200C8
:1045D000600423009E009000808F50000D00320088
:1045E00010003700007D2800346702000000000042
:1045F0000F003700307D2800346702000000000003
:104600000B003700607D28003467020000000000C6
:1046100007003700907D280034670200000000008A
:1046200003003700C07D280034670200000000004E
:10463000007E28006067020000000000E101200009
:104640009076200060930200000000000000EB0064
:10465000000F78000080FA00000006000000FA0059
:104660005100200050922000D6920200000000006D
:10467000C1BF2A000000EB00146B02000000000024
:10468000866A02000000000061002000A092200065
:10469000D692020000000000E1BF2A000000EB00FB
:1046A000146B020000000000866A02000000000097
:1046B000107428006067020000000000C1002000A4
:1046C0007078200060930200000000007000070076
:1046D000C2C2BF00614060000004E000050032007B
:1046E00011012000A0622000D6920200000000000C
:1046F0000400370021012000B0632000D6920200A0
:1047000000000000C0C2B300446C020000000000C2
:1047100000C2B300446C020000000000CBC2BF0026
:10472000684060000004E000050032004101200004
:10473000705D2000D69202000000000004003700E7
:1047400051012000205C2000D692020000000000F1
:10475000C0C2B300446C02000000000000C2B300FD
:10476000446C02000000000080AE20001040780081
:10477000704060000004E0000500320021022000CB
:104780003079200060930200000000000400370030
:10479000E1012000507B2000609302000000000037
:1047A00080AE200010407800684060000004E00007
:1047B00005003A00B1012000307D2000D6920200B1
:1047C0000000000004003700C1012000E07E20004E
:1047D000D692020000000000C0C2B300446C020088
:1047E0000000000000C2B300446C020000000000A2
:1047F000B1012000B01A2100D69202000000000092
:1048000070AD200010407800CC690200000000006C
:1048100010742800606702000000000080AE2000D5
:104820001040780063406000E14F500005003A00FE
:104830005101200000592000609302000000000098
:104840000400370061012000A0572000609302009F
:1048500000000000A1408000E00220000088B900B4
:104860004102200080804000C09220000080400073
:104870001000780000000100C100200070782000C6
:1048800060930200000000000080FA0000000600B3
:104890000000FA00A1002000400721006093020000
:1048A0000000000061042000C00C210060930200A1
:1048B00000000000A1012000E0072100D6920200C4
:1048C00000000000A1408000E00220000088B90044
:1048D0002102200080804000C09220000080400023
:1048E0001000780000000100A100200080092100D4
:1048F000D692020000000000004020005000070097
:10490000001020004E000700002020004C0007008F
:10491000000420004A0007000008200048000700AB
:1049200010742800606702000000000041002000B1
:1049300020112100D69202000000000021E3A8000F
:10494000A0C0B300FC90020000000000D06A02008A
:104950000000000011002000B0372000D6920200B5
:104960000000000090C0B300446C02000000000092
:1049700090C0B300FC90020000000000D06A02006A
:104980000000000011002000B0372000D692020085
:104990000000000090C0B300446C02000000000062
:1049A000C0C0B300FC90020000000000D06A02000A
:1049B0000000000011002000B0372000D692020055
:1049C0000000000090C0B300446C02000000000032
:1049D000B0C0B300FC90020000000000D06A0200EA
:1049E0000000000011002000B0372000D692020025
:1049F0000000000090C0B300446C02000000000002
:104A000021E3A900004020001C0007000010200046
:104A10001A000700002020001800070000042000F2
:104A2000160007000008200014000700107428007A
:104A300060670200000000000080FA00000006002D
:104A40000200FA00000F7800401680001E0060008F
:104A50000000E00004003200207E280034670200DD
:104A60000000000003003700507E28003467020079
:104A7000000000000080FA00000006000200FA00BA
:104A8000000F7800501680001E0060000000E0005B
:104A900004003200807E280034670200000000001D
:104AA00003003700B07E28003467020000000000D9
:104AB0000080FA00000006000200FA000064800096
:104AC0008000E800F00F2000008060000064880093
:104AD0001BFD070033FB0700000F78001E00E000FD
:104AE00006003400400020009E0F100003003C0030
:104AF0001E00E900904088000D0037000000EB0028
:104B00001064880021022000708120006093020060
:104B1000000000008001EB00420020001100200096
:104B2000100020009CFD07000000E9009040880074
:104B3000210120009083200060930200000000000B
:104B40000080FA00000006000200FA000040EB00BE
:104B5000004F7800006480008000E800F00F200023
:104B60000080600000648800F5FC07000DFB070072
:104B7000104798001E4090000004E0000900320039
:104B80001E409000EA4F500006003E001E4090007C
:104B90000040E90080407800008120000148780052
:104BA0000F0037000000EB0010648800D1082000DF
:104BB0006087200060930200000000008001EB008D
:104BC000A2002000110020009000200072FD0700CC
:104BD0000040E90080407800008120000148780012
:104BE0000081200010407800E94F500010003A008A
:104BF000D3FC0700EBFA0700004F78001E04E0002A
:104C00000B003A000000EB0010648800E07E2800F2
:104C100060670200000000008001EB00F2FF270047
:104C20008000EB00200220005BFD0700004F7800B1
:104C3000410120003090200060930200000000003D
:104C400011012000A0192100609302000000000063
:104C50000081200010407800E94F500003003A0026
:104C60001E407800626C020000000000386B0200F9
:104C70000000000000003700666B0200000000002A
:104C80000004E000FCFF3200246C02000000000081
:104C90008040780000C2B30080CF50000100320095
:104CA000F5FF37000080FA00000006005752490067
:104CB00054452000424954003A2020002A6E6500E5
:104CC00078742000636C6F00636B2000285E2900FD
:104CD000207769006C6C2000757365002074680093
:104CE0006973200076616C0075654E006F2064006A
:104CF0006576690063652C002074720079202800B5
:104D0000414C4100524D290020534500415243007F
:104D100048206D00616372006F2066006972730045
:104D20007441440044524500535320004D41430018
:104D3000524F200020302E004D616300726F200022
:104D40006D656E00754D610063726F00202020005C
:104D500020203100574952004520610064647200F0
:104D6000657373000D0A200020202A003157490086
:104D700052452000524F4D0020434F004D4D410001
:104D80004E4420004D414300524F73003A0D0A003B
:104D9000203531002E52450041442000524F4D0035
:104DA000202830007833330029202A00666F7200F3
:104DB000207369006E676C00652064006576690089
:104DC00063652000627573000D0A200038352E00DF
:104DD0004D41540043482000524F4D0020283000E0
:104DE0007835350029202A00666F6C006C6F7700DB
:104DF0006564200062792000363462006974200006
:104E00006164640072657300730D0A002032300023
:104E1000342E53004B49500020524F004D202800A3
:104E200030784300432920002A666F006C6C6F00C5
:104E3000776564002062790020636F006D6D61000A
:104E40006E640D000A20320033362E00414C4100C2
:104E5000524D200053454100524348002028300065
:104E600078454300290D0A0020323400302E5300CB
:104E70004541520043482000524F4D002028300049
:104E80007846300029414C0041524D0020534500E6
:104E90004152430048202800307845004329530000
:104EA0004541520043482000283078004630290010
:104EB0004465760069636500204944007320610001
:104EC0007265200061766100696C6100626C65004A
:104ED00020627900204D410043524F002C20730086
:104EE00065652000283029002E52450041442000ED
:104EF000524F4D002028300078333300293A2000EB
:104F00004D41540043482000524F4D0020283000AE
:104F10007835350029534B0049502000524F4D0041
:104F2000202830007843430029556E006B6E6F00D7
:104F3000776E20006D616300726F2C002074720028
:104F400079203F00206F7200202830002920660061
:104F50006F72200068656C0070425500532052004B
:104F6000455345005420570061726E00696E67001A
:104F70003A202A0053686F00727420006F7220007C
:104F80006E6F200070756C006C2D750070202A000B
:104F90004E6F2000646576006963650020646500DB
:104FA0007465630074656400204453003138530015
:104FB0003230200048696700682050007265730035
:104FC0002044690067205400686572006D445300F6
:104FD000313842003230200050726F00672052009A
:104FE00065732000446967002054680065726D0095
:104FF0004453310038323200204563006F6E200088
:10500000446967002054680065726D0044533200A3
:1050100034303400204563006F6E7200616D2000F3
:1050200074696D0065204300686970004453320064
:105030003433310020314B002045450050524F00A1
:105040004D556E006B6E6F00776E200064657600C4
:105050006963650050574D00206469007361620008
:105060006C656400314B48007A2D34002C303000E0
:10507000304B48007A205000574D46007265710051
:1050800075656E0063792000696E20004B487A00D8
:105090002050720065736300616C65003A505200E5
:1050A000323A44007574790020637900636C6500BE
:1050B00020696E002025200050574D0020616300BC
:1050C0007469760065455200524F52003A205000F4
:1050D000574D200061637400697665002C206700DD
:1050E00020746F0020646900736162006C65410088
:1050F0005558200046726500717565006E63790031
:105100003A20410055582000494E500055542F0078
:1051100048492D005A415500582048004947480049
:1051200041555800204C4F0057564F004C544D00ED
:105130004554450052204D004F444500564F4C0009
:105140005441470045205000524F4200453A20004C
:1051500056457200726F720028292000406C690069
:105160006E653A0020407000676D730070616300E7
:10517000653A20006279740065732E00546F6F00E9
:10518000206C6F006E67210053796E0074617800A7
:1051900020657200726F72004E6F2000454550000E
:1051A000524F4D004572610073696E0067646F0075
:1051B0006E655300617669006E672000746F200091
:1051C000736C6F00742049006E7661006C69640036
:1051D00020736C006F744C006F616400696E67002F
:1051E000206672006F6D2000736C6F0074204500A4
:1051F00052524F00523A2000636F6D006D616E0095
:1052000064206800617320006E6F20006566660090
:10521000656374002068650072654100434B4E0071
:1052200041434B0049324300205354004152540043
:10523000204249005449320043205300544F50004B
:10524000204249005449320043206D006F646500DC
:105250003A0D0A0020312E0020536F00667477004B
:10526000617265000D0A2000322E20004861720034
:105270006477610072655300657420007370650087
:1052800065643A000D0A2000312E20007E354B0067
:10529000487A0D000A2032002E207E0035304B0067
:1052A000487A0D000A2033002E207E003130300075
:1052B0004B487A000D0A2000342E20007E34300046
:1052C000304B48007A574100524E49004E473A0051
:1052D00020484100524457004152450020493200C5
:1052E0004320690073206200726F6B00656E2000BE
:1052F0006F6E2000746869007320500049432100DC
:10530000202852004556200041332900536574007F
:1053100020737000656564003A0D0A0020312E008C
:1053200020313000304B48007A0D0A0020322E0028
:1053300020343000304B48007A0D0A0020332E0014
:1053400020314D00487A490032432000286D6F001B
:1053500064207300706429003D28200020302E0056
:105360004D616300726F20006D656E00750D0A005F
:1053700020312E003762690074206100646472007D
:10538000657373002073650061726300680D0A0025
:1053900020322E004932430020736E006966660099
:1053A0006572530065617200636869006E67200072
:1053B0004932430020616400647265007373200009
:1053C0007370610063652E0020466F00756E640087
:1053D00020646500766963006573200061743A009B
:1053E000536E6900666665007228420041534900A9
:1053F000432952006561640079612F00412F40000C
:1054000020636F006E7472006F6C73002041550052
:1054100058207000696E61002F412F00402063000A
:105420006F6E7400726F6C00732043005320700025
:10543000696E43006F6D6D00616E6400206E6F00D9
:10544000742075007365640020696E002074680024
:10545000697320006D6F6400655075006C6C2D00E1
:105460007570200072657300697374006F72730049
:10547000204F4600465075006C6C2D007570200062
:1054800072657300697374006F727300204F4E0071
:1054900053656C00662D74006573740020696E009E
:1054A000204869005A206D006F646500206F6E000F
:1054B0006C7952004553450054424F004F544C0004
:1054C0004F4144004552410055582000494E50007C
:1054D00055542F0048492D005A2C200052454100B8
:1054E000443A2000504F5700455220005355500079
:1054F000504C4900455320004F4E50004F57450037
:1055000052205300555050004C49450053204F0045
:105510004646440041544100205354004154450044
:105520003A204400454C4100592075007357520001
:10553000495445003A205200454144003A20430076
:105540004C4F43004B2C200031434C004F434B0049
:105550002C2030004441540041204F00555450004D
:1055600055542C002031440041544100204F550037
:1055700054505500542C200030202A0070696E00D1
:1055800020697300206E6F0077204800695A43003D
:105590004C4F43004B20540049434B00533A2000EA
:1055A000524541004420420049543A0020537900BA
:1055B0006E7461007820650072726F007220610065
:1055C000742063006861720020782E0020657800E6
:1055D0006974280077697400686F7500742063002F
:1055E00068616E00676529006E6F20006D6F640052
:1055F0006520630068616E00676523003A204E00F5
:105600006F2073006F66740077617200652072000E
:105610006573650074206F006E207600342C2000C6
:1056200075736500207468006520720065736500FD
:1056300074206200757474006F6E2E004E6F6E00E1
:1056400065786900737465006E74200070726F0075
:10565000746F63006F6C2100782E200065786900FC
:10566000740D0A00496E7600616C69006420630065
:10567000686F690063652C002074720079206100F6
:10568000676169006E444500564944003A687400F9
:1056900074703A002F2F6400616E670065726F00AE
:1056A00075737000726F74006F74790070657300A9
:1056B0002E636F006D2A2D002D2D2D002D2D2D0018
:1056C0002D2D2D002A4F7000656E20006472610040
:1056D000696E20006F757400707574007320280067
:1056E000483D4800692D5A002C204C003D474E0093
:1056F00044294E006F726D00616C20006F7574005C
:105700007075740073202800483D33002E337600F6
:105710002C204C003D474E0044294D0053422000B0
:10572000736574003A204D004F5354002073690094
:1057300067206200697420006669720073744C000F
:1057400053422000736574003A204C0045415300D9
:105750005420730069672000626974002066690044
:105760007273740020426F006F746C006F6164008C
:1057700065722000762031002E20480045580D002B
:105780000A2032002E20440045430D000A20330039
:105790002E204200494E0D000A2034002E205200D7
:1057A00041574400697370006C61790020666F0096
:1057B000726D610074207300657456006F6C740024
:1057C00061676500206D6F006E6974006F72730011
:1057D0003A203500563A2000207C2000332E33003A
:1057E000563A2000207C2000565055004C4C550065
:1057F000503A20005365740020736500726961009F
:105800006C2070006F727400207370006565640016
:105810003A20280062707300290D0A0020312E0002
:1058200020333000300D0A0020322E0020313200AB
:1058300030300D000A2033002E203200343030008A
:105840000D0A2000342E200034383000300D0A00BC
:1058500020352E002039360030300D000A20360069
:105860002E20310039323000300D0A0020372E0052
:1058700020333800343030000D0A2000382E20004C
:105880003537360030300D000A2039002E20310027
:105890003135320030300D000A3130002E20420008
:1058A0005247200072617700207661006C756500B8
:1058B00041646A007573740020796F00757220006E
:1058C000746572006D696E00616C41007265200044
:1058D000796F75002073750072653F0020434600A4
:1058E00047313A002043460047323A00285C2D00F9
:1058F0002F5F5C002D2928005C5F2F002D295300AD
:10590000656C6500637420006F75740070757400B9
:105910002074790070653A000D0A2000312E2000B5
:105920004F7065006E206400726169006E2028006F
:10593000483D4800692D5A002C204C003D474E0040
:1059400044290D000A2032002E204E006F726D0097
:10595000616C200028483D00332E3300562C200077
:105960004C3D47004E442900523257002028730016
:105970007064200068697A00293D280020203000EA
:105980002E4D610063726F00206D65006E750D0015
:105990000A2031002E4953004F37380031362D0090
:1059A0003320410054520D000A2032002E4953008A
:1059B0004F37380031362D0033207000617273008C
:1059C00065206F006E6C790049534F002037380016
:1059D00031362D003320410054522000285245001A
:1059E00053455400206F6E0020435300290D0A00D8
:1059F000524553004554200048494700482C200098
:105A0000434C4F00434B2000544943004B2C200093
:105A100052455300455420004C4F570049534F0006
:105A20002037380031362D003320720065706C004D
:105A30007920280075736500732063007572720009
:105A4000656E7400204C530042207300657474002E
:105A5000696E6700293A200050726F00746F63000E
:105A60006F6C3A0020736500726961006C3320002E
:105A700077697200653220007769720065524600CE
:105A800055756E006B6E6F00776E52006561640035
:105A90002074790070653A0020746F0020656E00F4
:105AA0006476610072696100626C6500206C65005B
:105AB0006E6774006844610074612000756E69004F
:105AC00074733A00206E6F0020696E006469630091
:105AD000617469006F6E44006174610020756E002E
:105AE000697420006C656E0067746800202862008D
:105AF00069747300293A200043532000454E410049
:105B0000424C450044435300204449005341420065
:105B10004C45440052335700202873007064200025
:105B200063736C00206869007A293D0028202900F1
:105B30000D0A4400697363006F6E6E006563740044
:105B400020616E00792064006576690063657300EA
:105B50000D0A43006F6E6E006563740020285600C6
:105B600070752000746F20002B35560029206100CD
:105B70006E64200028414400432074006F202B00F5
:105B8000332E33005629430074726C00415558007F
:105B90004D4F440045204C0045445000554C4C00AE
:105BA00055502000485055004C4C550050204C009A
:105BB0005652450047414400432061006E64200076
:105BC00073757000706C790035565600505533006F
:105BD0002E3356004144430042757300206869002B
:105BE000676842007573200048692D005A20300014
:105BF00042757300204869002D5A2000314D4F0036
:105C000044452000616E6400205652004547200044
:105C10004C45440073207300686F75006C6420006D
:105C2000626520006F6E2100466F75006E64200073
:105C300020657200726F7200732E4D004F53490041
:105C4000434C4B004D4953004F435300204F4B00F2
:105C500020464100494C5300657420007370650074
:105C600065643A000D0A2000312E200033304B00CD
:105C7000487A0D000A2032002E20310032354B00C8
:105C8000487A0D000A2033002E20320035304B00B8
:105C9000487A0D000A2034002E2031004D487A0049
:105CA000436C6F00636B2000706F6C006172690061
:105CB00074793A000D0A2000312E200049646C00EE
:105CC00065206C006F7720002A64650066617500AE
:105CD0006C740D000A2032002E204900646C6500AF
:105CE0002068690067684F00757470007574200043
:105CF000636C6F00636B200065646700653A0D009C
:105D00000A2031002E204900646C650020746F0069
:105D10002061630074697600650D0A0020322E0050
:105D20002041630074697600652074006F2069006B
:105D3000646C6500202A640065666100756C7400FF
:105D4000496E70007574200073616D00706C6500A1
:105D500020706800617365003A0D0A0020312E0042
:105D6000204D690064646C0065202A00646566004B
:105D700061756C00740D0A0020322E0020456E0003
:105D800064535000492028007370640020636B0046
:105D9000702073006B652000736D700020637300CA
:105DA0006C206800697A29003D28200020302E00F0
:105DB0004D616300726F20006D656E00750D0A0005
:105DC00020312E00536E6900666620004353200088
:105DD0006C6F77000D0A2000322E53006E6966004A
:105DE000662061006C6C2000747261006666690058
:105DF000632D7000202D6600202A42007974650012
:105E000073206400726F7000706564002A46410060
:105E1000494C4500442C20004E4F20004441540082
:105E20004144610074612000626974007320610064
:105E30006E64200070617200697479003A0D0A0086
:105E400020312E0020382C00204E4F004E452000DF
:105E50002A646500666175006C7420000D0A2000DC
:105E6000322E2000382C2000455645004E200D00D3
:105E70000A2033002E2038002C204F0044442000FC
:105E80000D0A2000342E2000392C20004E4F4E00E9
:105E9000455374006F70200062697400733A0D00FE
:105EA0000A2031002E203100202A6400656661003E
:105EB000756C74000D0A2000322E200032526500ED
:105EC0006365690076652000706F6C00617269001F
:105ED00074793A000D0A2000312E200049646C00CC
:105EE00065203100202A640065666100756C7400CD
:105EF0000D0A2000322E200049646C00652030001D
:105F000055415200542028007370640020627200D2
:105F10006720640062702000736220007278700055
:105F2000206869007A293D0028202000302E4D008D
:105F3000616372006F206D00656E75000D0A2000B0
:105F4000312E540072616E007370610072656E00D4
:105F5000742062007269640067650D000A203200D7
:105F60002E4C6900766520006D6F6E0069746F00BD
:105F7000720D0A0020332E004272690064676500CA
:105F80002077690074682000666C6F0077206300DA
:105F90006F6E7400726F6C000A0D2000342E410089
:105FA00075746F00204261007564200044657400C0
:105FB00065637400696F6E005541520054206200A1
:105FC000726964006765520065736500742074002F
:105FD0006F20650078697400526177002055410098
:105FE00052542000696E700075745500415254007F
:105FF000204C49005645200044495300504C410074
:10600000592C20007D2054004F205300544F500045
:106010004C49560045204400495350004C4159001A
:10602000205354004F5050004544570041524E00F9
:10603000494E47003A207000696E7300206E6F0071
:1060400074206F0070656E002064720061696E00DC
:1060500020284800695A290020524500564944002A
:106060003A0D0A00496E7600616C69006420630095
:10607000686F690063652C002074720079206100EC
:10608000676169006E6D7300525320004C4F5700DA
:106090002C2043004F4D4D00414E4400204D4F00F9
:1060A0004445520053204800494748002C204400F2
:1060B00041544100204D4F0044454100646472004A
:1060C00065737300206F660020504300463835002A
:1060D00037343F005468690073206D006F646500B9
:1060E00020726500717569007265730020616E0031
:1060F000206164006170740065724C0043442000AC
:1061000074797000653A0D000A2031002E20480095
:1061100044343400373830002028750073696E002D
:1061200067205000434638003537340020494F007F
:106130002065780070616E0064657200294C430030
:106140004420280074797000206164006472290082
:10615000203D200028202000302E4D006163720079
:106160006F206D00656E75000D0A2000312E4C0009
:10617000434420005265730065740D000A2032000C
:106180002E496E00697420004C4344000D0A200023
:10619000332E43006C65610072204C0043440D00B7
:1061A0000A2034002E43750072736F007220700055
:1061B0006F73690074696F006E206500783A28007B
:1061C00034292000300D0A0020362E005772690055
:1061D000746520007465730074206E00756D620034
:1061E00065727300206578003A283600292038004F
:1061F000300D0A0020372E005772690074652000A8
:1062000074657300742063006861720061637400D8
:1062100065727300206578003A283700292038001D
:106220003044690073706C00617920006C696E0005
:1062300065733A000D0A2000312E200031200D0038
:106240000A2032002E204D00756C740069706C00BD
:1062500065494E00495443004C45410052435500A6
:1062600052534F005220530045544E006F204100BE
:10627000434B2C002063680065636B002061640061
:1062800061707400657243004C4B09004D4F530020
:106290004909430053094D0049534F0050696E00AE
:1062A00073746100746573003A474E00440933000B
:1062B0002E33560009352E00305609004144430064
:1062C0000956500055094100555809005009500021
:1062D0000950090049094900092D09004F57440098
:1062E000092D09002D2D090054784400092D0900BD
:1062F0005278440053434C000953440041092D0097
:10630000092D50004743090050474400092D09005A
:106310002D312E0028425200290932002E28520029
:1063200044290900332E28004F52290009342E0039
:1063300028595700290935002E2847004E29090001
:10634000362E2800424C290009372E0028505500CF
:10635000290938002E28470052290900392E280023
:106360005754290009302E0028426C006B29470041
:106370004E440900474E440009414400430935009A
:106380002E30560009332E00335609005650550062
:10639000094155005809650078656300757465000A
:1063A000203A200020617500746F7200616E6700F2
:1063B00065202B004D487A00292B6B00487A290074
:1063C00052617700207661006C75650020666F0071
:1063D0007220420052472000284D490044493D00A8
:1063E0003132370029574100524E49004E473A009A
:1063F00020506F0073736900626C65002062750045
:1064000066666500726F7600657266006C6F770075
:10641000416E7900206B6500792074006F20650063
:10642000786974005370610063652000746F200008
:10643000636F6E0074696E0075654E00756D620065
:10644000657220006F66200062697400732072001C
:10645000656164002F777200697465003A2043001B
:10646000533A0D000A2031002E204300530D0A003C
:1064700020322E00202F430053202A00646566003E
:1064800061756C0074506F0073697400696F6E0001
:1064900020696E00206465006772650065735300B3
:1064A000657276006F20610063746900766557003D
:1064B00061697400696E6700206163007469760029
:1064C00069747900206F6E00204D4900534F200001
:1064D00028416E0079206B0065792000746F2000E0
:1064E0006578690074292E002A2A2000456172000F
:1064F0006C7920004578690074212A005761720088
:106500006E696E00672A200042617500643E3100AA
:10651000366D3A0020546800652042005020690022
:1065200073206E006F742000666173007420650034
:106530006E6F750067682000746F20006D656100E4
:1065400073757200652062006175640073206100DC
:10655000626F760065203100363030003030300018
:10656000302C2000446F6E00652E0A000D41630040
:10657000747561006C204300616C6300756C610090
:1065800074656400204261007564200052617400EB
:10659000653A2000090A0D004E65610072657300BE
:1065A000742043006F6D6D006F6E200042617500B6
:1065B00064205200617465003A2009002062700076
:1065C00073204700656E650072616C00090909005F
:1065D00009095000726F74006F636F006C206900CE
:1065E0006E7465007261630074696F006E202D0027
:1065F0002D2D2D002D2D2D002D2D2D002D2D2D007F
:106600002D2D2D002D2D2D002D2D2D002D2D2D006E
:106610002D2D2D002D2D2D002D2D2D002D2D2D005E
:106620002D2D2D002D2D2D002D2D2D002D2D2D004E
:106630002D2D2D002D2D2D002D2D2D002D2D2D003E
:106640002D2D2D002D2D2D002D2D2D002D2D2D002E
:106650002D2D20003F0954006869730020686500F3
:106660006C70090009092800302909004C69730081
:106670007420630075727200656E7400206D610095
:1066800063726F0073203D00582F7C00580943004F
:106690006F6E760065727400732058002F7265006B
:1066A0007665720073652000580909002878290072
:1066B000094D610063726F00207820007E0953004D
:1066C000656C66007465730074090900095B090054
:1066D00053746100727420002309520065736500D1
:1066E00074207400686520004250200020200900BA
:1066F00009095D00095374006F70200024094A00E5
:10670000756D700020746F0020626F006F746C00F4
:106710006F61640065720900097B090053746100B0
:1067200072742000776974006820720065616400EB
:1067300020262F0025094400656C61007920310076
:10674000207573002F6D7300090909007D0953003E
:10675000746F700020612F00412F400009415500E7
:10676000585049004E2028006C6F77002F48490090
:106770002F5245004144290009092200616263004B
:1067800022095300656E64002073740072696E0004
:10679000672062000953650074206200617564001F
:1067A0007261740065090900093132003320630009
:1067B0002F43090041555800206173007369670039
:1067C0006E6D65006E74200028617500782F43009F
:1067D00053290900093078003132330020642F003A
:1067E00044094D00656173007572650020414400E5
:1067F000432028006F6E6300652F43004F4E540006
:106800002E290900306231003130090053656E00D5
:1068100064207600616C750065206600094D650096
:1068200061737500726520006672650071756500A0
:106830006E637900090972000952650061642000E5
:10684000672F5300094765006E657200617465002B
:10685000205057004D2F5300657276006F090900D4
:106860002F0943004C4B2000686920006809430051
:106870006F6D6D00616E640068697300746F720003
:1068800079090900095C0900434C4B00206C6F003A
:10689000206909005665720073696F006E696E00A9
:1068A000666F2F007374610074757300696E660003
:1068B0006F0909005E0943004C4B200074696300B6
:1068C0006B206C002F4C0900426974006F726400E9
:1068D00065722000286D7300622F4C00534229001E
:1068E00009092D00094441005420680069206D0009
:1068F00009436800616E670065206D006F64650084
:10690000090909005F094400415420006C6F200010
:106910006F095300657420006F7574007075740002
:10692000207479007065090009092E0009444100AE
:10693000542072006561640020702F0050095000DF
:10694000756C6C007570200072657300697374005B
:106950006F72730020286F0066662F004F4E29006B
:1069600009210900426974002072650061642000F9
:10697000730953006372690070742000656E6700CC
:10698000696E6500090909003A09520065706500E1
:1069900061742000652E67002E2072003A313000AD
:1069A0002076090053686F00772076006F6C7400C2
:1069B000732F73007461740065730900093B09004B
:1069C00042697400732074006F2072006561640076
:1069D0002F7772006974650020652E00672E2000F5
:1069E00030783500353B320020772F0057095000B2
:1069F00053552000286F6600662F4F004E2909006E
:106A0000093C78003E2F3C00783D20003E2F3C00A2
:106A1000303E090055736500726D610063726F004E
:106A200020782F006173730069676E0020782F0053
:106A30006C697300742061006C6C00000400FA0043
:106A400006960200000000000004E0002200320070
:106A500032C2BF00684060000004E0000400320061
:106A60003100200040CF2000D6920200000000003C
:106A700032C2BF00644060000004E0000400320045
:106A80003100200070CF2000D692020000000000EC
:106A9000F695020000000000000F780032C2BF002F
:106AA000624060000004E00008003200F1002000B5
:106AB000A0CF2000D69202000000000090118000BC
:106AC000D1FF2F0001006000901188001E007800A7
:106AD0001007980006003700F100200090D0200039
:106AE000D6920200000000000000EB0010079800A2
:106AF0001E0090000080FA00000006000200FA006C
:106B0000000F78001E007800E295020000000000EF
:106B10000000EB000080FA00000006000000FA0010
:106B200001022000F0DB2000D692020000000000ED
:106B300060AD200010407800CC6902000000000029
:106B400000C2B300446C02000000000060AD2000F1
:106B500010407800E94F500007003A00C011800053
:106B60006E6902000000000000C2B300446C020025
:106B7000000000000C00370060AD200010407800DD
:106B80000080FB0080004000E0AA20000080400060
:106B9000100078006E6902000000000000C2B3001F
:106BA000446C02000000000000D320001040780078
:106BB00063406000CC6902000000000000C2B30026
:106BC000446C02000000000000D320001040780058
:106BD0000080FB004200DE0061406000CC690200E2
:106BE0000000000000C2B300446C0200000000007E
:106BF00000D32000104078000080FB004300DE003E
:106C000061406000CC6902000000000000C2B300D7
:106C1000446C02000000000080AE200010407800AC
:106C20000080FB004400DE0061406000CC6902008F
:106C30000000000000C2B300446C0200000000002D
:106C40003100200020AE2000D6920200000000009B
:106C50000080FA00000006000C00FA000000EB00C3
:106C6000000F7800A01F020000000000D21B0200ED
:106C700000000000500798005E009000EA0F5000EE
:106C800005003A00A01F020000000000D21B020015
:106C900000000000000F7800A01F020000000000AC
:106CA000D21B02000000000040079800A01F020055
:106CB00000000000D21B0200000000003007980016
:106CC000A01F020000000000D21B02000000000014
:106CD00020079800A01F020000000000D21B020045
:106CE00000000000100798005E0090000000E00027
:106CF000090034005E009000EA0F500006003C00DE
:106D00005E0090000040E9008040780060AD200007
:106D100001487800020037000000EB00500798009F
:106D20004E0090000000E0000F0034004E00900084
:106D3000E40F50000C003C004E0090000040E900C1
:106D4000E340600000D320001040780063C1600081
:106D5000C1CFB300014060000240700001D32000A9
:106D600080487800020037000000EB0050079800D0
:106D70003E0090000000E000100034003E00900053
:106D8000E20F50000D003C003E0090000040E90082
:106D90006141600000D320009040780061406100B4
:106DA0004201DD00B0CFB30080C0600082C070003F
:106DB00000D3200001487800020037000000EB00FB
:106DC000500798002E0090000000E00010003400F2
:106DD0002E009000E20F50000D003C002E009000AD
:106DE0000040E9006141600000D32000904078003D
:106DF000614061004301DD0070CFB30080C06000DE
:106E000082C0700000D320000148780002003700E3
:106E10000000EB00500798001E0090000000E0000A
:106E2000100034001E009000E20F50000D003C00E6
:106E30001E0090000040EA006141600080AE20002A
:106E400090407800614061004401DD00F0CEB30065
:106E500080C0600082C0700080AE200001487800D1
:106E6000020037000000EB00500798005E00900021
:106E70000000E00073003A000000EB00106488009E
:106E8000D10820006087200060930200000000000D
:106E90008001EB00A2002000110020001000200063
:106EA000CC200200000000000040E9008040780093
:106EB00060AD20000148780060AD200010407800EF
:106EC000E94F50000B003A00C1012000F0142100EE
:106ED00060930200000000008001EB00F2FF270039
:106EE0001100200020022000CC2002000000000041
:106EF000000F78004105200080D12000D6920200CA
:106F0000000000008001EB00420020001100200082
:106F100010002000CC200200000000000040E9002A
:106F2000E340600000D320001040780063C160009F
:106F3000C1CFB300014060000240700001D32000C7
:106F40008048780011022000C0D62000D6920200AE
:106F5000000000008001EB00220020001100200052
:106F600010002000CC200200000000000040E900DA
:106F70006141600000D320009040780061406100D2
:106F80004201DD00B0CFB30080C0600082C070005D
:106F900000D320000148780021032000D0D8200031
:106FA000D6920200000000008001EB0022002000C9
:106FB0001100200010002000CC2002000000000082
:106FC0000040E9006141600000D32000904078005B
:106FD000614061004301DD0070CFB30080C06000FC
:106FE00082C0700000D3200001487800F104200026
:106FF000E093200060930200000000008001EB009D
:10700000220020001100200010002000CC200200EF
:10701000000000000040EA006141600080AE2000F6
:1070200090407800614061004401DD00F0CEB30083
:1070300080C0600082C0700080AE200001487800EF
:1070400001003700B5FE070060AD20001040780059
:10705000E94F50001C003A0000D320001040780097
:107060000080FB004200DE0061406000804178004B
:1070700000D3200010407800634060008042780018
:1070800000D32000104078000080FB004300DE00A9
:10709000614060000041780080AE20001040780020
:1070A0000080FB004400DE0061406000804078000A
:1070B0001E00780003427800854178003695020072
:1070C000000000002200370000D3200010407800AC
:1070D0000080FB004200DE0061406000004178005B
:1070E00000D32000104078006340600080417800A9
:1070F00000D32000104078000080FB004300DE0039
:10710000614060008042780080AE2000104078002E
:107110000080FB004400DE00614060000043780016
:1071200060AD2000104078000080FB00800040002F
:10713000E0AA2000008040001000780002427800A1
:107140000541780086407800369502000000000076
:1071500000D320001040780063406000E34F5000EF
:1071600003003A0091C0B30070AD200001487800E0
:10717000BA95020000000000C1118000401180009B
:10718000808F50000400310001022000B016210061
:1071900060930200000000000080FA00000006007A
:1071A0000000FA00C6950200000000000080FA000E
:1071B000000006000400FA00000F78001E007800AE
:1071C000100798001E009000E20F50006D00320082
:1071D0001E009000E20F500007003E001E009000CD
:1071E0000000E0000B0032001E009000E10F500094
:1071F00011003200910037001E009000E30F500094
:10720000090032001E009000E40F50007C003200A4
:107210008A003700A1062000F0DD2000D69202008F
:107220000000000089003700C062A900C082A800E9
:10723000C8C2A800C902A900B100200090E4200043
:107240006093020000000000D100200040E5200013
:10725000609302000000000006940200000000009D
:107260000000E0007900320090118000D1FF2F0073
:1072700001006000901188000000370032C2BF009A
:10728000614060000004E0000600320023C2BF003D
:10729000624060000004E00002003A00B01180008B
:1072A00020118800666B020000000000E14F5000D2
:1072B00008003A0033C2BF00624060000004E000F2
:1072C00004003A00246C0200000000000080FB0073
:1072D000A011880032C2BF00624060000004E000DC
:1072E00004003A0022C2BF00624060000004E000D7
:1072F0000900320091118000D0FF2F000080600053
:107300009011880011118000D0FF2F0000806000D4
:1073100010118800C222A900300020009E0F10002A
:10732000D6FF3A00C2C2BF000080FB004400DE006E
:107330006140600061416000B12C20009140780004
:10734000E0CFB30000C0600002407000CBE2B700A5
:10735000CAC2BF000080FB004600DE006140600042
:10736000614060004301DD00212C20009140780045
:1073700070CFB30000C0600002407000C2E2B700EE
:10738000BEFF3700E100200010E6200060930200FD
:1073900000000000F1002000B018210060930200FE
:1073A0000000000090118000D1FF2F00010060005C
:1073B0009011880032C2BF00614060000004E0000C
:1073C0000600320023C2BF00624060000004E000FB
:1073D00002003A00B011800020118800666B0200A4
:1073E00000000000E14F5000F2FF3A00246C020060
:1073F000000000000080FB00000F78001300370041
:10740000C6950200000000000000EB008A010700A2
:10741000BA95020000000000C111800040118000F8
:10742000808F50000900310001022000B0162100B9
:1074300060930200000000000400370041022000B9
:10744000E01D200060930200000000000080FA00B0
:10745000000006000000FA0091118000D0FF2F000C
:10746000008060009011880000D320001040780058
:107470000040A00001D320008048780080AE2000AA
:10748000104078000020A00081AE200080487800E5
:10749000C1012000F0E6200060930200000000001F
:1074A0000080FA00000006000000FA0000D320006F
:1074B000104078000040A10001D3200080487800EF
:1074C00080AE2000104078000020A10081AE200096
:1074D0008048780041012000B0E82000609302005D
:1074E000000000000080FA00000006000200FA0020
:1074F0000000EB00000F78003400370000D32000BC
:1075000010407800704060000004E0002B00320062
:10751000E086280060670200000000006100200093
:1075200080662000D69202000000000032C2BF0038
:10753000684060000004E0000400320031002000D8
:1075400040CF2000D69202000000000032C2BF00EF
:10755000644060000004E0000400320031002000BC
:1075600070CF2000D692020000000000F6950200C5
:1075700000000000869102000000000032C2BF003F
:10758000624060000004E00008003200F1002000CA
:10759000A0CF2000D69202000000000090118000D1
:1075A000D1FF2F000100600090118800E0862800C4
:1075B000606702000000000002003700F69502003C
:1075C0000000000010002000000F78000696020066
:1075D000000000000004E000C8FF3A001E00780030
:1075E0000080FA00000006000000FA00B100200050
:1075F000B00A210060930200000000000080FA0041
:10760000000006000000FA000000EB00F00888000F
:107610000000EB00800888008000200080088800BF
:107620000000EB00400888000000EB0030088800F4
:107630000000EB00B00888000000EB00A008880004
:1076400080002000F00888000080FA00000006009A
:107650000000FA0011E1A9001FE1A90086C6BF00E1
:10766000F041B30086E6B7000000EB00F0088800A8
:107670000000EB00800888000000EB003008880064
:107680000000EB00400888000080FA0000000600BF
:107690000800FA00008FBE00900F200001002000BB
:1076A000BE0F1000AE8F18000A003600201C20000C
:1076B00001002000BE0F1000AE8F180005003E0034
:1076C000C012200001002000200798003107980018
:1076D000D5003700201C200001002000BE0F100044
:1076E000AE8F18000A00360040382000010020004C
:1076F000BE0F1000AE8F180005003E008025200050
:10770000010020002007980031079800C6003700CC
:107710004038200001002000BE0F1000AE8F18007E
:107720000A0036008070200001002000BE0F10000B
:10773000AE8F180005003E00004B20000100200025
:107740002007980031079800B700370080702000AC
:1077500001002000BE0F1000AE8F18000A00360096
:10776000C0DA200001002000BE0F1000AE8F18000C
:1077700005003E0000962000010020002007980030
:1077800031079800A8003700C0DA2000010020006F
:10779000BE0F1000AE8F18000A00360000C2210094
:1077A00001002000BE0F1000AE8F180005003E0043
:1077B000002C2100010020002007980031079800CC
:1077C0009900370000C2210001002000BE0F100008
:1077D000AE8F18000A00360000EE220001002000E3
:1077E000BE0F1000AE8F180005003E0000582200AA
:1077F0000100200020079800310798008A00370018
:1078000000EE220001002000BE0F1000AE8F180015
:107810000A003600001A240001002000BE0F1000EC
:10782000AE8F180005003E000084230001002000F8
:1078300020079800310798007B003700001A2400C9
:1078400001002000BE0F1000AE8F18000A003600A5
:107850000046250001002000BE0F1000AE8F18006A
:1078600005003E0000B02400010020002007980021
:10787000310798006C003700004625000100200009
:10788000BE0F1000AE8F18000A003600009E2700C1
:1078900001002000BE0F1000AE8F180005003E0052
:1078A00000082700010020002007980031079800F9
:1078B0005D003700009E270001002000BE0F100071
:1078C000AE8F18000A00360000F6290001002000E3
:1078D000BE0F1000AE8F180005003E0000602900AA
:1078E0000100200020079800310798004E00370063
:1078F00000F6290001002000BE0F1000AE8F180016
:107900000A00360000DE2D0001002000BE0F10002E
:10791000AE8F180005003E0000AC2D0001002000D5
:1079200020079800310798003F00370000DE2D0047
:1079300001002000BE0F1000AE8F18000A003600B4
:107940000018250011002000BE0F1000AE8F180097
:1079500005003E0000102E000100200020079800C6
:107960003107980030003700001825001100200072
:10797000BE0F1000AE8F18000A00360000B02D00B8
:1079800011002000BE0F1000AE8F180005003E0051
:1079900000202C00110020002007980031079800DB
:1079A0002100370000B02D0011002000BE0F100094
:1079B000AE8F18000A00360000E02E0021002000E3
:1079C000BE0F1000AE8F180005003E0000402F00D3
:1079D000110020002007980031079800120037009E
:1079E00000E02E0021002000BE0F1000AE8F180016
:1079F0000A003600003E290041002000BE0F1000A2
:107A0000AE8F180005003E0000802E0031002000DF
:107A10002007980031079800030037006000B80085
:107A200020079800310798002E009000BE009000BB
:107A30000080FA00000006001000FA0050079800CD
:107A40000000EB00400798006000B8002007980095
:107A5000310798006000B800008FBE00CAE2A9009C
:107A6000C8E2A8005E0090000000E00006003A00B6
:107A7000B1022000202021006093020000000000DD
:107A80000100370000000000CAC2BF0001C8B300F7
:107A9000014060000004E0000400320022C2BF0088
:107AA000614060000004E000F6FF320022C2BF0027
:107AB000614060000004E0000B00320030118000E3
:107AC00040079800E2FE0700E1002000D0222100DC
:107AD00060930200000000006000B800600798009A
:107AE00071079800750037000000EB004007980010
:107AF00041003700C3FE0700CAC2BF0001C8B3007F
:107B0000014060000004E000FBFF32001FE1A8001C
:107B100011E1A800CAC2BF0001C8B3000140600063
:107B20000004E000FBFF3A0011E1A9001FE1A900F9
:107B300086C6BF00F041B30086E6B7000000EB0048
:107B4000F00888000000EB008008880040088000F2
:107B50000100200020079800310798002E009000B7
:107B6000BE009000C000DD0000002000200798004B
:107B700031079800300880006101B8002E009000A5
:107B8000BE0090000000410081804900200798005D
:107B9000310798004E0090000000E0001000320015
:107BA0001E00BE00E00F5000E08F580004003A00B5
:107BB0002E009000BE009000008FBE00080037002D
:107BC0002E009000BE009000BE0F1000AE8F180077
:107BD000030036002E009000BE009000008FBE0013
:107BE0006000B80020079800310798004E00900010
:107BF0000000E800400798004E009000F80F500089
:107C0000BCFF360092FE07001E01BE0000402200AD
:107C1000410F20002406020000000000008FBE007B
:107C20005E0090000000E00021003A00009F240068
:107C300021002000BE0F1000AE8F18000500360096
:107C400041052000B02321006093020000000000E5
:107C50001700370001022000F0282100D692020010
:107C6000000000001E00BE00CE6702000000000001
:107C700041002000C02C21006093020000000000A1
:107C8000D1012000F02A2100D6920200000000005D
:107C90001E00BE007EFE0700CE670200000000004E
:107CA00041002000C02C2100609302000000000071
:107CB0001E00BE0060079800710798006E009000DB
:107CC000FE0090000080FA00000006000000FA00AC
:107CD000F086280034670200000000000080FA00EF
:107CE000000006000400FA0000D3200010407800D5
:107CF0000000A1000010A10001D3200080487800FE
:107D000000D32000104078000020A10001D3200003
:107D10008048780000D32000104078000030A10097
:107D200001D320008048780080AE20001040780009
:107D30000040A00081AE20008048780010568000EE
:107D40005069880000D32000104078000040A10056
:107D500001D320008048780000D320001040780034
:107D60000080FB004200DE0061406000804178003E
:107D700000D320001040780063406000804278000B
:107D800000D32000104078000080FB004300DE009C
:107D9000614060000041780080AE20001040780013
:107DA0000080FB004400DE006140600080407800FD
:107DB00050698000034278008541780036950200C2
:107DC00000000000BA95020000000000BFFF07009D
:107DD0000000370006960200000000000004E000EA
:107DE0000C00320000D3200010407800704060008A
:107DF0000004E00005003200F695020000000000DB
:107E0000446C02000000000002003700F6950200FA
:107E10000000000032C2BF00624060000004E000C9
:107E20000400320090118000D1FF2F00010060009B
:107E300090118800666B020000000000E14F5000C6
:107E4000E4FF3A00246C020000000000804078004B
:107E5000E0D2200001487800E0D2200010407800F5
:107E60000080FB004400DE0080407800D0D220007B
:107E700001487800D0D22000104078000080FB003C
:107E8000100798001E009000E40F5000CC00320054
:107E90009E009000E48F500007003C001E00900000
:107EA0000000E0000F0032009E009000E18F5000C3
:107EB0009D003200860137001E009000E60F500042
:107EC000C70032009E009000E68F50008001350010
:107ED0009E00900068805000E10F50007C013E0041
:107EE000F7003700E0D22000104078000080FB004F
:107EF000000F78001E007800E20F500019003200D9
:107F00009E007800E28F500007003C001E007800C1
:107F10000000E0000E0032009E007800E18F50006B
:107F20000E0032007C0037001E007800E70F500082
:107F3000260032009E007800EF8F5000570032007C
:107F40001E007800E30F5000170032007200370067
:107F5000C695020000000000610137005BFF0700CA
:107F60009CFF370010C0B300446C0200000000000A
:107F700032C2BF00624060000004E0000400320032
:107F800090118000D1FF2F00010060009011880047
:107F900000D32000104078000040A00001D3200052
:107FA000804878008BFF370000D320001040780015
:107FB0000040A10001D320008048780010C0B30029
:107FC000446C02000000000082FF370010C0B300C4
:107FD000446C020000000000C69502000000000092
:107FE000246C0200000000000080FB004800DD005F
:107FF0005069880010C0B300446C0200000000000B
:10800000246C0200000000008080FB0050698000AA
:10801000008070005069880000D320001040780074
:108020000080FB004200DE0061406000804178007B
:1080300000D3200010407800634060008042780048
:1080400000D32000104078000080FB004300DE00D9
:10805000614060000041780080AE20001040780050
:108060000080FB004400DE0061406000804078003A
:1080700050698000034278008541780036950200FF
:1080800000000000BA9502000000000010C0B3001C
:10809000446C0200000000004EFF370010C0B30027
:1080A000446C02000000000090118000D1FF2F00FE
:1080B00001006000901188000000370032C2BF004C
:1080C000614060000004E0000600320023C2BF00EF
:1080D000624060000004E00002003A00B01180003D
:1080E00020118800666B020000000000E14F500084
:1080F000F2FF3A0033C2BF00624060000004E000BB
:10810000EEFF3A00246C0200000000000080FB003B
:10811000A0118800E9FF37000040EB00446C02002A
:10812000000000002BFF3700E0D2200090407800D4
:10813000F0C0B30080C06000E0D2200001487800A9
:10814000E0D22000104078008040E800E0D220001B
:108150000148780010C0B300446C02000000000029
:108160008040EB00C0D22000014878000D003700AD
:10817000246C0200000000000080FB00E295020079
:108180000000000010C0B300446C020000000000BA
:10819000C0D22000104078008040E800C0D220000B
:1081A00001487800C0D2200090407800E0D2200042
:1081B0001040780080CF5000EDFF390005FF3700F8
:1081C000E0D2200010407800BA97020000000000C2
:1081D00010C0B300446C020000000000FDFE370038
:1081E000E0D2200090407800F0C0B30080C0600072
:1081F000E0D2200001487800E0D220001040780052
:10820000EA4F500003003600A1C0B300E0D22000C6
:1082100001487800E0D22000104078000080FB0088
:108220008000400020AC200000804000100078005A
:1082300050698800C69502000000000000D32000AD
:10824000104078000080FB004200DE0061406000CA
:108250008041780000D32000104078006340600027
:108260008042780000D32000104078000080FB009E
:108270004300DE00614060000041780080AE2000D5
:10828000104078000080FB004400DE006140600088
:108290008040780050698000034278008541780072
:1082A0003695020000000000BA95020000000000B0
:1082B00010C0B300446C020000000000C5FE37008F
:1082C00000D32000104078000000A1000010A100A1
:1082D00001D320008048780000D3200010407800AF
:1082E0000020A10001D320008048780000D32000A6
:1082F000104078000030A10001D3200080487800B1
:1083000080AE2000104078000040A10081AE200027
:1083100080487800E0D22000104078000080FB0008
:108320004300DE00610060000004E0000D00320048
:1083300000D3200010407800634060000014A000CB
:10834000E340600000D320001040780063C160006B
:10835000C1CFB300014060000240700001D3200093
:1083600080487800E0D22000104078000080FB00B8
:108370004200DE00610060000004E0000D003200F9
:1083800000D3200010407800634060000004A0008B
:10839000E340600000D320001040780063C160001B
:1083A000C1CFB300014060000240700001D3200043
:1083B00080487800E0D22000104078000080FB0068
:1083C0000000D100610060000004E0000500320000
:1083D00000D32000104078000020A00001D320002E
:1083E00080487800E0D22000104078000080FB0038
:1083F000610060000004E0000500320000D32000AE
:10840000104078000030A00001D3200080487800A0
:10841000E0D22000104078000080FB004400DE0025
:108420000000A200610060000004E00005003200CE
:1084300080AE2000104078000040A00081AE2000F7
:1084400080487800C69502000000000000D320009C
:10845000104078000080FB004200DE0061406000B8
:108460008041780000D32000104078006340600015
:108470008042780000D32000104078000080FB008C
:108480004300DE00614060000041780080AE2000C3
:10849000104078000080FB004400DE006140600076
:1084A0008040780050698000034278008541780060
:1084B0003695020000000000BA950200000000009E
:1084C00010C0B300446C02000000000041FE370001
:1084D0000040EB00446C0200000000003DFE37004D
:1084E0000080FA00000006000000FA0080AE2000C4
:1084F000104078000060A00081AE20008048780025
:1085000060AF200010407800684060000004E00088
:1085100002003200CAC2A90001003700CAC2A80086
:1085200060AF200010407800684060000004E00068
:1085300003003200F0C2B300446C020000000000EF
:10854000A100200090AB200060930200000000001A
:108550000080FA00000006000000FA0080AE200053
:10856000104078000060A10081AE200080487800B3
:1085700060AF200010407800684060000004E00018
:1085800002003200CAC2A90001003700CAC2A80016
:1085900060AF200010407800684060000004E000F8
:1085A00003003200F0C2B300446C0200000000007F
:1085B000A100200090AB20006093020000000000AA
:1085C0000080FA00000006000000FA0060AF200002
:1085D00010407800684060000004E00002003200B3
:1085E000CAC2A80001003700CAC2A90060AF2000BB
:1085F00010407800684060000004E0000300320092
:10860000F0C2B300446C020000000000B100200082
:1086100030AC200060930200000000000080FA00EF
:10862000000006000000FA0000C0EB008302070013
:108630000080FB000080FA00000006000600FA003F
:10864000100798001E0090007C020700004F780081
:1086500080AE2000104078000044B2000004E0002A
:10866000030032001E80FB00200798000200370044
:108670000000EB00200798002E0090000080FA0018
:10868000000006000000FA000102200000CA2000DD
:10869000D69202000000000060AD2000104078007B
:1086A0000040E800CC6902000000000000C2B300F6
:1086B000446C02000000000060AF20001040780011
:1086C00061406000CC6902000000000000C2B300FD
:1086D000446C02000000000060AF200010407800F1
:1086E0000080FB000000D10061406000CC69020006
:1086F0000000000000C2B300446C02000000000053
:1087000060AF2000104078000080FB004200DE00D7
:1087100061406000CC6902000000000000C2B300AC
:10872000446C02000000000060AF200010407800A0
:108730000080FB004300DE0061406000CC69020065
:108740000000000000C2B300446C02000000000002
:1087500080AE2000104078000080FB004400DE0066
:1087600061406000CC6902000000000000C2B3005C
:10877000446C0200000000003100200020AE200008
:10878000D6920200000000000080FA0000000600FF
:108790000C00FA00A01F020000000000D21B020023
:1087A0000000000050079800A01F02000000000019
:1087B000D21B02000000000040079800A01F02002A
:1087C00000000000D21B02000000000030079800EB
:1087D000A01F020000000000D21B020000000000E9
:1087E00020079800A01F020000000000D21B02001A
:1087F00000000000000F7800A01F02000000000031
:10880000D21B020000000000100798005E009000DC
:108810000000E000090034005E009000E40F50000A
:1088200006003C005E0090000040E90080407800B7
:1088300060AD200001487800020037000000EB0026
:10884000500798004E0090000000E0000F00340038
:108850004E009000E20F50000C003C004E009000D3
:108860000040E900E140600060AF20001040780067
:1088700061C16000E1CFB3000140600002407000C0
:1088800061AF200080487800020037000000EB0054
:10889000500798003E0090000000E00010003400F7
:1088A0003E009000E20F50000D003C003E009000A2
:1088B0000040E9006141600060AF20009040780016
:1088C0006140610000414000D0CFB30080C0600033
:1088D00082C0700060AF20000148780002003700BD
:1088E0000000EB00500798002E0090000000E00010
:1088F000100034002E009000E20F50000D003C00EC
:108900002E0090000040E9006141600060AF20004F
:1089100090407800614061004201DD00B0CFB300BB
:1089200080C0600082C0700060AF20000148780005
:10893000020037000000EB00500798001E00E00026
:1089400010003400200020009E0F10000D003C009D
:108950001E0078000040E9006141600060AF200027
:1089600090407800614061004301DD0070CFB300AA
:1089700080C0600082C0700060AF200001487800B5
:10898000020037000000EB00500798001E00900026
:108990000000E000100034001E009000E20F5000C4
:1089A0000D003C001E0090000040EA0061416000A4
:1089B00080AE200090407800614061004401DD00FD
:1089C000F0CEB30080C0600082C0700080AE200096
:1089D00001487800020037000000EB0050079800C3
:1089E0005E0090000000E00079003A000000EB001B
:1089F000106488007103200000BC20006093020016
:108A0000000000008001EB00420020001100200067
:108A100010002000CC200200000000000040E9000F
:108A20008040780060AD20000148780051032000AC
:108A300070BF200060930200000000008001EB0086
:108A4000220020001100200010002000CC20020095
:108A5000000000000040E900E140600060AF20003D
:108A60001040780061C16000E1CFB30001406000B8
:108A70000240700061AF200080487800310420007F
:108A8000C0C2200060930200000000008001EB00E3
:108A9000220020001100200020002000CC20020035
:108AA000000000000040E9006141600060AF20006C
:108AB000904078006140610000414000D0CFB30099
:108AC00080C0600082C0700060AF20000148780064
:108AD00011032000F0C62000609302000000000097
:108AE0008001EB0022002000110020001000200077
:108AF000CC200200000000000040E900614160005D
:108B000060AF200090407800614061004201DD00CC
:108B1000B0CFB30080C0600082C0700060AF2000A2
:108B200001487800D1012000601C21006093020000
:108B3000000000008001EB00220020001100200056
:108B400020002000CC200200000000000040E900CE
:108B50006141600060AF200090407800614061009A
:108B60004301DD0070CFB30080C0600082C07000A0
:108B700060AF200001487800F1042000E09320005D
:108B800060930200000000008001EB002200200042
:108B90001100200010002000CC2002000000000086
:108BA0000040EA006141600080AE20009040780003
:108BB000614061004401DD00F0CEB30080C0600080
:108BC00082C0700080AE20000148780001003700AC
:108BD000ACFE070080AE2000104078000060A100CD
:108BE00081AE20008048780060AD20001040780001
:108BF0008080FB00E0812000008040001040780071
:108C0000A600070060AF2000104078000080FB0045
:108C10004300DE0061406000614060004601DD000D
:108C2000A12C200091407800F0CBB30000C0600080
:108C300002407000CAE2B7000080FA00000006009F
:108C40000000FA00E90007000080FA0000000600BA
:108C50000600FA00000F78001E0078006101B800DD
:108C60001207980023079800F00020000100200060
:108C70001E019000AE019000800F5100818F5900BD
:108C800079003E001E009000AE00900000600100E0
:108C90000F003700130037001E0037007600370042
:108CA00071003700700037006F0037006E0037002A
:108CB0006D0037006C0037002200370027003700B6
:108CC0002C00370031003700360037003B003700FA
:108CD0004103200000CC200060930200000000004F
:108CE000650037007100200070562000609302007C
:108CF00000000000F1002000B01821006093020085
:108D00000000000011C0B3000040EB00D9000700D4
:108D10005900370071002000705620006093020057
:108D200000000000F1002000B01821006093020054
:108D30000000000011C0B30010C0B300CD00070058
:108D40004D00370060AF2000104078000000A10007
:108D500061AF2000804878001D00370060AF200020
:108D6000104078000000A00061AF2000804878002B
:108D70001700370060AF2000104078000010A100FD
:108D800061AF2000804878001100370060AF2000FC
:108D9000104078000010A00061AF200080487800EB
:108DA0000B00370060AF2000104078000020A100C9
:108DB00061AF2000804878000500370060AF2000D8
:108DC000104078000020A00061AF200080487800AB
:108DD00060AF20001040780061406000614060009A
:108DE0004601DD002124200091407800F0CBB30043
:108DF00000C060000240700042E2B70060AF200097
:108E0000104078000080FB000000D100614060004D
:108E1000614160003124200091407800E0CFB30030
:108E200000C060000240700043E2B70060AF200065
:108E3000104078000080FB004200DE0061406000CE
:108E400061406000004140003124200091407800E2
:108E5000D0CFB30000C060000240700043E2B70012
:108E600008FE07000400370041022000E01D20003A
:108E700060930200000000000080FA00000006007D
:108E80000000FA000101200040062100609302006A
:108E9000000000000080FA00000006000200FA0056
:108EA000004F780041E2A90080AE20001040780019
:108EB000704060000004E00004003200CEE2A80030
:108EC000CF02A800CEC2A80003003700CEE2A9005E
:108ED000CF02A900CEC2A900816A2000914078008B
:108EE00000CEB30000C060007040B300A8E6B70039
:108EF000916C20009140780000CEB30000C060006B
:108F00007040B300C9E6B700816C20009140780042
:108F100000CEB30000C060000034A000C8E6B70077
:108F2000CAC2A800C8C2A900C902A900C8E2A80014
:108F3000C922A9001E80FB001012880042A2A800CE
:108F400060AF200010407800614060006140600028
:108F50004601DD002124200091407800F0CBB300D1
:108F600000C060000240700042E2B70060AF200025
:108F7000104078000080FB000000D10061406000DC
:108F8000614160003124200091407800E0CFB300BF
:108F900000C060000240700043E2B70060AF2000F4
:108FA000104078000080FB004200DE00614060005D
:108FB0006140600000414000312420009140780071
:108FC000D0CFB30000C060000240700043E2B700A1
:108FD0000000EB00201288000000EB000012880067
:108FE00041E2A8000080FA00000006000000FA003C
:108FF00041E2A900A8C6BF00F041B300A8E6B7004F
:10900000916C20009140780000CEB30000C0600059
:10901000C9E6B700816C20009140780000CEB30013
:1090200000C06000C8E6B700CEE2A900CF02A900E8
:10903000CEC2A9000080FA00000006000200FA007B
:10904000004F78001E80FB004012880085C0BF00E2
:10905000644060000004E000FCFF32004012800029
:10906000004F78008540A9001E80FB000080FA00B8
:10907000000006000400FA002047980031479800DD
:1090800010C0B300004F7800726B020000000000B7
:10909000D6FF0700820007002E4090000004E00089
:1090A00002003A0042E2A80062E2A8002E409000CE
:1090B000E14F500002003E0041E2A80061E2A8003A
:1090C0001E04E00009003A00CAC2BF000044B2001A
:1090D0000004E00005003200D0C5B300EE6B0200D2
:1090E0000000000010C0B300004F780040C2BF0075
:1090F0000042B2000004E0002F003A0060C2BF004E
:109100000042B2000004E0002B003A004012800050
:109110001047980010C0B3009E4F100005003A00A1
:10912000B0C5B300EE6B0200000000000040EB0091
:10913000004F78003E4090000004E000050032003F
:109140001E4090000080FB00586A020000000000F2
:1091500006003700C0C5B300EE6B0200000000003F
:109160001E409000EE6B02000000000040138000E3
:10917000104798003E4090000004E0000B003200D1
:1091800080C2B300EE6B0200000000001E409000A1
:109190000080FB00586A02000000000090C2B3008B
:1091A000EE6B020000000000030037001E4090003C
:1091B000EE6B02000000000040C2BF000044B2009D
:1091C0000004E00009003A0060C2BF000044B200A1
:1091D0000004E00005003A00D0408000014020007B
:1091E000010060000000E00014003200D040800068
:1091F00001402000010060000000E00002003A0091
:10920000B86B0200000000000000EB0000128800B4
:109210000000EB00001388003E4090000004E000D6
:109220000400320040822800606702000000000055
:1092300093FF3700C222A9000F003700866B02009F
:1092400000000000666B020000000000E14F5000CB
:109250009BFF3A00246C02000000000010479800B9
:109260003E4090000004E0000300320050832800DC
:1092700060670200000000008800070060AD200069
:10928000104078008080FB00E081200000804000DA
:109290001040780001FF07000080FA00000006007F
:1092A0000000FA00C8C2A800C902A800C8E2A800CD
:1092B000C922A800A16A20009140780000CEB30026
:1092C00000C060006040B300AAE6B700E16A200079
:1092D0009140780000CEB30000C060006040B30051
:1092E000AEE6B700816A20009140780000CEB3005E
:1092F00000C060009040B300A8E6B700916A20006B
:109300009140780000CEB30000C060000034A0009F
:10931000A9E6B700C16A20009140780000CEB300F2
:1093200000C060007040B300ACE6B700D16A200016
:109330009140780000CEB30000C060000034A0006F
:10934000ADE6B70060AD2000104078008080FB00E3
:10935000E081200000804000104078000080FB0089
:109360001012880060AF200010407800614060005B
:10937000614060004601DD0021242000914078001A
:10938000F0CBB30000C060000240700042E2B700C2
:1093900060AF2000104078000080FB000000D1008A
:1093A00061406000614160003124200091407800FC
:1093B000E0CFB30000C060000240700043E2B7009D
:1093C0000000EB00201288000000EB000012880073
:1093D00060AD2000104078008080FB00E08120001C
:1093E00000804000104078000080FB0010138800CF
:1093F00060AF200010407800614060006140600074
:109400004601DD002126200091407800F0CBB3001A
:1094100000C060000240700062E2B70060AF200050
:10942000104078000080FB000000D1006140600027
:10943000614160003126200091407800E0CFB30008
:1094400000C060000240700063E2B7000000EB0063
:10945000201388000000EB00001388000000EB00E0
:10946000401288000000EB00401388004322A9004E
:109470006322A9004362A80042A2A9006362A80077
:1094800062A2A90040C2A90060C2A9004402A800CB
:109490006402A8000080FA00000006000000FA0044
:1094A00041E2A9004362A90061E2A9006362A90048
:1094B000AAC6BF00F041B300AAE6B700AEC6BF001F
:1094C000F041B300AEE6B700A8C6BF00F041B3005C
:1094D000A8E6B700A9C6BF00F041B300A9E6B700EF
:1094E000ACC6BF00F041B300ACE6B700ADC6BF00EC
:1094F000F041B300ADE6B7000080FA0000000600BE
:109500000000FA00608328003467020000000000B9
:109510000080FA00000006001400FA00881F78009E
:1095200011C0B30060AD20000148780060AF20009A
:10953000104078000000A10061AF20008048780052
:1095400060AF2000104078000010A00061AF200044
:109550008048780060AF2000104078000020A10013
:1095600061AF20008048780080AE20001040780075
:109570000040A00081AE20008048780060AD20004F
:10958000104078008080FB00208220000080400096
:109590001040780041FE0700D9FF070000003700A7
:1095A000246C0200000000008040780040AF2000E2
:1095B0000148780040AF2000104078000080FB0098
:1095C0004400DE008040780030AF20000148780081
:1095D00030AF2000104078000080FB00100F980092
:1095E0001E089000E40F5000A90132009E08900070
:1095F000E48F500007003C001E0890000000E000CF
:109600000B0032009E089000E18F50007D01320077
:109610000B0237001E089000E60F5000A401320034
:109620009E089000E88F5000B60132000402370017
:1096300040AF2000104078000080FB00000F980031
:109640000E089000E50F500014003C008E089000BA
:10965000E48F50003D003D000E089000E10F5000E7
:109660001A0032008E089000E18F500004003C0088
:109670000E0890000000E000120032005D0137008B
:109680008E089000E28F5000120032000E08900009
:10969000E30F500017003200560137008E0890008B
:1096A000ED8F50001B0032000E089000EE0F5000AE
:1096B0001F0032008E089000E68F500099003200A3
:1096C0004C01370049FE0700E10137008CFF07001D
:1096D000B3FF370060168000F1FB2F00010060002F
:1096E0006016880010C0B300446C02000000000047
:1096F000ABFF3700601680000104200001007000FD
:109700006016880010C0B300446C02000000000026
:10971000A3FF370010C0B300446C0200000000003B
:109720008040EB0010C0B30052FE07009CFF3700E2
:1097300010C0B300446C0200000000008040EB0049
:109740000040EB004BFE070095FF3700246C020041
:10975000000000000080FB00500798005E009000B1
:109760004800DD0050079800246C02000000000053
:109770008080FB005E0090000100700050079800A0
:10978000246C0200000000000080FB0040079800ED
:109790004E0090004800DD0040079800246C020055
:1097A000000000008080FB004E009000010070006F
:1097B00040079800DE00900000002100808F5000DC
:1097C00004003E00CE00900000002100808F500079
:1097D000040036000040EB00446C02000000000072
:1097E0006FFF37000000EB006007980009003700AA
:1097F000714080006E00900000844000246C0200E4
:1098000000000000004C78006E0090000000E800AE
:1098100060079800EE0090005E009000808F50007E
:10982000F3FF390040AF200010407800E44F5000B3
:1098300001003A00CAC2A9000000EB0060079800CE
:1098400008003700714080006E00900000804000EA
:1098500010407800F9FD07006E0090000000E8005D
:1098600060079800EE0090005E009000808F50002E
:10987000F4FF3900100020005892020000000000A0
:109880000000EB006007980009003700714080007D
:109890006E0090000084400000C0EB00E7FD070070
:1098A000004C78006E0090000000E800600798000F
:1098B000EE0090004E009000808F5000F3FF3900C2
:1098C00040AF200010407800E44F500001003A0003
:1098D000CAC2A80010C0B300446C0200000000001F
:1098E0000000EB006007980009003700714080001D
:1098F0006E0090000080400010407800446C020030
:10990000000000006E0090000000E8006007980072
:10991000EE0090004E009000808F5000F3FF390061
:109920001FFF370010C0B300446C020000000000AD
:1099300022C2BF00614060000004E000FCFF320072
:10994000301180008040780040AF2000014878004E
:1099500040AF2000104078000080FB0070079800A6
:109960007E009000E10F50000B003200FE009000DE
:10997000E28F5000120032007E0090000000E000F4
:10998000010032009700370010C0B300446C0200A1
:109990000000000002FF370010C0B300446C02005A
:1099A000000000000040EB00446C020000000000DA
:1099B00010C0B300446C020000000000F8FE370045
:1099C0006000B80020079800310798000000EB0005
:1099D000600798001900370022C2BF006140600094
:1099E0000004E000FCFF320030118000804078006D
:1099F00040AF2000014878002E009000BE0090008B
:109A00004809DD00C801DE00830171004801DD0066
:109A100040AF2000104078000080FB0001002000D3
:109A200000007100818071002007980031079800C4
:109A30006E0090000000E800600798006E00900043
:109A4000E30F5000E4FF36006000B800008FBE0056
:109A50000000EB00600798001600370022C2BF002C
:109A6000614060000004E000FCFF32003011800023
:109A70008040780040AF2000014878001E00BE0002
:109A80004809DD00C801DE00830171004801DD00E6
:109A900040AF2000104078000080FB000100200053
:109AA000001F7100019771006E0090000000E80037
:109AB000600798006E009000E30F5000E7FF36004B
:109AC0002E019000BE019000F0FF2F000100200049
:109AD000800F5100818F59000E003E00F0FF2F00D3
:109AE00001002000BE0F1000AE8F180009003E00DC
:109AF0002E009000BE0090003E014000AE81480064
:109B0000F0FF2F0001002000800F5100818F5900CD
:109B1000040036000040EB00446C0200000000002E
:109B20009FFE370010C0B300446C0200000000002C
:109B3000AE009000610798002500370000C2B30016
:109B40003EFD07006E0090004800DE003BFD070070
:109B50006E00900039FD07000040EB0037FD070064
:109B6000446C0200000000000080EB008080EB00ED
:109B70001E0F40005E9748001E00BE00E00F500020
:109B8000E08F580086FE320080C2B3002BFD070034
:109B90006E0090004800DE0028FD07006E00900077
:109BA00026FD07000040EB0024FD0700446C020086
:109BB000000000000080EB008080EB001E0F4000E2
:109BC0005E9748006E0090000000E8006007980073
:109BD0001E00BE00E00F5000E08F5800D7FF3A0093
:109BE0006FFE37000040EB00446C020000000000F4
:109BF0006BFE37000040EB00446C020000000000E8
:109C000067FE370040AF200090407800F0C0B300FE
:109C100080C0600040AF20000148780040AF2000C5
:109C2000104078008040E80040AF200001487800F4
:109C300010C0B300446C0200000000008040EB0044
:109C400020AF2000014878000A003700246C020091
:109C500000000000F9FC0700446C02000000000056
:109C600020AF2000104078008040E80020AF2000A6
:109C70000148780020AF20009040780040AF2000DD
:109C80001040780080CF5000F0FF390044FE3700CC
:109C900040AF200010407800BA970200000000009A
:109CA00010C0B300446C0200000000003CFE37000E
:109CB00040AF20009040780070C0B30080C06000CA
:109CC00040AF20000148780040AF2000904078006D
:109CD00060AD20000148780060AD200010407800A1
:109CE0008080FB002082200000804000104078002F
:109CF0006AFC070010C0B300446C020000000000C2
:109D000027FE370060AF2000104078000000A1005F
:109D100061AF20008048780060AF200010407800DC
:109D20000010A10061AF20008048780060AF2000E3
:109D3000104078000020A10061AF2000804878002A
:109D400080AE2000104078000040A10081AE2000CD
:109D50008048780040AF2000104078000080FB0071
:109D60004200DE00610060000004E00005003200F7
:109D700060AF2000104078000000A00061AF20001C
:109D80008048780040AF2000104078000080FB0041
:109D90000000D100610060000004E0000500320016
:109DA00060AF2000104078000010A00061AF2000DC
:109DB0008048780040AF2000104078000080FB0011
:109DC000610060000004E0000500320060AF200088
:109DD000104078000020A00061AF2000804878008B
:109DE00040AF2000104078000080FB004300DE0000
:109DF0000000A200610060000004E00005003200E5
:109E000080AE2000104078000040A00081AE20000D
:109E10008048780060AD2000104078008080FB0012
:109E20002082200000804000104078001BFC0700CA
:109E300010C0B300446C020000000000D8FD3700E1
:109E40000040EB00446C020000000000D4FD37002D
:109E50004F0478000080FA00000006000000FA00BD
:109E600000C0EB00F2940200000000000080FB0044
:109E70000080FA00000006000200FA00000F7800DF
:109E80001E007800F2940200000000000010200084
:109E90000080FA00000006000000FA0010C0B300C5
:109EA000A6940200000000000080FB000080FA0081
:109EB000000006000000FA0000B02000104078000A
:109EC000A6940200000000000080FA0000000600D6
:109ED0000000FA0000B02000104078000080FB0075
:109EE0000080FA00000006000000FA008040EB004D
:109EF00000B020000148780041022000B00020009E
:109F000060930200000000000080FA0000000600DC
:109F10000000FA0011C0B30000B020000148780032
:109F200041022000B0002000609302000000000009
:109F30000080FA00000006000000FA0080AE200059
:109F4000104078000040A00081AE200080487800DA
:109F50008040EB0020B1200001487800C922A80011
:109F6000CB22A9000080FA00000006000400FA00DD
:109F7000881F7800000F78001E00E00044003200C7
:109F8000200320009E0F100041003E001E0FE9003C
:109F900020B12000104078000080FB009E0F500090
:109FA00005003E0091022000F002200060930200B4
:109FB0000000000064013700E1002000800520005F
:109FC000D6920200000000001E0078000040E80069
:109FD000CC69020000000000A08428003467020061
:109FE000000000008040EB00C0B020000148780075
:109FF0001F0037001E017800C0B02000104078001C
:10A000008080FB004310DD008100400030B1200063
:10A0100000804000104078000080FB008691020024
:10A020000000000000C2B300446C02000000000009
:10A030001E017800C0B02000104078008080FB0036
:10A040004310DD008100400030B12000008040005E
:10A0500010407800F294020000000000C0B0200020
:10A06000104078008040E800C0B02000014878002F
:10A07000C0B0200010407800E74F5000DDFF3600F0
:10A08000D084280060670200000000002E01370025
:10A090001E00780010079800500520009E009000D8
:10A0A000808F500012013200500520009E00900069
:10A0B000808F500008003E001E0090000000E0006D
:10A0C00012003200300320009E009000808F50006C
:10A0D000DD00320018013700C00E20009E00900005
:10A0E000808F500063003200000F20009E0090001F
:10A0F000808F50005F003200C00C20009E00900056
:10A10000808F5000030132000B013700D100200086
:10A110006006200060930200000000007101200032
:10A1200030072000609302000000000020B12000F2
:10A13000104078000004E00005003A009102200081
:10A14000F00220006093020000000000440037008D
:10A150008040EB00D0B02000014878003A00370082
:10A1600000C2B300446C020000000000D0B0200028
:10A17000104078000040E800CC69020000000000B8
:10A18000E084280034670200000000008040EB00FB
:10A19000C0B020000148780016003700D0B0200081
:10A1A000104078000081FB00C0B020001040780013
:10A1B0008080FB004310DD008100400030B12000B2
:10A1C00000804000104078000080FB008691020073
:10A1D0000000000000C2B300446C02000000000058
:10A1E000C0B02000104078008040E800C0B02000DF
:10A1F00001487800C0B0200010407800E74F5000C0
:10A20000E6FF360061002000A0082000D692020080
:10A2100000000000D0B02000104078000080FB005B
:10A22000C300DD0030B12000008040001040780005
:10A23000F8000700D0B02000104078008040E8000F
:10A24000D0B020000148780020B120009040780074
:10A25000D0B020001040780080CF5000C0FF3E00FA
:10A26000310D200000092000609302000000000072
:10A27000B50037001E00780080407800A0822000E2
:10A2800001487800C00E20009E0F100005003A0023
:10A290003101200030162000609302000000000011
:10A2A00004003700D10020006017200060930200F6
:10A2B00000000000710120003007200060930200C0
:10A2C000000000008040EB00C0B020000148780092
:10A2D0000B01070080407800D0B0200001487800D2
:10A2E0008040EB0020B12000014878004D0037008D
:10A2F00000C2B300446C020000000000C0B02000A7
:10A30000104078000040E800CC6902000000000026
:10A31000E084280034670200000000000000EB0029
:10A32000505888000D0037005158800030B620008A
:10A3300000804000104078000080FB008691020001
:10A340000000000000C2B300446C020000000000E6
:10A35000505880000000E800505888005058800095
:10A36000E70F5000F0FF360061002000A008200039
:10A37000D69202000000000030B6200010407800A5
:10A38000A4000700C0B0200010407800E94F500042
:10A390001B003E000000EB00505888001000370002
:10A3A00020B12000104078008081FB0054588000CC
:10A3B0005158800030B620000080400010417800E5
:10A3C0004318DD008400400030B1200000804000D0
:10A3D00002487800505880000000E800505888007B
:10A3E00050588000E70F5000EDFF360020B12000EC
:10A3F000104078008040E80020B12000014878003B
:10A40000C0B02000104078008040E800C0B02000BC
:10A4100001487800C800070080407800D0B02000D4
:10A4200001487800D0B02000104078000004E0001F
:10A43000AFFF3A00B1022000301820006093020004
:10A440000000000040003700490007001101200013
:10A45000E01A2000D69202000000000030C3B300D2
:10A46000F2940200000000000000EB005058880049
:10A47000150037005858800000C0EB00F29402002D
:10A48000000000008040780010B020000000440070
:10A49000014878005158800010B020000080400032
:10A4A000104078000080FB00869102000000000050
:10A4B00000C2B300446C020000000000505880004D
:10A4C0000000E8005058880050588000E70F500006
:10A4D000E8FF3600D084280060670200000000001A
:10A4E00010B02000104078004A0007001600370026
:10A4F0001F00070001012000F01B200060930200F4
:10A500000000000050C5B300F294020000000000FB
:10A510000D00370016000700F1002000F01C20009D
:10A520006093020000000000C0CCB300F29402006F
:10A53000000000000400370041022000E01D200060
:10A5400060930200000000004F0478000080FA00D1
:10A55000000006000000FA0091002000200A2100FF
:10A5600060930200000000000080FA000000060076
:10A570000200FA004494020000000000004F78003E
:10A58000A100200020202000D69202000000000040
:10A590001E04E00005003A003100200080BB2000CE
:10A5A00060930200000000001800370091002000B6
:10A5B000C0202000D6920200000000001E80FB0098
:10A5C000610060000004E00004003200510120003E
:10A5D00050212000D6920200000000001E80FB00E7
:10A5E0000000D100610060000004E00004003200BF
:10A5F00041012000A0222000D692020000000000AD
:10A60000D084280060670200000000000080FA008B
:10A61000000006000400FA00004F78001E80FB00D6
:10A6200010079800200220009E009000808F5000AC
:10A630001E003200200220009E009000808F5000FB
:10A6400007003C001E009000E40F50001C00320088
:10A650009E009000F08F50000A0032002200370068
:10A66000800220009E009000808F50000A0032007F
:10A67000D00220009E009000808F50001500320014
:10A6800019003700B1012000E02320006093020090
:10A690000000000018003700A101200090252000D4
:10A6A00060930200000000001300370051012000F9
:10A6B0003027200060930200000000000E003700E9
:10A6C000810120008028200060930200000000002B
:10A6D0000900370001012000002A200060930200D9
:10A6E0000000000004003700E1002000002B2000E3
:10A6F000D6920200000000000080FA000000060070
:10A700000000FA008040EB00B0B62000014878005D
:10A710008040EB00D0B62000014878008040EB007C
:10A72000C0B6200001487800080007000080FB0048
:10A730000080FA00000006000000FA000300070095
:10A740000080FB000080FA00000006000A00FA000A
:10A7500010C0B300704798000040EB0060479800BD
:10A760000040EB005047980010C0B300104798001D
:10A770000040EB00404798008040EB00E0B620002E
:10A7800001487800D0B62000104078000004E000B6
:10A790009C003A0044940200000000000004E00025
:10A7A0000C0032008040EB00B0B620000148780079
:10A7B0008040EB00D0B62000014878008040EB00DC
:10A7C000C0B62000014878000000EB004007980068
:10A7D000A1003700A082200010407800F29402000F
:10A7E0000000000010C0B300A694020000000000AA
:10A7F0003047980010C0B300A6940200000000008B
:10A80000204798003E409000E14F500003003A007E
:10A810002E409000E14F500066003200BE40900094
:10A820002E40900080CF500003003200BE409000C8
:10A83000014F780026003700B0B620009040780025
:10A840007E409000814F50000E0031005E4090002D
:10A850008080FB0030B620000080400090407800EF
:10A860001E40900080C060000040EB00004F780068
:10A870000104E0000C00320010C0B300004F78006B
:10A8800009003700B0B62000904078000040EB008F
:10A89000004F78007E409000814F500002003A0047
:10A8A00010C0B300004F78001E04E00008003A001A
:10A8B0007E409000604798006E409000E84F500046
:10A8C00003003E00C0B62000EE4090000148780032
:10A8D00010C0B3009E4F10000D003A005E40900083
:10A8E0000081FB005E4090008080FB0030B62000BD
:10A8F00000804000904078001E40900080C07000B2
:10A9000030B6200000004100014878000F003700F9
:10A910005E4090000081FB005E4090008080FB0064
:10A9200030B6200000804000104078008040780061
:10A930001E40900000C0EA0000C060008040780027
:10A9400030B6200000004100014878001E40780029
:10A95000A6940200000000007E4090000040E80045
:10A96000704798001E40900000404000104798003B
:10A970001E4090000004E0000B003A005E40900092
:10A980008080FB0030B6200000804000104078003E
:10A99000920007005E4090000040E8005047980099
:10A9A00010C0B300104798005E409000E74F500081
:10A9B0008CFF3600FE40900000C4B30080CF5000F2
:10A9C00010003600E0B62000104078000004E000DF
:10A9D0000C003A00B0B62000EE409000014878002C
:10A9E000B0B62000104078000004E00003003A00F8
:10A9F00011C0B300D0B620000148780010C0B300E9
:10AA0000404798004E4090000004E00004003200EF
:10AA100030B62000104078000004E0000B003A003F
:10AA20008040EB00B0B62000014878008040EB0089
:10AA3000D0B62000014878008040EB00C0B620006E
:10AA4000014878000040EB00404798004E409000DD
:10AA50000080FB00400798004E0090000080FA0044
:10AA6000000006000E00FA000040EB00404798008E
:10AA70000C0037004E4090000081FB004E409000DB
:10AA80008080FB0030B620000080400090407800BD
:10AA900065004700017178004E4090000040E800DA
:10AAA000404798004E409000E74F5000F1FF3600BD
:10AAB000B0B620009040780021479800D0B6200022
:10AAC0009040780011479800C0B62000104F7800E1
:10AAD00001C4B300B0B62000014878008040EB000C
:10AAE000D0B620000148780018FF07000004E000FD
:10AAF0001A00320010C0B300304798000040EB004D
:10AB000040479800110037004E4090008080FB00C5
:10AB100065004700614178004E4090008080FB0056
:10AB200030B620000080400010407800804F510077
:10AB3000030032000040EB00304798000900370066
:10AB40004E4090000040E800404798004E40900082
:10AB5000E74F5000ECFF3600020037000040EB00EA
:10AB6000304798000040EB00404798000C00370049
:10AB70004E4090000081FB004E4090008080FB0022
:10AB800065004700E140780030B620000000410039
:10AB9000014878004E4090000040E800404798008F
:10ABA0004E409000E74F5000F1FF3600B0B6200055
:10ABB000AE40900001487800D0B620009E40900042
:10ABC00001487800C0B620001E4878003E40900042
:10ABD0000080FB000080FA00000006000200FA007E
:10ABE000004F7800E0B62000104078001E4068005A
:10ABF0008080FB00B0822000008040009040780000
:10AC0000E0B6200001487800E0B62000104078004F
:10AC10000080FB000080FA00000006000000FA003F
:10AC20000085280034670200000000000080FA0060
:10AC3000000006000400FA00C922A800CB22A900E7
:10AC4000C8C2A90080AE2000104078000040A000DB
:10AC500081AE20008048780080AE2000104078004F
:10AC60000030A10081AE200080487800EBFF070093
:10AC700000003700246C02000000000080407800D3
:10AC800010B120000148780010B120001040780079
:10AC90000080FB004400DE008040780000B120000E
:10ACA0000148780000B12000104078000080FB00CF
:10ACB000100798001E009000E10F5000790032004C
:10ACC0009E009000E48F50009B0032001E00900018
:10ACD0000000E000010032009F00370010B12000AA
:10ACE000104078000080FB00000F78009E00780084
:10ACF000E28F5000170032001E007800E20F500073
:10AD000007003C009E0078000100E0009600320041
:10AD10001E007800E10F50000C0032005D0037008B
:10AD20009E007800E48F5000130032001E0078006F
:10AD3000E40F5000570035009E00780068805000F6
:10AD4000E10F500053003E0011003700B3FF070031
:10AD5000C8FF3700449402000000000080407800E3
:10AD6000E0B020000148780010C0B300446C02003D
:10AD700000000000BFFF370000C0EB00F2940200AB
:10AD800000000000446C020000000000B9FF370022
:10AD900010C0B300446C02000000000010B120009D
:10ADA00010407800E94F500004003A00C1CEB300D3
:10ADB000A0822000014878000300370001CFB300D3
:10ADC000A0822000014878004DFE070080407800F6
:10ADD000E0B0200001487800190037008040EB0007
:10ADE000F0B02000014878000D003700F0B02000DE
:10ADF000104078008080FB0030B6200000804000CA
:10AE000010407800446C020000000000F0B0200008
:10AE1000104078008040E800F0B020000148780041
:10AE2000F0B0200010407800E74F5000EFFF3600F0
:10AE300041FE070080407800E0B020000148780023
:10AE4000E0B02000104078000004E000E3FF3A008A
:10AE50008040EB00F0B02000014878000800370087
:10AE600000C0EB00446C020000000000F0B02000C5
:10AE7000104078008040E800F0B0200001487800E1
:10AE8000F0B0200010407800E74F5000F4FF36008B
:10AE900078FF37000040EB00446C02000000000027
:10AEA00074FF370010B1200090407800F0C0B3006C
:10AEB00080C0600010B120000148780010B120006F
:10AEC000104078008040E80010B120000148780070
:10AED00010C0B300446C0200000000008040EB0092
:10AEE000F0B02000014878000C003700246C02000C
:10AEF00000000000F29402000000000010C0B30047
:10AF0000446C020000000000F0B020001040780007
:10AF10008040E800F0B0200001487800F0B0200048
:10AF20009040780010B120001040780080CF500091
:10AF3000EEFF39004FFF370010B1200010407800BD
:10AF4000BA9702000000000010C0B300446C020079
:10AF50000000000047FF37000040EB00446C020097
:10AF60000000000043FF37000080FA0000000600E8
:10AF70000200FA000040EB00004F7800F05780001C
:10AF80000000E0001200320000C2B300446C020076
:10AF9000000000003100200030412000D692020065
:10AFA0000000000000C2B300446C0200000000007A
:10AFB000E05780000000E00003003A000040EB0092
:10AFC00004810200000000000000EB00F057880040
:10AFD000E05780000000E00003003A009480020087
:10AFE00000000000004F780010002000F05788009B
:10AFF0001E80FB000080FA00000006000400FA003A
:10B00000000F7800F05780000000E00012003200CE
:10B0100000C2B300446C02000000000031002000B8
:10B0200030412000D69202000000000000C2B300B0
:10B03000446C020000000000E05780000000E000C7
:10B0400003003A000040EB00048102000000000011
:10B050000000EB00F0578800E05780000000E0009F
:10B0600007003A001E007800408002000000000047
:10B07000E2800200000000000080FB00000F78006A
:10B0800000C2B300446C0200000000001E00E0009B
:10B0900007003A003100200030412000D692020023
:10B0A0000000000000302000100798000600370064
:10B0B0004100200060412000D69202000000000004
:10B0C00000102000100798001E0090000080FA0079
:10B0D000000006000000FA00F05780000000E000C9
:10B0E0000F0032004100200060412000D692020093
:10B0F00000000000C083280060670200000000001C
:10B10000E05780000000E00003003A0010C0B300E8
:10B1100004810200000000000000EB00F0578800EE
:10B12000E05780000000E0000F003A006E7F020050
:10B13000000000000000E0000B0032009100200041
:10B14000C0202000D6920200000000005101200023
:10B1500050212000D692020000000000C083280089
:10B160006067020000000000D1002000A041200024
:10B1700060930200000000000080FA00000006005A
:10B180000000FA00F05780000000E0000F003200DD
:10B190004100200060412000D69202000000000023
:10B1A000C08328006067020000000000E0578000B4
:10B1B0000000E00003003A0010C0B3000481020068
:10B1C000000000000000EB00F0578800E05780000E
:10B1D0000000E00002003A00AE7F02000000000024
:10B1E000C1002000704220006093020000000000B7
:10B1F0000080FA00000006000000FA0001012000B3
:10B20000404F2000D6920200000000000040EB00FA
:10B21000CC6902000000000000C2B300446C0200D0
:10B220000000000060AD200010407800CC690200F2
:10B230000000000000C2B300446C020000000000E7
:10B24000D083280060670200000000000080FA0040
:10B25000000006000400FA000000EB001007980050
:10B260000000EB00E0578800A01F02000000000073
:10B27000D21B020000000000000F78001E00E0005A
:10B2800009003400400020009E0F100006003C0022
:10B290001E0078000040E9008040780060AD20008A
:10B2A00001487800020037000000EB00000F780032
:10B2B0001E00E0002D003A000000EB001064880042
:10B2C0000000EB00E0578800E05780000000E0003D
:10B2D0000F003A00B1032000804520006093020077
:10B2E000000000008001EB0042002000110020005F
:10B2F00010002000CC200200000000000040E90007
:10B300008040780060AD20000148780022003700BE
:10B31000C140800030002300808F500004003E00B8
:10B320005103200030492000D692020000000000A6
:10B33000C1022000804C2000D692020000000000D4
:10B340008001EB00320020001100200010002000DE
:10B35000CC200200000000000040E900804078009E
:10B3600060AD2000014878000B003700C14080002C
:10B3700030002300808F500004003E005103200065
:10B3800030492000D6920200000000009AFF07001A
:10B390000000EB00F057880080AE200010407800DD
:10B3A0000040A00081AE200080487800E057800077
:10B3B0000000E00009003A00C922A800C902A80064
:10B3C000CB02A900CB22A90060AD200090407800FC
:10B3D00020C0B300E07E0200000000000080FA0000
:10B3E000000006000000FA000000EB00F0578800A3
:10B3F000E0578000E10F500001003A0007E2A90089
:10B400000080FA00000006000600FA00100798000D
:10B410001E009000200798002E009000E10F5000C1
:10B420000C0032002E009000E10F500004003900A3
:10B430002E009000E20F50006500320073003700CC
:10B440005103200040502000D6920200000000006E
:10B45000720037008040EB00003020008E81020037
:10B4600000000000E10220009053200060930200E1
:10B4700000000000CBC2BF00614060000004E0009B
:10B4800004003200CBC2BF00624060000004E00054
:10B490000C003A0091002000C0202000D69202004B
:10B4A000000000005101200050212000D69202002F
:10B4B00000000000C0832800606702000000000058
:10B4C000560037000000EB00000F7800390037000D
:10B4D000E05780000000E00009003A006E7F0200A3
:10B4E000000000001E007800408002000000000004
:10B4F000E2800200000000000080FB0010079800BE
:10B500001E0090000000E00024003A001E007800B9
:10B51000869102000000000080C2B300446C02006B
:10B52000000000001E0078000080D100869102001B
:10B53000000000001E0078000000A2006100600012
:10B540000004E00004003200F083280034670200A9
:10B55000000000000B003700E05780000000E00012
:10B5600005003A00948002000000000010C0B30003
:10B5700004810200000000002084280034670200DB
:10B5800000000000D08328003467020000000000A3
:10B5900000C2B300446C020000000000E0578000CD
:10B5A0000000E00002003A00AE7F02000000000050
:10B5B0001E0FE800F00F20009E0F1000C4FF3400A3
:10B5C000C0832800606702000000000013003700FD
:10B5D000E0578000E10F500001003A0007E2A900A7
:10B5E00071002000705620006093020000000000EF
:10B5F000F1002000B018210060930200000000005C
:10B6000010C0B3000E000700040037004102200004
:10B61000E01D200060930200000000000080FA009E
:10B62000000006000000FA00B1002000600B2100BD
:10B6300060930200000000000080FA000000060095
:10B640000A00FA00004F98000040EB0020479800E5
:10B650000040EB00104798000040EB00004F7800DE
:10B66000726B020000000000C922A800C902A800F5
:10B67000CB02A900CB22A90062A0A80062C0A8004A
:10B680008660A900CBC2BF000080FB000000D10093
:10B6900061406000604798006E40900050479800FD
:10B6A000CBC2BF0061406000604798006E409000D0
:10B6B000304798000000370086C0BF006840600037
:10B6C0000004E0000F003A00866B0200000000005A
:10B6D000666B0200000000000004E000F6FF32008C
:10B6E000246C020000000000004F780062A0A90056
:10B6F00062C0A9000E4890000004E00061003A001A
:10B70000630037008660A900CBC2BF000080FB0049
:10B710000000D1006140600060479800CBC2BF00CC
:10B7200061406000404798002E4090000004E00017
:10B730002E0032003E4090000004E0002B003A0052
:10B740004E4090000004E000280032001E409000AF
:10B75000E74F50000B003E001E40780000404000C4
:10B76000004F78006E4090000004E00001003200BD
:10B770001E04A0001E4090000040E8001047980002
:10B780003B0037000E4890000004E0000400320047
:10B790001E80FB00586A020000000000060037000F
:10B7A000C0C5B300EE6B0200000000001E40780030
:10B7B000EE6B0200000000006E4090000004E0000C
:10B7C00004003200D0C2B300EE6B020000000000A3
:10B7D00003003700B0C2B300EE6B020000000000AF
:10B7E0000040EB0010479800210037003E409000D9
:10B7F0000004E0001E0032004E4090000004E00013
:10B800001B0032005E4090000004E0000B0032009C
:10B810006E4090000004E00008003A0010C0B30041
:10B82000204798000040EB0010479800B0C5B300D7
:10B83000EE6B0200000000000D0037005E4090003B
:10B840000004E0000A003A006E4090000004E000AE
:10B85000070032000040EB00204798000040EB005A
:10B8600010479800D0C5B300EE6B02000000000046
:10B870006E409000504798004E409000304798002E
:10B880008DFF3700C08328006067020000000000C1
:10B890000080FA00000006000000FA005084280032
:10B8A00034670200000000000080FA00000006007B
:10B8B0000E00FA00881F7800C922A800C902A8005B
:10B8C000CB02A900CB22A900C8C2A90080AE2000EB
:10B8D000104078000040A00081AE20008048780031
:10B8E00080AE2000104078000030A10081AE200022
:10B8F0008048780080C0EB0020C0B300E07E0200EA
:10B9000000000000E4FF070000003700246C020084
:10B910000000000080407800A0AF200001487800BF
:10B92000A0AF2000104078000080FB004400DE0043
:10B930008040780090AF20000148780090AF200050
:10B94000104078000080FB00400798004E009000F7
:10B95000E10F500032013200CE009000E18F500024
:10B9600004003C004E0190000200E000080032009C
:10B970006D013700CE019000E48F5100620132006A
:10B980004E009000E60F5000500132006601370073
:10B99000A0AF2000104078000080FB006101B900DA
:10B9A0005207980063079800F00020000100200073
:10B9B0005E019000EE019000800F5100818F5900D0
:10B9C00013013E005E009000EE0090000060010058
:10B9D000590137000E0037000F0037001400370000
:10B9E000190037000A0137001C0037002200370019
:10B9F00028003700B6003700050137000401370082
:10BA0000030137000201370001013700FA00370057
:10BA1000A1FF0700BDFF37006E7F0200000000009D
:10BA200010C0B300446C020000000000B7FF3700F4
:10BA3000AE7F02000000000010C0B300446C0200A2
:10BA400000000000B1FF37009480020000000000F9
:10BA5000446C020000000000ACFF37000040EB0027
:10BA6000048102000000000010C0B300446C02001A
:10BA700000000000A5FF370010C0B30004810200E1
:10BA80000000000010C0B300446C02000000000081
:10BA90009EFF3700666B0200000000000004E0001B
:10BAA000FCFF3200246C0200000000000080FB005C
:10BAB000100798001E0090004800DD001007980055
:10BAC000666B0200000000000004E000FCFF320092
:10BAD000246C0200000000008080FB001E0090002B
:10BAE0000100700010079800666B02000000000063
:10BAF0000004E000FCFF3200246C020000000000A3
:10BB00000080FB00000F78001E0078004800DD0078
:10BB1000000F7800666B0200000000000004E000E7
:10BB2000FCFF3200246C0200000000000080FB00DB
:10BB30001E0F70009E00900000002100808F5000BA
:10BB400003003E00000021009E0F1000040036009C
:10BB50000040EB00446C0200000000006BFF370067
:10BB60000000EB00200798000D003700666B020014
:10BB7000000000000004E000FCFF32007140800083
:10BB80002E00900000844000246C020000000000A1
:10BB9000004C78002E0090000000E800200798007C
:10BBA000AE0090001E009000808F5000EFFF390023
:10BBB0006E7F0200000000000000EB0020079800EC
:10BBC0000E003700714080002E0090000080400081
:10BBD000104078000080FB00408002000000000060
:10BBE000E280020000000000E14F5000D8FF320068
:10BBF0002E0090000000E80020079800AE009000A2
:10BC00001E009000808F5000EEFF39001E00E900FA
:10BC1000100798000000EB00200798001400370080
:10BC2000714080002E00900000844000948002004B
:10BC300000000000004C7800AE0090001E00900054
:10BC4000808F5000040031000040EB0004810200AE
:10BC5000000000000300370010C0B30004810200A0
:10BC6000000000002E0090000000E800200798006F
:10BC70002E0090009E0F5000E9FF3900AE7F0200B9
:10BC80000000000010C0B300446C0200000000007F
:10BC90000000EB0020079800090037007140800089
:10BCA0002E0090000080400010407800446C02009C
:10BCB000000000002E0090000000E800200798001F
:10BCC0002E0090009E0F5000F4FF39000FFF370048
:10BCD00010C0B300446C02000000000022C2BF008C
:10BCE000614060000004E000FCFF32003011800081
:10BCF00080407800A0AF20000148780010002000AC
:10BD0000000F7800A0AF2000104078000080FB00FA
:10BD100030079800BE009000E28F50001B003200F8
:10BD20003E019000E20F510007003C00BE01900070
:10BD30000300E0000F0032003E009000E10F5000D1
:10BD40000F00320026003700BE009000F08F500038
:10BD500015003200000220003E019000800F5100CB
:10BD600018003200BE019000E38F51000A0032003B
:10BD70001B00370022760200000000001A00370086
:10BD8000007602000000000017003700E275020094
:10BD9000000000001400370044760200000000009C
:10BDA000000F78001000370080AE200010407800AF
:10BDB0000000A1000010A10081AE200080487800A2
:10BDC0000900370080AE2000104078000000A0007D
:10BDD0000010A10081AE20008048780002003700EA
:10BDE0000000EB00100798001E007800446C020071
:10BDF00000000000C5FE37000040EB0010FE070009
:10BE000010C0B300446C020000000000BFFE370009
:10BE10000040EB00446C020000000000BBFE370055
:10BE2000A0AF200090407800F0C0B30080C0600058
:10BE3000A0AF200001487800A0AF2000104078009B
:10BE40008040E800A0AF20000148780010C0B30097
:10BE5000446C0200000000008040EB0080AF200036
:10BE60000148780012003700666B020000000000F5
:10BE70000004E000FCFF3200246C0200000000001F
:10BE80000080FB004080020000000000E280020011
:10BE900000000000446C02000000000080AF2000A1
:10BEA000104078008040E80080AF20000148780012
:10BEB00080AF200090407800A0AF200010407800B4
:10BEC00080CF5000E8FF390090FE3700A0AF20007F
:10BED0009040780030C0B30080C06000A0AF200068
:10BEE00001487800A0AF20009040780020C0B30047
:10BEF000E07E02000000000010C0B300446C0200AD
:10BF00000000000081FE3700A0AF20001040780044
:10BF1000BA9702000000000010C0B300446C020099
:10BF20000000000079FE37000040EB00446C020086
:10BF30000000000075FE37004F0478000080FA0012
:10BF4000000006000000FA00A08728003467020005
:10BF5000000000000080FA00000006000000FA0067
:10BF60000040EB0004810200000000000040EB00F4
:10BF700004810200000000000040EB000481020088
:10BF8000000000000040EB000481020000000000FF
:10BF90000000EB0040800200000000000000EB0009
:10BFA00040800200000000000000EB004080020022
:10BFB000000000000080FA00000006000C00FA00FB
:10BFC000881F780080AE2000104078000040A0005C
:10BFD00081AE20008048780080AE200010407800BC
:10BFE0000030A10081AE20008048780011C0B3006D
:10BFF00060AD20000148780081C0B30070AD200022
:10C000000148780021C0B30070D4200001487800B6
:10C0100080C0EB0020C0B300E07E02000000000002
:10C02000C922A900C902A900C8E2A80010C0B30033
:10C030007081020000000000C2FF0700000037000E
:10C04000246C02000000000080407800B0D4200082
:10C0500001487800B0D42000104078000080FB0038
:10C060004400DE0080407800A0D420000148780021
:10C07000A0D42000104078000080FB00300798001A
:10C080003E009000E30F500014013200BE0090000B
:10C09000E38F50000A003C003E019000E10F510088
:10C0A000A5003200BE019000E18F5100F8003C0075
:10C0B0003E0090000000E00012003200CE02370087
:10C0C000BE009000E68F5000770232003E019000E3
:10C0D000E60F510004003C00BE019000E48F5100C7
:10C0E00069023200C40237003E009000E80F5000A1
:10C0F00084023200BE009000EA8F50002E01320010
:10C10000BD023700B0D42000104078000080FB0052
:10C110006101B9004207980053079800D000200041
:10C12000010020004E019000DE019000800F5100C0
:10C13000818F59007C003E004E009000DE00900090
:10C1400000600100B00237000C0037000D0037001E
:10C1500012003700170037001D003700230037009A
:10C1600044003700480037004C00370052003700C9
:10C17000580037005E0037006400370071FF070089
:10C18000AFFF37006E7F02000000000010C0B30058
:10C19000446C020000000000A9FF3700AE7F0200DF
:10C1A0000000000010C0B300446C0200000000005A
:10C1B000A3FF37000040EB00708102000000000088
:10C1C00010C0B300446C0200000000009CFF370068
:10C1D00010C0B300708102000000000010C0B30066
:10C1E000446C02000000000095FF370070D420006E
:10C1F00010407800E24F500006003A0094800200A0
:10C20000000000008040780090D4200001487800B1
:10C2100006003700F00F2000CE7F02000000000073
:10C220008040780090D420000148780080AE200043
:10C2300010407800684060000004E0000800320010
:10C2400090D42000104078000080FB008E92020005
:10C25000000000008040780090D420000148780061
:10C2600090D4200010407800446C020000000000D0
:10C2700073FF3700E280020000000000446C0200FF
:10C28000000000006EFF3700828102000000000005
:10C29000446C02000000000069FF370010C0B300CA
:10C2A000268102000000000010C0B300446C0200B0
:10C2B0000000000062FF37000040EB005E810200DA
:10C2C0000000000010C0B300446C02000000000039
:10C2D0005BFF370010C0B3005E8102000000000069
:10C2E00010C0B300446C02000000000054FF37008F
:10C2F0000040EB004C8102000000000010C0B300C1
:10C30000446C0200000000004DFF370010C0B30075
:10C310004C8102000000000010C0B300446C020019
:10C320000000000046FF37000040EB00446C0200B4
:10C330000000000042FF3700B0D420009040780099
:10C34000F0C0B30080C06000B0D420000148780085
:10C35000B0D42000104078008040E800B0D4200025
:10C360000148780010C0B300446C020000000000D7
:10C370008040EB0090D42000014878003D00370059
:10C38000246C0200000000008040780080D420006F
:10C390000148780080AE20001040780068406000BE
:10C3A0000004E0000800320080D420001040780033
:10C3B0000080FB008E9202000000000080407800A8
:10C3C00080D420000148780070D42000104078000C
:10C3D000E24F500009003A0080D42000104078005D
:10C3E0000080FB00408002000000000010C0B3008D
:10C3F000446C0200000000001900370080D42000C7
:10C40000104078000080FB00CE7F0200000000009A
:10C410008040780080D420000148780080AE200061
:10C4200010407800684060000004E000080032001E
:10C4300080D42000104078000080FB008E92020023
:10C44000000000008040780080D42000014878007F
:10C4500080D4200010407800446C020000000000EE
:10C4600090D42000104078008040E80090D4200054
:10C470000148780090D4200090407800B0D420008B
:10C480001040780080CF5000BDFF3900ECFE37002F
:10C49000B0D4200090407800F0C0B30080C06000AD
:10C4A000B0D4200001487800B0D4200010407800BB
:10C4B0008040E800B0D4200001487800B0D42000CB
:10C4C00010407800268102000000000010C0B30078
:10C4D000446C020000000000D9FE3700B0D42000F8
:10C4E00090407800F0C0B30080C06000B0D420005D
:10C4F00001487800B0D42000104078008040E80067
:10C50000B0D420000148780010C0B300446C020091
:10C5100000000000246C0200000000008040780051
:10C52000A0D42000014878008040EB0090D4200087
:10C530000148780016003700A0D420001040780091
:10C540000004E00004003D0010C0B30004810200BC
:10C5500000000000030037000040EB0004810200EF
:10C5600000000000A0D420001040780000404000EF
:10C5700080407800A0D420000148780090D42000AA
:10C58000104078008040E80090D4200001487800F6
:10C5900090D4200090407800B0D420001040780063
:10C5A00080CF5000E4FF390010C0B300446C02009B
:10C5B00000000000A2FE3700B0D420001040780038
:10C5C0000080FB0020079800400A2000AE00900089
:10C5D000808F500012003200500A20002E0190007F
:10C5E000800F5100B8003200000A2000AE01900018
:10C5F000808F5100010032001F013700246C0200BF
:10C60000000000008040780060D4200001487800DD
:10C6100010C0B300446C02000000000088FE370028
:10C6200060D42000104078000080FB0010079800C4
:10C630001E009000E10F5000040032009E009000A8
:10C64000E28F5000360032009B003700246C02005D
:10C65000000000000080FB00206A8800206A800043
:10C660006300B900206A88000000EB00106A8800AF
:10C670000900370071408000106A8000008440008B
:10C68000246C020000000000004C7800106A80005A
:10C690000000E800106A8800116A8000206A8000AB
:10C6A000808F5000F3FF39000000EB00106A880013
:10C6B0001300370071408000106A80000080400045
:10C6C0000080E8001041780071408000106A80000E
:10C6D000008040000000E800904178007140800038
:10C6E000106A80000080400010407800834078008D
:10C6F00048010700106A800063004000106A88004B
:10C70000116A8000206A8000808F5000E9FF3900A4
:10C7100010C0B300446C02000000000048FE370067
:10C72000246C0200000000000080FB00206A8800EA
:10C73000206A80004200DD00206A88000000EB00D3
:10C74000106A88000900370071408000106A80007C
:10C7500000844000246C020000000000004C7800BF
:10C76000106A80000000E800106A8800116A8000EA
:10C77000206A8000808F5000F3FF39000000EB003A
:10C78000106A8800440037000040EB00048102007A
:10C79000000000000040EB000481020000000000E7
:10C7A0000040EB0004810200000000000040EB00AC
:10C7B000048102000000000071408000106A8000C7
:10C7C00000804000104078000080FB0040800200A4
:10C7D0000000000071408000106A8000008040006E
:10C7E0000000E800104078000080FB00408002005C
:10C7F0000000000071408000106A8000008040004E
:10C800000080E800104078000080FB0040800200BB
:10C810000000000071408000106A8000008040002D
:10C820006301400071408000106A80000080400079
:10C8300063004000104078006F40600000497800BD
:10C840008040EB0090D420000148780006003700BB
:10C85000C2FD070090D42000104078008040E8001E
:10C8600090D420000148780071408000106A800058
:10C8700000804000630040009040780090D4200089
:10C880001040780080CF5000F1FF3E00106A800019
:10C8900064004000106A8800116A8000206A8000ED
:10C8A000808F5000B8FF390010C0B300446C020004
:10C8B00000000000E2FD37000040EB00446C020085
:10C8C00000000000DEFD370060D42000104078003A
:10C8D0000080FB00000F78001E017800E10F51007E
:10C8E000040032009E017800E28F510040003200C7
:10C8F000D3FD3700246C0200000000000080FB0024
:10C90000206A8800246C020000000000804078004B
:10C91000A0D42000014878000000EB00106A8800D5
:10C920002E003700A0D420009040780080D4200052
:10C93000014878008040EB0090D420000148780046
:10C940001900370080D42000104078000080FB00E0
:10C95000610060000004E0000400320010C0B30079
:10C960000481020000000000030037000040EB00DB
:10C97000048102000000000080D4200010407800F4
:10C980000080FB000000D1008040780080D42000AF
:10C990000148780090D42000104078008040E800E2
:10C9A00090D420000148780090D4200010407800F6
:10C9B000E34F5000E3FF36009480020000000000C7
:10C9C0009480020000000000446C0200000000009F
:10C9D000106A80000000E800106A8800116A800078
:10C9E000206A8000808F5000CEFF390094FD370010
:10C9F000246C0200000000000080FB00206A880018
:10CA00000000EB00106A88001600370022C0B30057
:10CA100060B92000A10B2000B8000700EB00070060
:10CA200022C0B30060BB2D00A10B2000B3000700A3
:10CA300022C0B300603D2D00A10B2000AF00070015
:10CA4000E200070022C0B30060BB2000A10B200061
:10CA5000AA000700DD000700106A80000000E8005F
:10CA6000106A8800116A8000206A8000808F500060
:10CA7000E6FF390072FD37000040EB00446C020015
:10CA8000000000006EFD3700B0D420001040780098
:10CA9000BA9702000000000010C0B300446C02000E
:10CAA0000000000066FD3700B0D420009040780000
:10CAB00030C0B30080C06000B0D4200001487800CE
:10CAC000B0D420009040780060AD2000014878008C
:10CAD00060AD20009040780070D4200010407800B5
:10CAE000E07E02000000000010C0B3007081020070
:10CAF0000000000010C0B300446C02000000000001
:10CB00004FFD370080AE2000104078000040A100AB
:10CB100081AE200080487800B0D42000104078001A
:10CB20000080FB004300DE000000A2006100600006
:10CB30000004E0000500320080AE200010407800C4
:10CB40000040A00081AE20008048780021C0B300E2
:10CB500070D4200001487800B0D420001040780044
:10CB60000080FB004200DE00610060000004E00085
:10CB70000300320031C0B30070D4200001487800B7
:10CB800080AE2000104078000030A10081AE20006F
:10CB900080487800B0D42000104078000080FB006E
:10CBA0000000D100610060000004E00005003200D8
:10CBB00080AE2000104078000030A00081AE200040
:10CBC0008048780060AD20009040780070D420004C
:10CBD00010407800E07E02000000000010C0B300AA
:10CBE000708102000000000010C0B300446C02001D
:10CBF0000000000012FD37000040EB00446C020012
:10CC0000000000000EFD37004F0478000080FA009D
:10CC1000000006000600FA002047980031479800FF
:10CC2000424798002E4090000080FB004600DE0046
:10CC3000004F78000040EB001047980022003700BA
:10CC40001E409000E34F50000C003A001E04E0002C
:10CC50000A00320010C0B3005E8102000000000034
:10CC60001E80FB002C920200000000000040EB0040
:10CC70005E81020000000000100037002E4090008E
:10CC80000080FB00610060000004E000040032004E
:10CC900010C0B30004810200000000000300370050
:10CCA0000040EB0004810200000000002E409000D4
:10CCB0000080FB000000D100204798001E4090003B
:10CCC0000040E800104798001E409000E34F5000DD
:10CCD000DBFF36003E4090000080FB0040800200F9
:10CCE000000000004E4090000080FB0040800200E9
:10CCF000000000000080FA00000006000800FA00B2
:10CD00001007980021079800624798000040EB0048
:10CD100004810200000000000040EB0004810200DA
:10CD2000000000000040EB00048102000000000051
:10CD30000040EB0004810200000000001E00900093
:10CD40008E920200000000004080020000000000FF
:10CD50001E009000AE0090004809DD004800DE0093
:10CD600000007100C808DE008E9202000000000082
:10CD700040800200000000001E009000AE00900005
:10CD80004008DE00010020008E920200000000003A
:10CD900040800200000000006E4090006F40600084
:10CDA000604798000040EB00004F78000200370019
:10CDB0006AFC07001E4FE8006E4090009E4F100076
:10CDC000FBFF39000080FA00000006000000FA00B6
:10CDD00010C0B30004810200000000000040EB001E
:10CDE00004810200000000000040EB00048102000A
:10CDF000000000000040EB00048102000000000081
:10CE00000000EB004080020000000000948002005F
:10CE100000000000446C020000000000948002004A
:10CE200000000000446C0200000000004BFC070002
:10CE30004AFC07000080FA00000006000200FA0029
:10CE4000000F78001E00E0000300320010C3B300A2
:10CE50008D0207000200370000C3B3008A020700FA
:10CE60000080FA00000006000600FA001007980093
:10CE7000020037001E407800830207001E00900069
:10CE8000104F78001E407800404798004E409000B8
:10CE90000004E0000200320010C0B30040479800D8
:10CEA0004E4090009E0090008100E800110798001D
:10CEB0000004E000EFFF3A000080FA0000000600E6
:10CEC0000600FA0010079800020037001E407800A4
:10CED0006D0207001E009000104F78001E40780081
:10CEE000404798004E4090000004E00002003200ED
:10CEF00010C0B300404798004E4090009E00900044
:10CF00008100E800110798000004E000EFFF3A00FC
:10CF1000D0C0B3005C020700A0C0B3005A020700F3
:10CF20000080FA00000006000400FA002047980084
:10CF300000C8B300004F780060802800CAFF0700D7
:10CF40000040EB00104798000F0037002E40900083
:10CF50001E4060000004E0000300320010C3B30074
:10CF6000490207000200370000C3B3004602070071
:10CF70001E80FB000000D100004F78001E40900092
:10CF80000040E800104798001E409000E74F500016
:10CF9000EEFF36000080FA00000006000E00FA00E6
:10CFA00050079800610798000040EB00004F7800A0
:10CFB00000102E00515F20003007980041079800B4
:10CFC0000040EB0010479800320037003E0190000F
:10CFD000CE0190005E009000EE009000240602005A
:10CFE0000000000010079800210798001E04E000D0
:10CFF00005003A001E009000AE009000E00F5000C7
:10D00000E08F5800180032001E0090000043B0006E
:10D010001D0207009E0090003E009000000AB8002C
:10D020009E0090004E0090000088B9000501780035
:10D0300000014100BE0090002E0090000088B90061
:10D0400000014100820278005E009000EE00900036
:10D050000400500085805800500798006107980030
:10D0600010C0B300004F78003E009000CE0090004A
:10D07000A20020000300200024060200000000009F
:10D0800030079800410798001E4090000040E800DB
:10D09000104798001E409000E74F5000CBFF36002D
:10D0A0005E0090000043B000F70107000080FA0026
:10D0B000000006000C00FA00400798005107980095
:10D0C0000000EB00100798000000EB00000F780054
:10D0D0006000B80020079800310798004E019000CA
:10D0E000DE019000F0232400F1002000800F5100A9
:10D0F000818F5900210036004E009000DE00900024
:10D1000002242400F3002000240602000000000096
:10D1100020079800310798002E0090006F0007004C
:10D12000C0C2B300D80107004E009000DE0090009E
:10D1300002242400F3002000440602000000000046
:10D1400040079800510798004E019000DE019000C2
:10D15000703E200001002000800F5100818F590097
:10D1600002003E00908028003FFF070010002000D2
:10D170001007980010002000000F78004E0190006A
:10D18000DE019000703E200001002000800F510061
:10D19000818F5900320036004E009000DE00900072
:10D1A000823E200003002000240602000000000050
:10D1B00020079800310798002E019000BE019000D2
:10D1C0004006200001002000800F5100818F59008F
:10D1D000030036002E0090004000070014003700C6
:10D1E0001E0090000000E0000F0032002E019000B1
:10D1F000BE019000A000200001002000800F51001F
:10D20000818F59000300360000C3B3009E01070060
:10D2100002003700E080280013FF07002E00900076
:10D220002E000700020037002E0090002B000700A0
:10D23000C0C2B300940107004E009000DE009000D1
:10D24000823E20000300200044060200000000008F
:10D25000400798005107980010002000000F780048
:10D260004E019000DE0190004006200001002000E9
:10D27000800F5100818F5900030036004E0090004E
:10D2800016000700130037001E00E0000F003200F8
:10D290004E019000DE019000A0002000010020005F
:10D2A000800F5100818F59000300360000C3B30086
:10D2B0007501070002003700E0802800EAFE070041
:10D2C0004E00900005000700020037004E0090005D
:10D2D000020007000080FA00000006000800FA00C3
:10D2E000300798000040EB00004F780000712200EA
:10D2F000200798000040EB00104798001E00370000
:10D300003E0090002E019000110009000280D8001C
:10D31000100798001E04E00003003A001E00900071
:10D320000000E0000C0032001E0090000043B0003E
:10D33000550107009E0090002E0090000088B90063
:10D34000800078003E0090000100500030079800F7
:10D3500010C0B300004F78002E009000A200200003
:10D36000110009000280D800200798001E4090009C
:10D370000040E800104798001E409000E34F500026
:10D38000DFFF36003E0090000043B0003E01070082
:10D390000080FA00000006000600FA0040479800EE
:10D3A0000040EB00004F780040C6B30030479800C3
:10D3B0000040EB0020479800200037004E409000CE
:10D3C0008080FB003E4090000081FB0011000900BE
:10D3D0008280D800104798001E04E00003003A0045
:10D3E0001E4090000004E0000B0032001E40900040
:10D3F0000043B000240107004E4190009E40900081
:10D400003E4090000088B90000405100404798001D
:10D4100010C0B300004F78003E4090000080FB0039
:10D42000A2002000110009000280D80030479800B7
:10D430002E4090000040E800204798002E409000C9
:10D44000E14F5000DDFF36004E4090000043B00039
:10D450000D0107000080FA00000006000400FA0039
:10D4600010079800108228007FFE07001E00900021
:10D470004400DE006F0F60009E00780010812800DD
:10D480000080400010407800FF0007001E00900060
:10D490006F0F60009E00780010812800008040001F
:10D4A00010407800F80007000080FA000000060035
:10D4B0000400FA001007980000C3B300C70007007B
:10D4C00080C7B300C50007001E0090004400DE00C6
:10D4D0006F0F60009E0078001081280000804000DF
:10D4E00010407800BD0007001E0090006F0F600024
:10D4F0009E007800108128000080400010407800D5
:10D50000B60007000080FA00000006000400FA00E0
:10D51000100798001082280053FE07001E0090009C
:10D520004C00DE006F0F60009E0078001081280024
:10D530000080400010407800D30007001E009000DB
:10D540004800DE006F0F60009E0078001081280008
:10D550000080400010407800CB0007001E009000C3
:10D560004400DE006F0F60009E00780010812800EC
:10D570000080400010407800C30007001E009000AB
:10D580006F0F60009E00780010812800008040002E
:10D5900010407800BC0007000080FA000000060080
:10D5A0000600FA00200798002E0090007D00B900C8
:10D5B000D2022000110009000280D800000F78007C
:10D5C0001E00780042062000110009000280D800E9
:10D5D00071FF0700E0C2B300AB0007001E00780037
:10D5E00042062000110009000280D8008000FD00E2
:10D5F000204798002E409000E94F500002003E0066
:10D6000000C3B300A00007001E00780042062000FF
:10D61000110009000280D8008000FD005EFF0700B5
:10D620000080FA00000006000800FA0020079800B9
:10D630003107980090018000100798002E0090009C
:10D64000900188003E0090001080BA00C800DD0004
:10D650003E0090001000BA00008F70001E00900085
:10D66000900188001E0078000080FA00000006008B
:10D670000000FA000081200010407800E94F5000BF
:10D680000800320000812000104078000080FB007C
:10D6900080004000C0A920000080400010007800F9
:10D6A000401188000000EB00001188002062A800F3
:10D6B0000000EB001011880021E2A8002342A8001E
:10D6C0008560A9000080FA00000006000000FA0052
:10D6D00022C2BF00614060000080FB000080FA00B1
:10D6E000000006000000FA000000EB00406988001E
:10D6F0001000200030698800D040800000A0A10008
:10D70000D04088000080FA00000006000200FA0005
:10D7100023C2BF00624060000004E00012003A0033
:10D7200040698000000FE800000021009E0F1000FB
:10D7300002003A000000EB00000F78003069800022
:10D740009E0F1000080032001E007800406988001B
:10D7500071408000406980000080400010407800E7
:10D760000080FB00201188000080FA000000060005
:10D770000200FA000000370040698000000FE80056
:10D78000000021009E0F100002003A000000EB0094
:10D79000000F7800306980009E0F10000D003200ED
:10D7A00023C2BF00624060000004E000F2FF3A00C4
:10D7B0001E00780040698800714080004069800048
:10D7C00000804000104078000080FB00201188009D
:10D7D000E9FF37000080FA00000006000200FA00AE
:10D7E000004F78003169800040698000808F5000D0
:10D7F00005003A00C222A900D040800000A0A0008D
:10D80000D04088000E0037007140800030698000F1
:10D81000808040001E407800804878003069800099
:10D820000000E800306988003169800000002100B4
:10D83000808F500002003A000000EB003069880041
:10D840000080FA00000006000000FA0022C2BF00BB
:10D85000614060000004E000FCFF320030118000F5
:10D860000080FB000080FA00000006000000FA00C3
:10D8700023C2BF00614060000004E000FCFF3200F2
:10D880000080FA00000006000200FA00004F780055
:10D89000D040800001102000010060000000E00086
:10D8A00006003A0023C2BF00624060000004E000AE
:10D8B000FCFF3A001E00FB00201188000080FA00E7
:10D8C000000006000200FA00004F78001E80FB00F6
:10D8D000401188000080FA00000006000000FA00F5
:10D8E00022C2BF000080FB000000D1006140600048
:10D8F0000080FB000080FA00000006000000FA0033
:10D9000010118000D1FF2F0001006000101188006D
:10D910000080FA00000006000000FA0095C0BF0079
:10D92000704060000004E00010003A0051408000A8
:10D9300040408000808F50000C00320023C2BF00A6
:10D94000624060000004E000FCFF3A008580A9000E
:10D950009580A80031408000404080000080400059
:10D96000104078000080FB00201188000080FA0041
:10D9700000000600809FBE000000FA000140800009
:10D980002040800080804000301180008048780076
:10D99000204080000000E8002040880021408000F6
:10D9A00010408000808F500001003A009560A9006F
:10D9B0008560A9000080FA004F00BE00004006000C
:10D9C000809FBE000000FA00404080000000E80098
:10D9D000404088004140800050408000808F5000CF
:10D9E00002003A009580A90006003700314080000F
:10D9F0004040800000804000104078000080FB0024
:10DA0000201188008580A9000080FA004F00BE0028
:10DA1000004006000000FA0040872800346702003A
:10DA2000000000000080FA00000006000600FA0076
:10DA3000C222A80029010700F6FF070000003700F6
:10DA40001C01070080407800E0D3200001487800E6
:10DA5000E0D32000104078000004E0000F01350002
:10DA6000E0D32000104078000004E00002003A00FB
:10DA7000E8FF0700F2FF3700E0D3200010407800F5
:10DA8000E14F500006003A00140107008C4A0200E2
:10DA90000000000011010700DEFF0700E8FF37006B
:10DAA000E0D3200010407800E24F500006003A001A
:10DAB0000A010700585C020000000000070107008F
:10DAC000D4FF0700DEFF3700E0D3200010407800CD
:10DAD000E34F500006003A0000010700723E0200CA
:10DAE00000000000FD000700CAFF0700D4FF370058
:10DAF000E0D3200010407800E44F500006003A00C8
:10DB0000F60007001A56020000000000F3000700AC
:10DB1000C0FF0700CAFF3700E0D3200010407800A4
:10DB2000E54F500006003A00EC000700DE5F0200FF
:10DB300000000000E9000700B6FF0700C0FF370043
:10DB4000E0D3200010407800E64F500006003A0075
:10DB5000E20007006A82020000000000DF00070008
:10DB6000ACFF0700B6FF3700E0D32000104078007C
:10DB7000E74F500004003A00D8000700D700070024
:10DB8000A4FF0700AEFF3700E0D32000104078006C
:10DB9000EF4F500008003A0010C0B300446C020080
:10DBA00000000000C222A900366C02000000000044
:10DBB0000000FE00A2FF3700E0D3200010407800F4
:10DBC000F04F500003003A000040EB000002070055
:10DBD0009BFF3700E0D3200010407800F14F500049
:10DBE00003003A0010C0B300F901070094FF3700AA
:10DBF000E0D3200010407800F24F500039003A0086
:10DC00000000EB00800888000000EB00F0088800AE
:10DC10000000EB00E00C8800A16C2000914078002F
:10DC200000CEB30000C060006041B300CAE6B70098
:10DC3000A00007000080FB00200798002E00900045
:10DC40000000D100610060000004E000010032002B
:10DC500010A1A8002E009000610060000004E00008
:10DC6000010032001081A800920007000080FB0034
:10DC70004800DD00200798008E0007008080FB0030
:10DC80002E00900001007000200798002E009000E8
:10DC9000D00C88002E019000C20C8800600020008B
:10DCA000E00C8800830007000080FB004800DD00D6
:10DCB000200798007F0007008080FB002E00900066
:10DCC00001007000200798002E0090006008880076
:10DCD00011E1A80010C0B300446C02000000000075
:10DCE00057FF3700E0D3200010407800F34F50007A
:10DCF0000D003A000000EB00800888000000EB00F7
:10DD0000E00C8800A16C20009140780000CEB300A8
:10DD100000C06000CAE6B70010C0B300446C020047
:10DD20000000000046FF3700E0D3200010407800DC
:10DD3000F44F50000E003A0021E3A800C0C0B30029
:10DD4000FC900200000000002007980021E3A900D9
:10DD50002E0090004800DE00446C0200000000002D
:10DD60002E009000446C02000000000034FF3700D9
:10DD7000E0D3200010407800F54F500018003A0022
:10DD800021E3A800C0C0B300FC9002000000000026
:10DD900020079800366C0200000000002E00900062
:10DDA0004800DE00446C0200000000002E009000DD
:10DDB000446C020000000000666B020000000000DE
:10DDC000E14F5000EFFF3A00246C02000000000019
:10DDD0000080FB002007980021E3A90018FF37000E
:10DDE000E0D3200010407800F64F500018003A00B1
:10DDF0002275020000000000008FBE001E00BE0061
:10DE00004808DE0001002000446C02000000000011
:10DE10001E00BE004008DE0001002000446C02002D
:10DE2000000000001E00BE004809DD004800DE00C2
:10DE300000007100C808DE00446C02000000000011
:10DE40001E007800446C020000000000FCFE370059
:10DE5000E0D32000104078000080FB004500DE0089
:10DE60000080FB000000D100610060000004E000C1
:10DE700006003200E0D32000104078001E000700AA
:10DE8000446C020000000000EDFE37000040EB0093
:10DE9000446C020000000000E9FE3700E0D32000DF
:10DEA00010407800A4000700446C0200000000004D
:10DEB000E3FE37000000FA00666B0200000000007D
:10DEC0000004E000FCFF3200246C020000000000AF
:10DED0000080FB000080FA00000006000000FA004D
:10DEE00000C0EB00040007000040EB0092000700B8
:10DEF0000080FA00000006000400FA0020479800A5
:10DF00000040EB00004F78002E4090000080FB00A6
:10DF10004400DE00610060000004E0000200320006
:10DF200010C0B300004F78009E40780061C06000D0
:10DF3000614060004201DD00912C2000914078009A
:10DF4000B0CFB30000C0600002407000C9E2B7006B
:10DF50000040EB00004F78002E4090000080FB0056
:10DF60004300DE00610060000004E00002003200B7
:10DF700010C0B300004F78009E40780061C0600080
:10DF80006140600000414000912C200091407800E9
:10DF9000D0CFB30000C0600002407000C9E2B700FB
:10DFA0000040EB00004F78002E4090000080FB0006
:10DFB0004200DE00610060000004E0000200320068
:10DFC00010C0B300004F78009E40780061C0600030
:10DFD00061416000912C200091407800E0CFB300B7
:10DFE00000C0600002407000C9E2B7000040EB00D2
:10DFF000004F78002E4090000080FB000000D10010
:10E00000610060000004E0000200320010C0B300B4
:10E01000004F78009E40780061C06000C700DD00BE
:10E02000C8C2BF000074A10001407000C8E2B70080
:10E030000040EB00004F78002E4090000080FB0075
:10E04000610060000004E0000200320010C0B30074
:10E05000004F78009E40780061C060006140600021
:10E060004601DD00812C200091407800F0CBB30008
:10E0700000C0600002407000C8E2B70050002000FD
:10E080005892020000000000AE40900000CEB300A5
:10E0900000C0600020479800CBC2BF006440600011
:10E0A0000004E000030032002E4090000044A00075
:10E0B00020479800CBC2BF00624060000004E0002F
:10E0C000030032002E4090000034A000204798004A
:10E0D000CBC2BF00614060000004E00003003200DA
:10E0E0002E4090000024A00020479800CAC2BF0024
:10E0F00001C8B300014060000004E00003003200EA
:10E100002E4090000014A00020479800CAC2BF0013
:10E110000044B2000004E000030032002E409000F2
:10E120000004A000204798002E4090000080FB00D3
:10E130000080FA00000006000400FA002047980062
:10E140002E4090000080FB004600DE006100600071
:10E150000004E00003003200C002A900C202A800CF
:10E1600002003700C002A900C202A9002E409000A0
:10E170000080FB004500DE00610060000004E0005C
:10E1800003003200C962A800CB62A9000200370078
:10E19000CB62A900C962A9000040EB00004F7800E3
:10E1A0002E4090000080FB004400DE006100600013
:10E1B0000004E0000200320010C0B300004F7800FD
:10E1C0009E40780061C06000614060004201DD0057
:10E1D000B12C200091407800B0CFB30000C06000A7
:10E1E00002407000CBE2B7000040EB00004F780027
:10E1F0002E4090000080FB004300DE0061006000C4
:10E200000004E0000200320010C0B300004F7800AC
:10E210009E40780061C060006140600000414000A5
:10E22000B12C200091407800D0CFB30000C0600036
:10E2300002407000CBE2B7000040EB00004F7800D6
:10E240002E4090000080FB004200DE006100600074
:10E250000004E0000200320010C0B300004F78005C
:10E260009E40780061C0600061416000B12C2000D8
:10E2700091407800E0CFB30000C060000240700021
:10E28000CBE2B7000040EB00004F78002E4090003A
:10E290000080FB000000D100610060000004E0008D
:10E2A0000200320010C0B300004F78009E4078009A
:10E2B00061C06000C700DD00CAC2BF000074A100D9
:10E2C00001407000CAE2B7000040EB00004F780048
:10E2D0002E4090000080FB00610060000004E00020
:10E2E0000200320010C0B300004F78009E4078005A
:10E2F00061C06000614060004601DD00A12C20008B
:10E3000091407800F0CBB30000C060000240700084
:10E31000CAE2B7005000200058920200000000003E
:10E32000AE40900000CEB30000C0600020479800CF
:10E33000CBC2BF00644060000004E0000300320074
:10E340002E4090000044A00020479800CBC2BF00A0
:10E35000624060000004E000030032002E409000A4
:10E360000034A00020479800CBC2BF00614060008D
:10E370000004E000030032002E4090000024A000C2
:10E3800020479800CAC2BF0001C8B3000140600026
:10E390000004E000030032002E4090000014A000B2
:10E3A00020479800CAC2BF000044B2000004E00049
:10E3B000030032002E4090000004A0002047980087
:10E3C0002E4090000080FB000080FA000000060054
:10E3D0000400FA0020479800AE4090000040EB0097
:10E3E000628B020000000000104798001E40900061
:10E3F0000004E00001003200C222A8001E4090008C
:10E40000446C02000000000000003700666B020050
:10E41000000000000004E0000F003200246C020045
:10E4200000000000004F780000C0EB009E4F10007D
:10E43000050032001E4090001E404000446C020067
:10E44000000000000400370010C0B300446C02005C
:10E45000000000001A0037001E4090000004E00099
:10E46000EAFF3A00006A80000000E00010003A0075
:10E470000080EB00006A8800C2C2BF000080FB0081
:10E480000000D100614060000004A2006140600013
:10E490006140600000414000212C20009140780044
:10E4A000D0CFB30000C0600002407000C2E2B700ED
:10E4B000006A80000000E900006A8800D3FF37008E
:10E4C0000080FA00000006000600FA000000EB00E1
:10E4D000800888000000EB00F00888000000EB00D6
:10E4E000E00C8800D05B80000000E00008003A00EB
:10E4F000A16C20009140780000CEB30000C0600005
:10E50000CAE6B7000000EB00805B88003D003700E2
:10E51000D05B8000E30F500005003C00E0032000CA
:10E52000000F780010A1A8001081A8001500370086
:10E53000D05B8000FE0F500005003C00A00F2000C3
:10E54000000F780010A1A8001081A9000D0037006D
:10E55000D15B8000400F2000808F500005003C0000
:10E56000007D2000000F780010A1A9001081A800F4
:10E570000400370000E82300000F780010A1A90074
:10E580001081A900D05B8000000178001E00780097
:10E59000110009000280D8000000E900200798005F
:10E5A0002E00900060088800E05B8000800078000A
:10E5B0002E0090000088B9004206200011000900DA
:10E5C0000280D80010079800A16C200091407800CC
:10E5D00000CEB30000C060006041B300CAE6B700DF
:10E5E0001E009000D00C88001E009000C00C880017
:10E5F00060002000E00C880011E1A800200020004D
:10E60000805B88000080FA00000006001200FA001B
:10E610000000EB00800888000000EB00F008880094
:10E620000000EB00E00C8800805B8000E20F5000EF
:10E6300014003A00A16C20009140780000CEB30095
:10E6400000C06000CAE6B700C1002000E02B200037
:10E6500060930200000000000000EB00805B880077
:10E66000006480008000E800F00F200080806000DF
:10E67000E0B7200000804000104078000004E00077
:10E68000AC0032000000EB0020079800006480001E
:10E690008000E800F00F2000008060000064880027
:10E6A000A01F020000000000D21B020000000000BA
:10E6B00040079800A01F020000000000D21B0200CB
:10E6C00000000000CF80DE00E80302000000000030
:10E6D000008FBE004E0090000000E00007003200F6
:10E6E000CE009000F0F92000808F500003003E0023
:10E6F0002E0090000000E800200798006011B8008C
:10E700001E00BE003E040200000000000000E00009
:10E7100001003C000B00370002002000832C240085
:10E720001E00BE0042040200000000000000E000E5
:10E7300001003500030037002E0090000000E800C3
:10E74000200798002E009000E20F500011003200C8
:10E750000000EB001064880011012000A02C2000B4
:10E76000609302000000000011012000B02D200085
:10E77000D6920200000000008001EB0002FA2000A7
:10E780001100200020032000CC2002000000000027
:10E79000400798004E009000E30F500005003E0037
:10E7A000E00320003007980010A1A8001081A80005
:10E7B000150037004E009000FE0F500005003E008F
:10E7C000A00F20003007980010A1A8001081A90018
:10E7D0000D003700CE009000400F2000808F5000C9
:10E7E00005003E00007D20003007980010A1A90020
:10E7F0001081A8000400370000E8230030079800CB
:10E8000010A1A9001081A9003E0090004E019000C7
:10E81000110009000280D8000000E900600798009C
:10E820002E009000E20F50000E0032000101200087
:10E83000902F2000D6920200000000008001EB0023
:10E84000320620008000EB0020032000CC200200D4
:10E8500000000000CF80DE00E8030200000000009E
:10E86000008FBE0002002000832C24001E00BE008A
:10E870004604020000000000008FBE006E00900001
:10E88000CF80DE00E803020000000000700798005F
:10E89000010F98006E0090000000E00008003D00AD
:10E8A00002002000037824007E0090008E08900073
:10E8B000CC0402000000000070079800010F9800CF
:10E8C0001E01BE007E0090008E08900086050200AA
:10E8D00000000000EE050200000000005007980054
:10E8E000A16C20009140780000CEB30000C0600011
:10E8F0006041B300CAE6B7005E009000D00C88000B
:10E900005E009000C00C880060002000E00C8800D1
:10E910006E0090006008880011E1A800A1002000AE
:10E9200090302000609302000000000020002000D2
:10E93000805B88000080FA00000006000400FA00F6
:10E94000805B8000E20F500005003A00F1012000DA
:10E9500030312000609302000000000037003700D3
:10E96000F100200020332000D692020000000000B9
:10E970000000EB00F00888000000EB008008880031
:10E98000C942A800616820009140780000CEB30021
:10E9900000C06000A040B30086E6B700A0032000DE
:10E9A0008008880051000700008FBE00F00F200093
:10E9B00001002000BE0F1000AE8F180007003600C7
:10E9C0001E00BE00C808DD000080FD008040780009
:10E9D0000040EB00008FBE0008003700B1002000AF
:10E9E000A0132100D692020000000000A000200029
:10E9F000800888003D000700008FBE001E00BE009A
:10EA00005A68020000000000808628003467020077
:10EA100000000000C08628006067020000000000BF
:10EA200086C6BF00F041B30086E6B7000000EB00E9
:10EA3000F00888000000EB00800888000080FA00E1
:10EA4000000006000400FA000000EB00F008880057
:10EA50000000EB0080088800C942A800616820001F
:10EA60009140780000CEB30000C06000A040B30029
:10EA700086E6B700A0032000800888001B0007007E
:10EA8000008FBE00F00F200001002000BE0F10001C
:10EA9000AE8F1800070036001E00BE00C808DD005B
:10EAA0000080FD00804078000040EB00008FBE0039
:10EAB00004003700A0002000800888000B00070039
:10EAC000008FBE0086C6BF00F041B30086E6B700E7
:10EAD0000000EB00F00888000000EB0080088800D0
:10EAE0001E00BE000080FA00000006000000FA00D0
:10EAF0000080EB00700888000080EB006008880050
:10EB00000000EB00400888000000EB00300888009F
:10EB10000000EB00B00888000000EB00A0088800AF
:10EB200080002000F0088800400F2000E0088800E6
:10EB300000402200D00888008780A9001FE1A800BB
:10EB400011E1A80087C0BF00704060000004E00031
:10EB5000FCFF320011E1A9001FE1A900300880008C
:10EB6000C05B880040088000B05B8800B05B80001C
:10EB700001002000905B8800A15B8800905B800012
:10EB8000A15B8000C000DD0000002000905B8800D9
:10EB9000A15B8800C05B80006101B800905B8000D1
:10EBA000A15B80000200400083804800905B8800E9
:10EBB000A15B8800905B8000A15B80000080FA0070
:10EBC000000006000000FA0080AE2000104078002F
:10EBD000634060000004E00002003A00C942A8005F
:10EBE00001003700C8C2A800E10020001034200056
:10EBF000D6920200000000000080FA00000006002B
:10EC00000000FA0080AE20001040780063406000F1
:10EC10000004E00003003A00C942A900CB42A8006A
:10EC200002003700C8C2A900CAC2A80081002000A3
:10EC3000F034200060930200000000000080FA0021
:10EC4000000006000000FA0080AE200010407800AE
:10EC5000634060000004E00003003A00C942A900DC
:10EC6000CB42A90002003700C8C2A900CAC2A9004D
:10EC70007100200070352000609302000000000049
:10EC80000080FA00000006000200FA0080AE2000BA
:10EC900010407800634060000004E00009003A0082
:10ECA000C942A8000000000000000000CBC2BF0065
:10ECB0000080FB004200DE0061406000004F7800F1
:10ECC00008003700C8C2A8000000000000000000D3
:10ECD000CAC2BF000080FB004600DE006140600049
:10ECE000004F78001E80FB000080FA000000060044
:10ECF0000E00FA000040EB00404798000000EB00D7
:10ED0000800888000000EB00F00888000000EB009D
:10ED1000E00C8800805B8000E20F500015003A0094
:10ED2000006480008000E800F00F20008080600018
:10ED3000E0B7200000804000104078000004E000B0
:10ED40000C003A00A16C20009140780000CEB30086
:10ED500000C06000CAE6B700C1002000E02B200020
:10ED600060930200000000000000EB00805B880060
:10ED70007D003700006480008000E800F00F200074
:10ED80000080600000648800A01F020000000000F6
:10ED9000D21B020000000000CF80DE00E80302006A
:10EDA00000000000008FBE00106480000000E00042
:10EDB00008003A0002002000433324001E00BE0079
:10EDC0003E040200000000000000E00001003C00E2
:10EDD000120037000000EB001064880031012000B1
:10EDE000301E210060930200000000008001EB0053
:10EDF000420B20008000EB00A0052000CC20020088
:10EE000000000000CF80DE00E803020000000000E8
:10EE1000008FBE0010C0B3004047980010A1A800AA
:10EE20001081A800204E20004007980002002C000E
:10EE3000A35524001E00BE0046040200000000008E
:10EE4000008FBE004E009000CF80DE00E80302007D
:10EE50000000000050079800610798004E009000E5
:10EE60000000E00008003D000200200003782400BC
:10EE70005E009000EE009000CC0402000000000054
:10EE800050079800610798001E01BE005E009000C8
:10EE9000EE00900086050200000000000200200045
:10EEA00083272400CC04020000000000EE050200CD
:10EEB0000000000030079800A16C2000914078000D
:10EEC00000CEB30000C060006041B300CAE6B700E6
:10EED0003E009000D00C88003E009000C00C8800DE
:10EEE00060002000E00C88004E0090006008880060
:10EEF00011E1A800C1002000601F21006093020002
:10EF00000000000020002000805B88004E40900040
:10EF1000E14F500014003A0013002000420B200083
:10EF20008000EB000080EB00CC200200000000001D
:10EF3000CF80DE00E803020000000000008FBE006A
:10EF40006011B8001E00BE00420402000000000074
:10EF50000000E00001003500B0FF3700C086280047
:10EF600060670200000000000080FA000000060058
:10EF70000000FA0094800200000000000080FA0007
:10EF8000000006000200FA00000F78001E00780062
:10EF90004080020000000000001020000080FA0005
:10EFA000000006000000FA006E7F02000000000072
:10EFB0008100200000932000D69202000000000093
:10EFC000D1002000A041200060930200000000005A
:10EFD0000080FA00000006000000FA00AE7F020088
:10EFE000000000006100200080932000D692020003
:10EFF00000000000C1002000704220006093020069
:10F00000000000000080FA00000006000000FA0086
:10F01000E2800200000000000080FB000080FA0097
:10F02000000006000000FA008281020000000000DB
:10F030000080FB000080FA00000006000000FA00DB
:10F040000040EB005E810200000000000080FA003A
:10F05000000006000000FA0010C0B3005E8102004C
:10F06000000000000080FA00000006000000FA0026
:10F0700010C0B30026810200000000000080FA00EA
:10F08000000006000000FA000040EB004C81020086
:10F09000000000000080FA00000006000000FA00F6
:10F0A00010C0B3004C810200000000000080FA0094
:10F0B000000006000000FA0001012000D0982000A6
:10F0C000D69202000000000060AD200010407800E1
:10F0D000CC6902000000000000C2B300446C0200D2
:10F0E0000000000080AE2000104078000080FB008F
:10F0F0004400DE0061406000CC69020000000000B6
:10F1000000C2B300446C0200000000003100200087
:10F1100020AE2000D6920200000000000080FA001D
:10F12000000006000400FA00A01F0200000000001A
:10F13000D21B02000000000010079800A01F020070
:10F1400000000000D21B020000000000000F780049
:10F150001E0090000000E000090034001E00900036
:10F16000E40F500006003C001E0090000040E90043
:10F170008040780060AD2000014878000200370030
:10F180000000EB00100798001E00E00010003400A3
:10F19000200020009E0F10000D003C001E00780093
:10F1A0000040EA006141600080AE2000904078009D
:10F1B000614061004401DD00F0CEB30080C060001A
:10F1C00082C0700080AE2000014878000200370045
:10F1D0000000EB00100798001E0090000000E00007
:10F1E00026003A000000EB0010648800B103200004
:10F1F0008045200060930200000000008001EB00C9
:10F20000420020001100200010002000CC2002004D
:10F21000000000000040E9008040780060AD200060
:10F2200001487800F1042000E09320006093020080
:10F23000000000008001EB002200200011002000EF
:10F2400010002000CC200200000000000040EA0076
:10F250006141600080AE2000904078006140610014
:10F260004401DD00F0CEB30080C0600082C07000B9
:10F2700080AE200001487800010037008DFF0700B4
:10F28000CB02A900CB22A900C922A800C902A9006B
:10F2900060AD20009040780020C0B300E07E020006
:10F2A000000000000080FA00000006000400FA00E0
:10F2B000000F78001E007800100798001E009000D4
:10F2C000E10F50000C0032001E009000E10F5000D2
:10F2D000040039001E009000E20F500007003200C9
:10F2E0000800370081032000D0992000D692020048
:10F2F000000000000700370010000700250007008D
:10F300000400370041022000E01D2000609302004D
:10F31000000000000080FA00000006000200FA0071
:10F32000000F7800B1002000600B21006093020004
:10F33000000000000080FA00000006000000FA0053
:10F34000F1032000509D20006093020000000000A7
:10F350000040EB007081020000000000F00F200070
:10F36000589202000000000010C0B300708102003B
:10F370000000000010C0B300268102000000000061
:10F380000040EB0070810200000000000080FA00E5
:10F39000000006000A00FA00881F7800D102200051
:10F3A00040A12000D6920200000000000000EB0007
:10F3B000000F7800100037001E04780094800200CF
:10F3C000000000008040780063004700017478006E
:10F3D0009E00780063004700614078000080FB00D9
:10F3E0002E6A02000000000000C2B300446C02005C
:10F3F000000000001E0FE800300020009E0F1000EB
:10F40000EDFF3600808828006067020000000000E1
:10F41000A100200010A42000D692020000000000ED
:10F4200063004700104078000080FB004400DE00CD
:10F430000080FB00400798004E009000E90F50004C
:10F44000130032004E009000E90F500004003C0011
:10F450004E009000E80F5000080032001B003700FB
:10F460004E009000EA0F50000E0032004E00900057
:10F47000EF0F500010003200140037006100200030
:10F48000B0A42000D6920200000000001300370054
:10F490006100200010A52000D692020000000000AC
:10F4A0000E0037006100200070A52000D6920200F7
:10F4B000000000000900370031002000D0A5200026
:10F4C000D692020000000000040037007100200006
:10F4D00000A62000D69202000000000080882800CC
:10F4E0006067020000000000B100200070A620004C
:10F4F000D692020000000000630047001040900018
:10F500000080FB004700DE000004E00005003A0038
:10F510006100200020A72000D69202000000000019
:10F5200004003700F100200080A72000D6920200DE
:10F5300000000000808828006067020000000000D2
:10F54000C100200070A82000D69202000000000038
:10F5500063004700104090008080FB0080F72F0080
:10F56000008060004380DE00204798002E4090001D
:10F570000004E00005003A00D100200030A920007E
:10F58000D6920200000000001E0037002E409000BE
:10F59000EF4F500005003A0031002000D0A52000B8
:10F5A000D692020000000000160037000004200080
:10F5B000000F7800E30047000040EB00804878002F
:10F5C000080037001E00780000004000000F78009F
:10F5D00063004700104078008040E8006300470067
:10F5E0000148780063004700904078002E4090006A
:10F5F00080CF5000F3FF39001E0078006E690200D2
:10F600000000000080882800606702000000000001
:10F610009101200000AA2000D69202000000000004
:10F62000630047009040900070C0B30000C06000CD
:10F630002047980010002000000F7800E3004700EA
:10F640000040EB0080487800080037001E0078007A
:10F6500000004000000F7800630047001040780071
:10F660008040E800630047000148780063004700DD
:10F67000904078002E40900080CF5000F3FF39007A
:10F680001E007800CC69020000000000808828007D
:10F6900060670200000000004F0478000080FA005C
:10F6A000000006000000FA0040168000017C2000E7
:10F6B00001007000401688001100070020C0B30050
:10F6C0002D000700666B0200000000000004E0004F
:10F6D00005003200246C0200000000002600070034
:10F6E0000004E00004003A00750107000004E00097
:10F6F00001003A00F3FF37000080FA000000060026
:10F700000000FA00C222A9000000EB0040038800BC
:10F710000000EB00500388000000EB0000038800AD
:10F720000000EB00100388000000EB00F0088800E8
:10F73000D10A200091407800F0C8B30000C06000FA
:10F74000ADE0B7000000EB00E00888000064200096
:10F75000D008880000002100F06A88008040EB009B
:10F76000C0D52000014878000000EB00606A8800E6
:10F770000080FA00000006000C00FA002047980004
:10F780000000EB00000F78001E0078005007980082
:10F79000DE009000E18F5000800032005E0190009A
:10F7A000E10F5100040039005E009000E20F5000AC
:10F7B0008C0032003D0137002E4090000080FB009D
:10F7C00040079800CE009000E28F500018003200F1
:10F7D0004E019000E20F510007003C004E009000E7
:10F7E0000000E0000E003200CE009000E18F5000DB
:10F7F000130032005D0037004E019000F10F510000
:10F800002A0132004E009000F30F50002701320011
:10F81000CE009000E48F50001D00320053003700EE
:10F82000B7FF0700120020003207980021013700BF
:10F830006085280034670200000000001B013700CB
:10F84000C222A8000000EB00F00888000000EB00D6
:10F85000B00888000000EB00A008880080002000AD
:10F86000F00888008660A9009660A900D10A2000EF
:10F8700091407800F0C8B30000C060000044A000D0
:10F88000ADE0B70010002000606A88000701370073
:10F8900010C0B300446C020000000000B0852800D6
:10F8A00034670200000000000040EB00446C0200DE
:10F8B0000000000010C2B300446C02000000000011
:10F8C0000040EB00446C0200000000000040EB0030
:10F8D000446C02000000000000C1B300446C020050
:10F8E000000000000040EB00446C0200000000003B
:10F8F00030C2B300446C0200000000000040EB0086
:10F90000446C020000000000F0C0B300446C020030
:10F910000000000020C4B300446C0200000000009E
:10F9200000C4B300446C02000000000000C4B30037
:10F93000446C02000000000050C0B300446C0200A0
:10F940000000000010C4B300446C0200000000007E
:10F9500020C0B300446C0200000000000040EB0037
:10F96000446C020000000000D0003700E0D420000A
:10F97000AE4090000148780041C0B30030D520006F
:10F98000014878008040EB0040D520000148780015
:10F9900010002000000F7800C400370040D5200080
:10F9A000104078008040E80040D5200001487800F1
:10F9B00040D52000104078008080FB00E0D420007B
:10F9C000008040002E4190000248780040D5200081
:10F9D0009040780030D520001040780080CF500053
:10F9E000B2003900E0D42000104078000080FB0015
:10F9F0002007980010082000AE009000808F500073
:10FA00003E003200000C20002E019000800F5100BB
:10FA10000500320000082000AE009000808F5000EA
:10FA20004E0032009F003700F0D4200010407800D4
:10FA30000080FB004400DE00610060000004E00084
:10FA400003003200100380000000A00010038800B3
:10FA5000F0D42000104078000080FB004300DE005E
:10FA6000610060000004E000040032001003800028
:10FA7000010220000100700010038800F0D4200073
:10FA8000104078000080FB004200DE006100600052
:10FA90000004E00004003200100380000104200094
:10FAA0000100700010038800F0D42000104078009E
:10FAB0000080FB000000D100610060000004E00055
:10FAC00004003200100380000108200001007000D3
:10FAD00010038800F0D42000104078000080FB0064
:10FAE000610060000004E0000400320010038000A8
:10FAF00001102000010070001003880000D52000D4
:10FB0000104078000080FB00F06A8800F06A8000F6
:10FB10004800DD00F06A8800F0D420001040780032
:10FB20008080FB00F06A800000807000F06A88002E
:10FB3000F06A80004200DD0064004000F06A880046
:10FB4000F16A800000002100808F500055003600CF
:10FB500000002100F06A88005200370010D5200014
:10FB6000104078000080FB0001002000B06A88008F
:10FB7000C16A8800B06A8000C16A8000C808DD00E0
:10FB80000080FD00804078000040EB00B06A8800F3
:10FB9000C16A880000D52000104078000081FB0079
:10FBA00003002000B06A8000C16A8000000071007C
:10FBB00081807100B06A8800C16A8800B06A8000E4
:10FBC000C16A8000C808DD000080FD008040780028
:10FBD0000040EB00B06A8800C16A8800F0D42000C1
:10FBE000104078000081FB0003002000B06A800014
:10FBF000C16A80000000710081807100B06A8800D5
:10FC0000C16A8800B06A8000C16A80004209DD00D4
:10FC1000CE00DE00810071004200DD006400400083
:10FC2000E08048009201200003002000240602002A
:10FC300000000000B06A8800C16A8800B26A8000D3
:10FC4000C36A80000001200001002000800F5100E5
:10FC5000818F590007003600B06A8000C16A8000B9
:10FC600070005000E0805800B06A8800C16A8800C7
:10FC7000040037001000200001002000B06A880056
:10FC8000C16A8800B06A8000C16A80004008DE0056
:10FC900001002000E0088800B06A8000C16A80008E
:10FCA000D00888000000EB00000F78000000EB0097
:10FCB000300798003E0090000080FA000000060027
:10FCC0000200FA00606A8000E10F5000010032007B
:10FCD0003600370086C0BF00684060000004E000C6
:10FCE00003003A00100380000000E0002F003A00FB
:10FCF0001FE1A8008780A9000000EB00D06A8800FF
:10FD00000E00370071408000D06A80008080400083
:10FD1000501680004600DE008048780087C0BF0093
:10FD2000704060000004E000FCFF32008780A90002
:10FD3000D06A80000000E800D06A8800D16A8000A4
:10FD4000F06A8000808F5000EEFF39000000EB0069
:10FD5000100388000000EB00F0088800F06A8000C3
:10FD6000D06A88000A00370071408000D06A8000A5
:10FD7000008040000000E90010407800446C020060
:10FD800000000000D06A80000000E900D06A88000E
:10FD9000D06A80000000E000F3FF3A0058FE070040
:10FDA00010002000000F7800020037000000EB0078
:10FDB000000F78001E0078000080FA0000000600A6
:10FDC0000400FA00004F78001147980040D320004B
:10FDD0001E48780030C0B3009E4F100005003A0066
:10FDE00000202000B069880000082000C069880059
:10FDF0000400370000202000B069880000202000A7
:10FE0000C06988001E4090000080FB001007980029
:10FE10001E009000E10F5000110032001E00900003
:10FE2000E20F5000180032001E0090000000E000B9
:10FE3000010032001E00370041C1B300A0D32000F2
:10FE40000148780041C6B300B0D3200001487800D3
:10FE500021C3B300C0D32000014878001D00370043
:10FE600021C0B300A0D3200001487800A1C0B30096
:10FE7000B0D320000148780051C0B300C0D32000A7
:10FE8000014878001300370011C0B300A0D3200050
:10FE90000148780051C0B300B0D320000148780079
:10FEA00021C0B300C0D3200001487800090037000A
:10FEB0008040EB00A0D32000014878008040EB0098
:10FEC000B0D32000014878008040EB00C0D3200070
:10FED000014878000080FA00000006000200FA00E5
:10FEE0000000EB00000F7800B0D3200090407800B5
:10FEF0000030200009010700CBC2BF006140600054
:10FF00000004E00004003200CBC2BF006240600089
:10FF10000004E00002003A0010002000000F78000A
:10FF2000B0D320009040780000202000140107008A
:10FF3000B0D320009040780000102000100107008E
:10FF4000B0D320009040780000202000F30007008C
:10FF50001E0078000080FA00000006000000FA0091
:10FF6000B0D320009040780000302000040107004A
:10FF7000B0D320009040780000102000E700070078
:10FF8000B0D320009040780000202000E30007005C
:10FF90000000EB000080FA00000006000C00FA00F0
:10FFA000500798000000EB00000F780070AD2000B3
:10FFB000104078000080FB008000E9001000200065
:10FFC0000100DD00300798005E00900020079800D7
:10FFD0000000EB004007980020003700A0D320006D
:10FFE00010417800AE0090003E009000008060005C
:10FFF00001202000F3000700B0D3200090407800DB
:020000040001F9
:1000000000102000C50007000008200017010700AD
:100010000080FB0010079800B0D3200090407800CB
:1000200000102000D60007002E00900000004000C5
:10003000200798001E00780000004000000F7800A4
:100040001E0090000000E000010032001E0FE800DA
:100050004E0090000000E8004007980070AD2000BE
:10006000104078008080FB004E009000808F500090
:10007000DAFF3E001E0078000080FA000000060053
:100080000800FA003007980070AD2000104078009A
:100090000080FB008000E900100020000100DD006E
:1000A000100798003E009000000F78000000EB0061
:1000B0002007980014003700A0D3200010417800DA
:1000C0001E0090001E00600001202000BD000700FF
:1000D000B0D3200090407800001020008F0007006F
:1000E000B0D320009040780000102000A40007004A
:1000F0001E00780000004000000F78002E009000E5
:100100000000E8002007980070AD20001040780043
:100110008080FB002E009000808F5000E6FF3E00A4
:100120000080FA00000006000600FA000000EB0064
:10013000000F780000202000CC0007000000EB003A
:100140002007980016003700B0D3200090407800B8
:10015000001020007100070000202000C3000700ED
:100160000080FB0010079800B0D32000904078007A
:1001700000102000820007001E00780000004000F0
:10018000000F78001E0090000000E0000100320027
:100190001E0FE8002E0090000000E80020079800E5
:1001A00070AD2000104078008080FB002E00900091
:1001B000808F5000E4FF3E001E0078000080FA00AF
:1001C000000006000200FA00C0698000A7000700D6
:1001D000B0D3200090407800001020004F000700AE
:1001E000C0698000A1000700004F7800B0D3200054
:1001F0009040780000102000610007001E80FB0086
:100200000080FA00000006000200FA00004F7800AB
:10021000A0D3200010417800B16980001E80FB004F
:1002200068000700B0D32000904078000010200044
:100230003A000700B0D32000904078000010200062
:100240004F0007000080FA00000006000400FA00DA
:10025000204798000040EB00004F7800090037006D
:10026000B0D3200090407800001020002B00070041
:10027000B0D320009040780000102000400007001C
:100280001E4FE8002E4090009E4F1000F4FF3900F2
:100290000080FA00000006000200FA00004F78001B
:1002A000A0D3200010417800B16980001E80FB00BF
:1002B000440007000080FA00000006000200FA0077
:1002C000004F7800A0D32000104178001E80FB0072
:1002D000011020003B0007000080FA00000006002B
:1002E0000200FA00004F7800A0D3200010417800EF
:1002F0001E80FB0001042000320007000080FA008D
:10030000000006000000FA00C069800057000700E6
:100310000080FB000080FA00000006000400FA00E4
:10032000000F78002147980080AE20001040780030
:10033000704060000004E00008003A006016800091
:100340001E007000601688009E80EA004016800043
:1003500000806000401688000300370040168000CF
:100360001E007000401688002E4090000080FB00A8
:1003700058920200000000000080FA000000060011
:100380000400FA00000F7800214798009E80EA00E0
:100390006016800000806000601688009E80EA0081
:1003A0004016800000806000401688002E409000BB
:1003B0000080FB0058920200000000000080FA005C
:1003C000000006000600FA00000F780011079800F0
:1003D000424798001E00E0000B003A001E0090000B
:1003E0008080EA006016800000806000601688004F
:1003F0001E0090008080EA004016800000806000AF
:10040000401688001300370080AE200010407800AE
:10041000704060000004E0000A003A0061168000AD
:100420001E00900000807000601688001E00900082
:100430008080EA004016800000806000401688003E
:1004400004003700401680009E00900001007000FC
:10045000401688004E4090000080FB005892020039
:10046000000000000080FA00000006000400FA000E
:10047000000F7800401680001E00700040168800B3
:100480000000000000000000000000005016800086
:100490001E0060000000E000030032001000200099
:1004A00010079800020037000000EB0010079800CA
:1004B0001E0090000080FA00000006000000FA0014
:1004C0000088280034670200000000000080FA0065
:1004D000000006000A00FA00704080003007980013
:1004E00010002000106B8800F4FF070000003700A8
:1004F000246C020000000000104798001E4090008D
:100500000080FB0040079800CE009000E38F500071
:10051000200032004E009000E30F50000A003C0023
:10052000CE009000E18F50005B0032004E00900042
:10053000E10F50005E003C00CE0090000100E000A2
:10054000E7003200DB0037004E009000E60F50005D
:100550000E003200CE009000E68F500004003C00F8
:100560004E009000E50F500095003200D10037009A
:10057000CE009000E78F5000640032004E009000E3
:10058000E80F500054003200CA003700CBFF0700CC
:10059000D7FF3700BE00900030C0B300804878001D
:1005A0003E0090008000E80080C0B30080487800E2
:1005B00021E3A800C0C0B300FC90020000000000CE
:1005C000200798003E0090008080E8002E009000F8
:1005D0004800DE00804878003E009000E3004000C4
:1005E0002E00900080487800B0C0B300FC9002005C
:1005F00000000000200798003E009000E40040004A
:100600002E0090004800DE00804878003E009000F8
:10061000E50040002E00900080487800A0C0B300A4
:10062000FC90020000000000200798003E009000AF
:10063000E60040002E0090004800DE008048780070
:100640003E009000E70040002E00900080487800B7
:1006500090C0B300FC90020000000000200798004A
:100660003E009000E80040002E0090004800DE00B0
:10067000804878003E009000E90040002E00900085
:100680008048780021E3A900A10020003E009000EE
:10069000BF00070096FF3700246C02000000000036
:1006A000104798001E4090008F00070090FF370011
:1006B000246C02000000000010479800246C020027
:1006C00000000000004F78009E4078001E4090001F
:1006D000C100070086FF3700246C02000000000004
:1006E00010479800246C020000000000004F7800C2
:1006F0001E4090000080FB00C800DD001E80FB0053
:1007000000807000106B880079FF3700246C0200B5
:1007100000000000104798001E4090000080FB0081
:10072000200798001E409000E14F500004003A005E
:1007300030C0B300626C020000000000030037000C
:1007400020C2B300626C020000000000246C0200B2
:100750000000000010479800246C02000000000018
:10076000004F78009E409000A0CAB30080CF500098
:1007700003003A0050C5B3009E4F10000500320040
:100780000000EB002007980020C2B300626C02005A
:1007900000000000BE00900070C0B30080487800E8
:1007A0003E0090008000E8002E0090008048780015
:1007B000210020003E009000750007004CFF37002C
:1007C000246C02000000000010479800246C020016
:1007D00000000000004F78008560A9001E409000D6
:1007E0000080FB00C800DD001E80FB000080700060
:1007F000100798009E00900000002200808F50009B
:100800000200360000002200100798001E00900031
:10081000670040004300DE0020079800BE00900003
:1008200050C0B300804878003E0090000000E8000F
:100830009E409000014878003E0090000080E80053
:100840001E487800310020003E0090005000070054
:1008500070408000004088002E00900000004000A2
:10086000104088000000EB002040880071408000AC
:100870004083200000804000304088000000EB00F2
:10088000404088000000EB00504088009560A800C0
:10089000106B8000314080000440800080017800AF
:1008A0001E0190000400780036970200000000004E
:1008B0000FFF3700BE0090000040EB00804878003A
:1008C0003E0090008000E8000040EB008048780087
:1008D000110020003E0090002D00070004FF3700AB
:1008E0000080FA00000006000200FA00004F7800C5
:1008F000CAC2A900CB22A900CB02A900CB42A90001
:10090000CA02A90020C0B3009E4F100006003A00A2
:10091000CAC2A800CB02A800CB22A800CB42A800E4
:10092000CA02A80005003700CAC2A900CB02A9006C
:10093000CB22A900CB42A900CA02A90010C0B30073
:100940009E4F10000300320020C0B3009E4F1000E5
:1009500007003A00C8C2A900C922A900C902A9001B
:10096000C942A900C802A900C8E2A80006003700D1
:10097000C8C2A800C922A800C902A800C942A8008C
:10098000C802A800C8E2A8000080FA000000060023
:100990000600FA0010079800210798000000EB00FD
:1009A000000F7800070037009E0078001E009000BE
:1009B0000080400010407800446C020000000000FD
:1009C0001E0FE8002E0090009E0F1000F6FF390069
:1009D0000080FA00000006000400FA00004F7800D2
:1009E000114798001E80FB00100798001E00900021
:1009F000E40F50002F0032001E009000E40F500062
:100A000007003C001E009000E10F50000B00320078
:100A10001E009000E20F5000140032003900370031
:100A20001E009000E80F50002C0032001E009000C5
:100A3000F00F50001600320032003700C022A9002B
:100A40001E40900061406000614060000041400035
:100A5000212C200091407800D0CFB30000C060006E
:100A600002407000C2E2B700260037001E4090002E
:100A70000004E00003003200C002A900C202A80086
:100A800020003700C002A900C202A9001D003700E3
:100A90001E4090000004E00003003200C962A8007C
:100AA000CB62A90017003700CB62A900C962A90078
:100AB000140037001E4090006140600061416000FA
:100AC000A12C200091407800E0CFB30000C060006E
:100AD00002407000CAE2B7000A0037001E409000D2
:100AE00061406000614060004201DD00B12C2000E7
:100AF00091407800B0CFB30000C0600002407000A9
:100B0000CBE2B7000080FA00000006000200FA0005
:100B1000000F78001E0078008040780000D620008A
:100B2000104078000080FB000000D10061406000B0
:100B300044010700001020000080FA0000000600B9
:100B40000000FA0000D62000104078000010A1003C
:100B500001D62000804878004101200050EE20009E
:100B600060930200000000000080FA000000060010
:100B70000000FA0000D62000104078000010A0000D
:100B800001D62000804878002101200090EF20004D
:100B900060930200000000000080FA0000000600E0
:100BA0000000FA0080AE2000104078000040A00055
:100BB00081AE20008048780000D6200010407800E8
:100BC0000010A00001D6200080487800816A200033
:100BD0009140780000CEB30000C060007040B300C8
:100BE000A8E6B700916C20009140780000CEB300D9
:100BF00000C060007040B300C9E6B700816C2000FF
:100C00009140780000CEB30000C060000034A00026
:100C1000C8E6B700CAC2A900C8C2A900C902A90093
:100C2000C8E2A800C922A900D01320001012880031
:100C30000000EB00201288000000EB00001288008A
:100C400041E2A800D1012000E0F120006093020001
:100C5000000000000080FA00000006000800FA0012
:100C600020079800006480008000E800F00F20005A
:100C70000080600000648800A01F020000000000E7
:100C8000D21B020000000000100798000000EB00DB
:100C9000106488002E009000300798003E009000FD
:100CA000E30F50003C0032003E009000E30F500084
:100CB00004003E003E0090000000E0000B00320007
:100CC0000F0037003E009000E60F50004800320051
:100CD0003E009000E70F50006A0032003E00900096
:100CE000E40F5000370032008B00370081092000EC
:100CF00000F8200060930200000000008A00370026
:100D000051002000506020006093020000000000AD
:100D1000AC0007002E009000E10F5000820032006E
:100D20001E0090000000E000030034001E00900050
:100D3000E20F500013003400410220008001210026
:100D400060930200000000008001EB002200200000
:100D50001100200020002000CC2002000000000034
:100D6000100798001E009000E10F500003003A00A9
:100D70000040EB00750007000200370080C0B300A0
:100D80007200070041002000C003210060930200B0
:100D9000000000006400370011C0B3000040EB0009
:100DA000A8000700F00020002C92020000000000C4
:100DB00051002000000421006093020000000000A8
:100DC000590037001E0090008040780000C8B30032
:100DD00080C070000040EB009A000700A1002000D6
:100DE0005004210060930200000000004E00370014
:100DF00011C0B3000040EB0092000700F00020009B
:100E00002C92020000000000000320002007980040
:100E10001E0090000000E00002003A0000052000E3
:100E2000100798000000EB00000F78001100370059
:100E3000AE00900090032000808F5000020036002A
:100E400000032000200798002E00900080407800CA
:100E500010C0B3007B0007002E009000446C02001D
:100E6000000000002E0090000000E800200798001D
:100E70001E0FE8001E0090009E0F1000ECFF3500D2
:100E80002900370011C0B3000040EB006D000700DF
:100E9000F00020002C920200000000001002200050
:100EA000200798001E0090000000E00002003A00B9
:100EB00000052000100798000000EB00000F7800EC
:100EC00011003700AE009000F0072000808F500026
:100ED0000200360010022000200798002E0090002B
:100EE0008040780010C0B300560007002E0090002C
:100EF000446C0200000000002E0090000000E8009A
:100F0000200798001E0FE8001E0090009E0F1000A2
:100F1000ECFF35000400370041022000E01D2000F6
:100F200060930200000000000080FA00000006004C
:100F30000000FA00B1002000600B21006093020065
:100F4000000000000080FA00000006000200FA0025
:100F5000004F78001E4078000042B00080407800CA
:100F60000040EB0037000700F00020002C92020048
:100F70000000000081C0B3000040EB00310007001A
:100F8000F00020002C9202000000000011C0B3000D
:100F90000040EB002B000700F00020002C92020024
:100FA00000000000E1C0B3000040EB002500070096
:100FB000F00020002C920200000000000080FA00E7
:100FC000000006000000FA000040EB004A000700A5
:100FD000F00020002C9202000000000031C0B3009D
:100FE0000040EB0026000700500020002C92020079
:100FF0000000000031C0B3000040EB0020000700FB
:10100000000A2000589202000000000031C0B30026
:101010000040EB001A000700000A2000589202006E
:101020000000000021C0B3000040EB0014000700E6
:10103000000A200058920200000000000080FA0020
:10104000000006000200FA00004F780011479800E7
:101050001E4090000080FB004400DE0080407800CD
:101060001E407800060007001E409000EF40600020
:101070001E407800020007000080FA000000060011
:101080000200FA00004F7800114798001E409000BF
:101090004400DD00104798001E4090000004A000AE
:1010A0001047980010C0B3009E4F100003003A0094
:1010B0001E4090000014A000104798001E409000B1
:1010C0000D0007001E4090000034A000104798005B
:1010D0001E409000080007009E40900070CFB300B3
:1010E00000C06000104798001E40900002000700FA
:1010F0000080FA00000006000200FA00004F7800AD
:101100001E4078001E48020000000000CAC2A8006D
:10111000CAC2A9000080FA00000006000000FA0020
:10112000F00F2000CE7F0200000000000080FA00D7
:10113000000006000400FA00000F78001E0078008E
:10114000CE7F020000000000000F780080AE20007B
:10115000104078000044B2000004E00003003200B8
:101160001E00780010079800020037000000EB0016
:10117000100798001E0090000080FA000000060092
:101180000000FA0080AE2000104078000060A0004F
:1011900081AE20008048780000AF20001040780029
:1011A000614060000004E000040032000040EB00F9
:1011B00070810200000000000300370010C0B3007F
:1011C000708102000000000000AF20001040780095
:1011D000614060000004E00003003200F0C2B30090
:1011E000446C020000000000A100200090AB200031
:1011F00060930200000000000080FA00000006007A
:101200000000FA0080AE2000104078000060A100CD
:1012100081AE20008048780000AF200010407800A8
:10122000614060000004E000040032000040EB0078
:1012300070810200000000000300370010C0B300FE
:10124000708102000000000000AF20001040780014
:10125000614060000004E00003003200F0C2B3000F
:10126000446C020000000000A100200090AB2000B0
:1012700060930200000000000080FA0000000600F9
:101280000000FA0080AE2000104078000060A1004D
:1012900081AE20008048780000AF20001040780028
:1012A000614060000004E0000400320010C0B300A0
:1012B0007081020000000000030037000040EB00D6
:1012C000708102000000000000AF20001040780094
:1012D000614060000004E00003003200F0C2B3008F
:1012E000446C020000000000B100200030AC20007F
:1012F00060930200000000000080FA000000060079
:101300000000FA00E2800200000000000080FB0004
:101310000080FA00000006000000FA00828102004E
:10132000000000000080FB000080FA0000000600C2
:101330000000FA0010C0B300268102000000000087
:101340000080FA00000006000000FA0010C0B300A0
:101350005E810200000000000080FA00000006002C
:101360000000FA000040EB005E8102000000000077
:101370000080FA00000006000000FA0010C0B30070
:101380004C810200000000000080FA00000006000E
:101390000000FA000040EB004C8102000000000059
:1013A0000080FA00000006000000FA004101200061
:1013B000E0AC2000D69202000000000060AD2000EA
:1013C00010407800CC6902000000000000C2B300A9
:1013D000446C02000000000000AF200010407800C4
:1013E00061406000CC6902000000000000C2B30050
:1013F000446C02000000000080AE20001040780025
:101400000080FB004400DE0061406000CC69020007
:101410000000000000C2B300446C020000000000A5
:10142000A088280060670200000000000080FA0029
:10143000000006000600FA00A01F020000000000E5
:10144000D21B02000000000020079800A01F02002D
:1014500000000000D21B020000000000000F780016
:10146000A01F020000000000D21B020000000000CC
:10147000100798002E0090000000E00009003400E2
:101480002E009000E40F500006003C002E0090005B
:101490000040E9008040780060AD200001487800FD
:1014A000020037000000EB00200798001E00E0005B
:1014B0000F003400200020009E0F10000C003C00A4
:1014C0001E0078000040E900E140600000AF20000D
:1014D0001040780061C16000E1CFB30001406000BE
:1014E0000240700001AF2000804878000200370001
:1014F0000000EB00200798001E0090000000E000B4
:10150000100034001E009000E20F50000D003C005F
:101510001E0090000040EA006141600080AE2000A3
:1015200090407800614061004401DD00F0CEB300DE
:1015300080C0600082C0700080AE2000014878004A
:10154000020037000000EB00200798002E009000FA
:101550000000E0003A003A00B1032000804520007E
:1015600060930200000000008001EB0042002000B8
:101570001100200010002000CC200200000000001C
:101580000040E9008040780060AD2000014878000C
:10159000D1012000601C21006093020000000000C7
:1015A0008001EB002200200011002000200020001C
:1015B000CC200200000000000040E900E140600093
:1015C00000AF20001040780061C16000E1CFB3009F
:1015D000014060000240700001AF200080487800A8
:1015E000F1042000E093200060930200000000005E
:1015F0008001EB00220020001100200010002000DC
:10160000CC200200000000000040EA0061416000C0
:1016100080AE200090407800614061004401DD0010
:10162000F0CEB30080C0600082C0700080AE2000A9
:10163000014878000000EB001064880001003700CA
:1016400059FF070080AE2000104078000060A10024
:1016500081AE20008048780080AE200010407800E5
:101660000050A10081AE20008048780060AD2000CD
:101670009040780030C0B300E07E0200000000001F
:10168000C922A900C902A900C8E2A80000AF200031
:10169000104078006140600070810200000000008E
:1016A0000080FA00000006000000FA00010120009E
:1016B0004006210060930200000000000080FA0054
:1016C000000006000200FA00004F78001147980061
:1016D0008040EB0020D32000014878001E04E00089
:1016E00003003A00D04080000080A000D040880075
:1016F0001E04E000110032001E4090000004E000D3
:101700000E003200F103200050AE20006093020072
:101710000000000011012000A019210060930200C8
:1017200000000000666B0200000000000004E00002
:10173000FCFF3200246C0200000000004100200089
:1017400040B220006093020000000000CB42A800DD
:10175000C942A9003100200080B22000D6920200C8
:1017600000000000CBC2BF000080FB004200DE0092
:101770006140600011C0B30011010700CB42A90015
:10178000C942A800C222A800C022A90081002000EE
:10179000B0B22000D692020000000000C2C2BF001A
:1017A0000080FB000000D1006140600011C0B30068
:1017B00003010700C222A900C962A800CB62A900E8
:1017C0008100200030B32000D6920200000000000B
:1017D000CBC2BF000080FB004300DE006140600020
:1017E00011C0B300F6000700CB62A900C962A900CE
:1017F00081002000B0B32000D6920200000000005B
:10180000CBC2BF000080FB004300DE0061406000EF
:101810008040EB00EA000700C002A900C202A80055
:10182000200020002C920200000000004100200057
:1018300030B42000D692020000000000C2C2BF00F7
:101840006140600011C0B300DD000700E10020002E
:1018500070B42000609302000000000021E3A800A3
:101860002100200050B52000D692020000000000A8
:1018700072352000712B200090C0B3008600070055
:101880001E4090000004E0000800320031002000FB
:1018900070B52000D69202000000000072352000D2
:1018A000712B2000B0C0B3007B0007004100200076
:1018B000A0B52000D6920200000000000225200002
:1018C000011B2000A0C0B300730007001E40900061
:1018D0000004E0000800320031002000E0B52000E4
:1018E000D69202000000000002252000011B20000B
:1018F000C0C0B3006800070021E3A90081002000F8
:1019000010B6200060930200000000004116800025
:10191000F0C32F0000806000401688006116800030
:10192000003C200000807000601688004006200007
:101930002C9202000000000010C0B30077000700E6
:10194000A100200090B6200060930200000000007B
:1019500061168000F0C32F000080600060168800D0
:101960001E4090000004E00002003200C962A8009E
:10197000CB62A900400620002C920200000000006B
:101980000040EB00650007001E4090000004E000EE
:101990000D003200A100200030B72000609302004B
:1019A0000000000040168000013C20000100700093
:1019B00040168800400620002C9202000000000023
:1019C00010C0B300550007001E04E0001C003200E8
:1019D0001E4090000004E00019003200C002A9007F
:1019E000C202A800201680000010A0002016880067
:1019F00001022000D0B72000609302000000000028
:101A0000F1002000B01821006093020000000000E7
:101A1000666B0200000000000004E000FCFF3200E2
:101A2000246C02000000000020168000D1FF2F006F
:101A30000100600020168800C002A900C202A900AF
:101A4000B29002000000000061002000D0B9200028
:101A5000D69202000000000020D320001040780041
:101A6000CC690200000000008100200030BA200094
:101A70006093020000000000D04080000080A100C0
:101A8000D040880020D32000104078000080FB0068
:101A90000080FA00000006000A00FA0020479800C3
:101AA000210798003207980080C2B300446C0200FE
:101AB000000000002E409000FC900200000000009A
:101AC000000F78001E007800D06A020000000000BD
:101AD00090C2B300446C0200000000002E00900091
:101AE0009E0F1000060036003E0090009E0F100072
:101AF000030031001000200040079800020037006A
:101B00000000EB00400798000E48900011C0B300A1
:101B10002B0007000080FA00000006000200FA0017
:101B2000004F780041002000B0BA2000D692020099
:101B300000000000CBC2BF000080FB000000D1000D
:101B4000614060009E4078001D00070031002000C9
:101B5000F0BA2000D692020000000000CBC2BF0005
:101B6000614060009E4078001500070041002000A1
:101B700020BB2000D692020000000000CAC2BF00B5
:101B80000080FB004700DE009E4078000C0007004C
:101B90002100200060BB2000D6920200000000005F
:101BA000CAC2BF000080FB004600DE00614060004A
:101BB0009E407800020007000080FA000000060046
:101BC0000200FA00004F7800114798001E40900074
:101BD0009E4F100005003A003100200080BB20001D
:101BE000609302000000000009003700510020004F
:101BF000B0BB2000609302000000000020D3200052
:101C0000104078008040E80020D320000148780090
:101C10000080FA00000006000C080000120000001E
:101C200002000000000064000D0000000000000041
:101C3000000000000000000000000000D60A0000C4
:101C40001A00000000000000640D000000100000F9
:101C500000000000F00A0000020000000000000088
:101C60001E0800000C0000000200000000181C000C
:101C70001D0018001C1D030008101800F20A0000C7
:101C80000600000000000000F80A00000800000044
:101C9000000000002A08000002010000020000000D
:101CA000F0005E00BCE261003FDD8300C29C7E006C
:101CB00020A3FD001F419D00C3217F00FCA2400026
:101CC0001E5F0100E3BD3E006082DC00237D9F00BB
:101CD000C1421C00FEA0E100BF5D030080DE3C00AD
:101CE00062BEE000025CDF0081633D007C22C00038
:101CF0009E1D4300A1FF460018FAA40027799B000F
:101D0000C584DA003866E500BB590700DB8567004B
:101D100039BAE4000658190047A5FB007826C4002C
:101D20009A653B00D98704005AB8E600A7F91B0062
:101D300045C698007A24F800A6441A0099C72500E1
:101D40007B3A640086D85B0005E7B9008CD230008E
:101D50006EEDB300510F4E0010F2AC002F719300E6
:101D6000CD114F00ADF370002ECC9200D38D6F00DB
:101D700031B2EC000E50AF00F1134D00CE90720066
:101D80002C6D3300D18F0C0052B0EE00326C8E00FF
:101D9000D0530D00EFB1F000AE4C120091CF2D00EA
:101DA00073CA94007628AB00F51749000856B400B2
:101DB000EA693700D58B570009EBB50036688A0011
:101DC000D495CB002977F400AA481600E9B755004E
:101DD0000B88D600346A2B007597C9004A14F600A8
:101DE000A8742A00C89615004BA9F700B6E80A00A7
:101DF00054D789006B350000000B00007000000014
:101E000000000000700B00000E0000000000000049
:101E10002C09000070010000020000001296120060
:101E20009612960012962400963A96001296120088
:101E30009612960012963A00961296003A963A003A
:101E4000964E960062967800968E96009C96480074
:101E5000695A00000000000000B85200B852120099
:101E6000961296003C4F2E004F1296001296880054
